:020000040000FA
:040000006FD00400B9
:101000006F00507B000000000000000090200020D6
:10101000AA220020A9BDF9F56C23002000000000E1
:10102000000000006C230020902000200000000041
:101030000000000090200020000000009020002010
:101040000000000090200020902000209020002030
:101050009020002090200020242F00205E240020DB
:101060000000000090200020902000200424002098
:1010700090200020D22300209020002090200020EB
:101080009020002090200020902000209020002020
:101090009020002001A04111B7170040985F3AC688
:1010A000945F3247E39CE6FE3245410182800111A4
:1010B00013078008F337078093F787083EC20100C3
:1010C0000100B7170040930570052380B70413068D
:1010D00080FA2380C7040100010083C6B70493F699
:1010E000F60DA385D704238007049246F3A6068055
:1010F0000100010093760502D5CEF336078093F602
:10110000860836C4010001002380B7042380C70489
:1011100001000100B70614007D89558D88C70100C4
:1011200001000100010023800704A246F3A6068007
:101130000100010073370780137787083AC6010062
:1011400001002380B7042380C704010001000100CF
:1011500001003727004093061005A303D7802380A2
:101160000704B247F3A70780010001009307800836
:10117000F3B7078093F787083ECE01000100B71749
:101180000040130770052380E704130780FA2380CB
:10119000E7040100010003C7B70413670708A3852C
:1011A000E70423800704F247F3A70780010001004A
:1011B0000561828093760504BDC6F336078093F6F9
:1011C000860836C8010001002380B7042380C704C5
:1011D00001000100B7061400938606047D89558D31
:1011E00088C7010001000100010023800704C246F6
:1011F000F3A6068001000100733707801377870884
:101200003ACA010001002380B7042380C70401000B
:1012100001003727004093062005A303D7802380D1
:101220000704D24781B773370780137787083ACC12
:10123000010001002380B7042380C70401000100DE
:1012400098471367070C98C723800704E24719BF24
:101250000111814601468145114506CE97000000E7
:10126000E780005593078008F3B7078093F7870856
:101270003EC601000100B717004013077005238028
:10128000E704130780FA2380E7040100010003C785
:101290006704136717002383E70423800704B2471A
:1012A000F3A7078001000100F2400561828041112F
:1012B000814601468145114597000000E780404F77
:1012C00013078008F337078093F787083EC40100AF
:1012D0000100B7170040130670052380C70493066A
:1012E00080FA2380D70401000100FD552396B70240
:1012F00023800704A245F3A5058001000100733790
:101300000780137787083AC6010001002380C704CD
:101310002380D7040100010003C767041367170087
:101320002383E70423800704B247F3A70780010063
:10133000010001A0BD473305F50201007D1575FDD3
:101340008280411122C426C206C6AA8401446317C2
:101350009400B24022449244410182800504130566
:10136000803E420497000000E78000FD4180C5B741
:101370009305000273A04580824573901534924016
:101380002242B2424243D2436244F2440255925551
:101390002256B2564257D2576258F25806499649D9
:1013A000264AB64A464BD64B664CF64C065D965DD1
:1013B000265EB65E465FD65F09617300203041113C
:1013C000B7170040985F3AC6945F3247E39CE6FE49
:1013D000324541018280B71700401307000323887C
:1013E000E702854717170000232EF74273002030CD
:1013F000411122C406C637040020976000E0E78050
:1014000020E21C408297D5BF373700408347470012
:101410009146BD8B6389D70099466394D700834773
:101420005740730020309736000083C6662C9387A0
:10143000160017360000230DF62A0347870097375A
:1014400000009387E71AB6972380E700B7E7040008
:10145000BC4F0946894517150000034565F482977E
:10146000C9B7B787004003C76700098B6309071036
:1014700003C777009306000313770703630DD708AC
:10148000173800000348586217360000130606613B
:101490000547B30606012380E60083C577001737AA
:1014A000000013072760429793F5F50F2300B7005C
:1014B00003C58700973500009385855EC295137537
:1014C000F50F2380A5000347070089451377F7032D
:1014D000630CB70C63E7E50A6306071A8545630CDE
:1014E000B7129737000083C7375C3307F60003470E
:1014F00007001377F70F19CB850793F7F70F0D4701
:101500006363F71A17370000A300F75AB787004044
:1015100009472383E700B787004083C77700E207C6
:10152000E18763DE07049737000083C7F757173753
:1015300000001307A7563E9785462300D7001737AC
:101540000000130727563E97930600032300D70099
:10155000173700001307C7543E97A146850723009D
:10156000D70093F7F70F0D476364F71417370000A0
:10157000A30CF752B787004009472383E7007300A5
:101580002030930610026300D70E930620026305F5
:10159000D70693060002E316D7F403C72702137792
:1015A000C70F13672700D5A803C767001377070481
:1015B00065CB03C7A702173800001308A82F1735FB
:1015C00000001305E526134707082385E70203C734
:1015D000A7021377370F136787002385E702814738
:1015E00013070004B305F5008C41B306F80091071A
:1015F0008CC2E399E7FEF5B503C7A70213470704BA
:101600002385E70203C7A7021377C70F13672700D5
:101610002385E702F9B503C767001377070449C3B9
:1016200003C76702173800001308881C173500002D
:101630001305C513134707082383E70203C767028F
:101640001377370F136787002383E7028147130758
:101650000004B305F5008C41B306F80091078CC275
:10166000E399E7FEBDBD03C7670213470704238361
:10167000E70203C767021377C70F136727002383A7
:10168000E70285B503C767001377070411CB03C7CB
:1016900027021377370F136787002381E70291B57D
:1016A000238006003DBD97370000A38F073EB9BDDC
:1016B00097370000A38A073E75BD230304801547B2
:1016C0002303E48001002302A480828083076480D6
:1016D000E3CE07FE23030480828083076480E3CE89
:1016E00007FE03454480828083076480E3CE07FEC3
:1016F0002302A4808280411126C44AC24EC006C67D
:101700001377F50BAD47AA892E899544630CF70032
:10171000194597000000E78080FA97000000E780F5
:1017200020FB8D444E8597000000E78040F9FD596D
:10173000FD1463983401B240A24412498249410128
:101740008280135509011375F50F97000000E7809B
:10175000E0F92209F1BF011126CC06CEB70408003A
:1017600097000000E780C0F6154597000000E7806D
:1017700000F597000000E78080F697000000E78002
:1017800000F62AC697000000E78080F43245937780
:10179000150089EB136515001375F50FF240E2444F
:1017A00005618280FD14E9F00145CDBF397126DC69
:1017B0004ADA4ED852D656D45AD25ED006DE62CE1F
:1017C00066CCB7E700E07D5783AA070022C603AACC
:1017D000470023A0E71823A2E718B7170040130714
:1017E00070052380E704130780FA2380E70483C78A
:1017F0004704930B75FFB684E20793FBFB0F854606
:10180000AA892E8B328937240040E187015763FA79
:1018100076016308D5008946130700026313D500DB
:101820000157D98F93F7F70FB71C00402382FC04B0
:1018300011472303E4801305F00F97000000E780B1
:1018400000E8094C97000000E78080E863657C159C
:10185000B7050700DA9537870700795563FEE50479
:10186000B3879500636AF704370B0800A94733EB89
:1018700065016395F90881E8814497000000E780DD
:1018800020E5268515A8DA85094597000000E78040
:10189000C0E605090345F9FFFD14050B970000009C
:1018A000E780C0E481C49377FB0FE5F79700000061
:1018B000E780A0EA69F17D55B7170040130770056E
:1018C0002380E704130780FA2380E70403C7470453
:1018D000418B2382E704F250B7E700E023A05711C1
:1018E00023A24711E25432445259C259325AA25AE1
:1018F000125B825B724CE24C21618280A547639B44
:10190000F90685691309F00FB3069900B3742B012A
:10191000B6941349F9FFB3749900856B3379690163
:10192000416B9387F9FFB3F7270199E363FC340117
:1019300093D94900C147E3E637FF3DBF0569C16957
:101940007D19D9B71305800D63886901130500025D
:101950006384790113051008CA8597000000E780A9
:10196000C0D997000000E78040DF31D54E99B3849D
:1019700034416DBFDA852D4597000000E780E0D740
:10198000CA94E30B99EE050997000000E78020D583
:10199000A30FA9FEFDB79387F9FF93F7F70F636DC8
:1019A000FC0C83C71C04130730086315F7063707C0
:1019B00008006361EB06B3079B00B706100063FBEA
:1019C000D704334BEB0089476399F9068980D549E1
:1019D000E38404EADA85094597000000E780E0D156
:1019E00011090327C9FF91472320E480030764807E
:1019F000E34E07FE23033481FD17EDFBFD14110BAD
:101A000081C49377FB0FE9FF97000000E780E0D4E3
:101A100061F155B5B717004003C75704B707080071
:101A20001377070219E3B78707007955E376FBE8D8
:101A300033079B00E3F9E7F841B58547E380F9F008
:101A4000DA852D4597000000E78020CB9389F4FFCD
:101A5000E38404E297000000E78060C893F7390050
:101A600091EB832604800327090093074900E3963E
:101A7000E6E03E89CE84D9BFB5476399F9001305E6
:101A8000900B97000000E78080C3FDB3B1471305BA
:101A9000B00AE388F9FE99476397F904B70508008F
:101AA000B365BB002D4597000000E78000C5814469
:101AB0008D4BA14997000000E78060C263967401D6
:101AC000832704802320F9008504E39534FF8327CE
:101AD000048013172B01635507002312F90069BB1B
:101AE0002322F90051BB9D47639FF90281451305ED
:101AF000B00497000000E78040C0BD4423200900E7
:101B000023220900FD5997000000E78040BD93F7AC
:101B10007400CA9703C70700FD14398D2380A700FE
:101B2000E39334FF91BBA1476397F9069700000048
:101B3000E780A0C28144630D0B008D479304C0036E
:101B40006308FB009304000563048B0193044004C5
:101B50001375C507E30295D2194597000000E78089
:101B600000B697000000E780A0B60545970000008A
:101B7000E780E0B4268597000000E78020B709459C
:101B800097000000E78080B697000000E780E0BC87
:101B9000E31405CE0DB39147639FF900130560066A
:101BA00097000000E780A0B197000000E78040B2F6
:101BB00013059009F9B5E38109CCF1547DB9BD66EF
:101BC0000147173600001306660B938606A6854567
:101BD0008347060093F7F70F91C382800507E3F967
:101BE000E6FE97370000238BB708DDB77D16620647
:101BF000618693178601E18763D4070001458280DF
:101C0000931726003307F500AE9718439C4363E70C
:101C1000E7007D16E37FF7FC7D55828005458280D5
:101C2000FD15E205E18513978501618793F7F50FAF
:101C300063480700FD15139725002A97584365D779
:101C4000138517006205618582803308B5021C4246
:101C500083A80600B335B502C29733B50701AE9825
:101C6000469585486367B5006394A50063E3070163
:101C700081480C43C6950CC388C21CC28280814730
:101C80001397870161876343B7008280139727000A
:101C90002A97232007008507E5B7814701479396D8
:101CA0008701E18663C5B6001335170082809396DD
:101CB0002700AA9694428507558FD5B793D75540EC
:101CC0008A07AA979C4305453315B5007D8D828010
:101CD00017F3FFDFE702A33D2A8497000000E780A7
:101CE00060F405C5931725003E940327C4FF814780
:101CF00011EB7D1516053E954205418517F3FFDF73
:101D00006700233D05838507E5B70145C5BF8147CA
:101D10001397870161876343C70082801397270069
:101D2000B386E50094422A97850714C3D5B77D167C
:101D300062066186014793178601E18763D5070034
:101D400013351700828093172600B306F500AE976F
:101D500094429C437D16B58F5D8FF1BF8A05AA958D
:101D600001476363B500828083A6C5FFF11593D751
:101D70001600D98F9CC11397F601E5B72A83014855
:101D8000014701456343D7008280B387050183A8DB
:101D90000700B30706019C43C697AA976384F8001F
:101DA00033B517010507B3080301620723A0F80044
:101DB00061871108C1BF2A8301478147014563C379
:101DC000D70082803388E50083280800330EE600C0
:101DD000032E0E003388A8403308C84163840801ED
:101DE00033B508018507B308E300E20723A0080123
:101DF000E1871107E9B717F3FFDFE702432B011172
:101E0000B286B2842E86AA850A8597000000E780F4
:101E1000C0FA2A84A6850A8597000000E78020E89A
:101E200033348000060413351500018D056117F366
:101E3000FFDF6700032A17F3FFDFE702C324411126
:101E4000AA89AE8A328BB68402C202C402C6014499
:101E5000131C8401135C8C4163499C02939B140006
:101E6000FD1B0549138CF4FFF15C33048901620406
:101E700061846340740792478E04CE9423AEF4FECF
:101E8000410117F3FFDF6700832313192400B30B0D
:101E90002B01014A93172A00D69783A50B0088438C
:101EA00078003400500097000000E78040DA050A0F
:101EB00093178A01E187F11BE35EFCFC92474E9980
:101EC00005042320F900A2473EC2B24702C63EC421
:101ED00041B7131A8901135A8A41131D240093171D
:101EE0008A01E18763CF970092470A044E941CC091
:101EF000A24705091379F90F3EC2B24702C63EC494
:101F0000ADB7B3079A0313152A0056950841780018
:101F100034005000050AEA97DA978C4397000000D6
:101F2000E780E0D26DBF0000197106C212C416C668
:101F30001AC81ECA22CC26CE2AD02ED232D436D6E9
:101F40003AD83EDA42DC46DECAC0CEC2D2C4D6C6D9
:101F5000DAC8DECAE2CCE6CEEAD0EED2F2D4F6D6C9
:101F6000FAD8FEDA971500009385458B8841E70083
:101F7000050092402242B2424243D2436244F244BC
:101F8000025592552256B2564257D2576258F258CD
:101F900006499649264AB64A464BD64B664CF64CFD
:101FA000065D965D265EB65E465FD65F096173008C
:101FB00020300000972100209381C1041751002098
:101FC0001301418417F5FFFF130505049705002051
:101FD00093854503171600201306C6FD63FAC50056
:101FE0008322050023A0550011059105E3EAC5FEF3
:101FF00017050200130585D197150020938585FBF1
:10200000171600201306066563FAC5008322050033
:1020100023A0550011059105E3EAC5FE1715002020
:102020001305456397450020938545116377B500F7
:10203000232005001105E36DB5FEFD42739002BC3F
:102040008D4273904280B722000093828288739001
:102050000230970200209382E2FA93E232007390FA
:102060005230975200009382A296739012346FB050
:10207000347973002030397101436EC619A039716B
:1020800041536AC866CA62CC5ECE19A03971015349
:102090005AD056D252D44ED64AD826DA22DC06DEA0
:1020A00033016140828241114AC026C222C406C661
:1020B0008282B24D4101024D924C224CB24B410101
:1020C000024B924A224AB2494101024992442244B7
:1020D000B240410182803D432A876373C3029377F4
:1020E000F700BDEFADE5937606FF3D8ABA960CC3C7
:1020F0004CC30CC74CC74107E36BD7FE11E282808B
:10210000B306C3408A069702000096966780A60031
:102110002307B700A306B7002306B700A305B7003F
:102120002305B700A304B7002304B700A303B70037
:102130002303B700A302B7002302B700A301B7002F
:102140002301B700A300B7002300B700828093F5F6
:10215000F50F93968500D58D93960501D58D61B7C2
:10216000939627009702000096968682E78086FA6B
:102170009680C1171D8F3E96E374C3F8A5B73367E9
:10218000B500FD530D8B79E7B7877F7F9387F7F70E
:1021900010419441B372F6003363F600BE92B3E28D
:1021A00062006397720C6318D6065041D441B37233
:1021B000F6003363F600BE92B3E262006398720ADF
:1021C000631BD60410459445B372F6003363F600E2
:1021D000BE92B3E262006391720A631ED60250455A
:1021E000D445B372F6003363F600BE92B3E26200E8
:1021F000639A72086311D60210499449B372F600CB
:102200003363F600BE92B3E2620063937208510535
:10221000D105E30FD6F61317060193970601631C49
:10222000F7001357060193D706013305F74093755E
:10223000F50F91E982804183C1833305F74093759F
:10224000F50F91E182801377F70F93F7F70F3305BE
:10225000F74082800346050083C605000505850515
:102260006313D60065FA3305D640828011059105C7
:10227000E312D6FE014582802105A105E31CD6FCB0
:10228000014582803105B105E316D6FC0145828007
:102290004105C105E310D6FC01458280B717004017
:1022A00003C777051377E70FA38BE704130700F83D
:1022B000A38DE7043D47238CE70413075003A38C49
:1022C000E70403C7A7051377D70F238DE7048280A0
:1022D000B717004003C7E7020D8941111377C70FF5
:1022E000498F93068008F3B6068093F6860836C6B3
:1022F00001000100930670052380D704930680FA3D
:102300002380D704010001002387E702238007040C
:10231000B247F3A70780010001004101828041110B
:102320002A83014E930E407E130F0019930F40062F
:1023300063E56E129308001913034006B378150382
:10234000854E0D4FA14F337365020D89133515006E
:1023500063EFBE121308F6FF7946729842081358CD
:1023600008013307C70213D61700BE07329761462C
:10237000B3F6C60213068070B386C6023697A1660E
:10238000F58F42075D8FB716004083C7F60293F7BB
:102390000708A303F1000346710083C7F60293F711
:1023A0000708E394C7FE83477100B716004093F710
:1023B000F70F6388071293078008F3B7078093F736
:1023C00087083EC401000100B7170040930670055E
:1023D0002380D704930680FA2380D70401000100EC
:1023E00023AA070383C6170393E60608A388D70228
:1023F00023800704A247F3A70780010001001166AC
:10240000B71700407D16D45BC85F93854703A98E3C
:10241000F18EF5FA93068008F3B6068093F68608E7
:1024200036C601000100930670052380D704930689
:1024300080FA2380D7040100010098C103C7170365
:1024400013670704A388E70223800704B247F3A7B2
:10245000078001000100410182807D133368E3039E
:102460009308E016630E08003368F3039308D01650
:10247000630808009378330093B818009388D8163F
:1024800033081E01131E0801135E0E0155B5639338
:10249000E5030548638608000148630303002A88B2
:1024A00071087298FD15131E0801C205135E0E0116
:1024B000C18179BD13F8150063F4BF007908D5B761
:1024C00013381800E5BF83C7F60293F70708A30384
:1024D000F1000346710083C7F60293F70708E394FF
:1024E000C7FE8347710093F7F70FF1DFE9B531714C
:1024F0004AD966CB06DF22DD26DB4ED752D556D32E
:102500005AD15ECF62CD6AC96EC7AA8C02D8971025
:102510000000E78020B12A8993078008F3B707807D
:1025200093F787083EDA01000100B7170040130750
:1025300070052380E704130780FA2380E704010075
:10254000010003C7F7021377770FA387E70203C7DA
:10255000F70213678700A387E70223800704D25797
:10256000F3A7078001000100054597000000E78000
:1025700060D6130780C13347E902116A93070AE85E
:1025800093065002BD69930BA004814A014B1304CA
:102590008008930470057D1AB347F9023307D70208
:1025A0003EC0FD873ECC938709A69309803E334702
:1025B000F7023AC27D873AC4334739038549B39954
:1025C000990193D93940B306D702B30B7703B3C649
:1025D000F602B3CBFB0236C6FD8636C893D6FB4166
:1025E00036CEB7460F00938606243349D902856656
:1025F000938606FAB3969601B389E90213076055EC
:102600003309D90293060010B389E9023349D9028C
:10261000B3C9F9029316390036CA37190040FD864E
:1026200036D0930D090493D7F9413ED2F336048096
:1026300093F6860836DC01000100930770052380BD
:10264000FD00930680FA2380DD000100010083462F
:10265000390593F6860FA309D9048346390593E615
:102660001600A309D90423800D00E256F3A60680C4
:1026700001000100130C80FA116DF336048093F60B
:10268000860836DE01000100930770052380FD00F7
:1026900023808D010100010083463905216693E600
:1026A0000602A309D90483560905B3E6A601231837
:1026B000D90483560905D18E2318D90423800D002F
:1026C000F256F3A60680010001008346390593F611
:1026D00006026381061A03463905218A6DDE081851
:1026E00097100000E7800098733604801376860800
:1026F000B2C20100010023809D0023808D010100F2
:102700000100B717004003C637051376F60DA389FD
:10271000C70403C6370513660602A389C704835698
:1027200009052166B3E6A6012318D90483560905D5
:10273000D18E2318D90423800D009646F3A6068077
:10274000010001008346390593F60602638B0614E7
:1027500083463905A18AEDFE97000020E780A0930B
:10276000AA8636D497000020E780E092A256E30ABA
:10277000D5FE835609054255B3E6A6012318D904B0
:1027800097100000E780C08F83463905A18AEDDEEF
:10279000035609058346290582473376CA00B306E6
:1027A000DA0293D5F641B296B388F640E24733B8E1
:1027B000C6002E983308F840A247B3B61601330876
:1027C000D84063C70701631DF800924763FA1701F9
:1027D000C247634FF80E63950701B24763EAF80EEC
:1027E000894663E9660FF2469315180013D3F80182
:1027F0005E8613951800B365B30042D646D497B0F1
:102800000100E780E0793258050B137BFB0F63472B
:102810000001631A0838A2586387083813081500A6
:10282000B336A800B69513D6F5013298B336C80072
:10283000AE9613581800FE06B3E606017336048000
:1028400013768608B2C60100010023809D00238014
:102850008D01010001000356C902B296C206C18271
:102860002316D90223800D00B646F3A60680010088
:10287000010021B5F336048093F68608B6C0010046
:10288000010023809D0023808D010100010083460B
:10289000390593E60602A309D90423800D00864674
:1028A0000DB5F336048093F68608B6C40100010026
:1028B00023809D0023808D0101000100834639059E
:1028C00093E60602A309D90423800D00A646BDB5F0
:1028D000E30B0BF0F336048093F68608B6C80100CC
:1028E0000100930680FA23809D002380DD00010013
:1028F00001008346390593F5FC0F93F6860FA30973
:10290000D90483463905CD8EA309D90423800D004F
:10291000C646F3A6068001000100130580FA0346AF
:102920003905930639051D8A631C96297336048080
:1029300013768608B2CC01000100130680FA2380CA
:102940009D002380CD000100010003C60600137620
:10295000F60D2380C60003C6060013660602238018
:10296000C600835609051166D18E2318D9048356F3
:1029700009052166D18E2318D90423800D00E6466F
:10298000F3A6068001000100130680FA834639058C
:1029900093F606026380062683463905130C390533
:1029A000A18AFDDA081897000000E780A06BF336D3
:1029B000048093F68608B6D001000100930680FAE1
:1029C00023809D002380DD000100010083460C0070
:1029D000116693F6F60D2300DC0083460C0093E6A7
:1029E00006022300DC0083560905D18E2318D90482
:1029F000835609052166D18E2318D90423800D0042
:102A00008656F3A6068001000100130680FA83466D
:102A1000390593F60602638A062083463905A18AA2
:102A2000EDFE97F0FF1FE78000672A8C97F0FF1FED
:102A3000E7806066E30C85FF835609051166425501
:102A4000D18E2318D90497000000E7806063834685
:102A5000390513063905A18AFDDAF336048093F6A9
:102A60008608B6D401000100930680FA23809D00F9
:102A70002380DD00010001008346060093F6F60D79
:102A80002300D60023800D00A656F3A60680010081
:102A900001008356090503462905D247B376DA00BB
:102AA0003306CA021305800C9355F6413696330D52
:102AB000F6408257333CD6002E9C3336A601330CA9
:102AC000FC40330CCC403308850392564E86B33518
:102AD000A5033305A503C29597B00100E780404CDC
:102AE00063468001631E0C16630C0D161306150059
:102AF0003335A6002E959356F5013696B335D6009C
:102B0000AA959396F50105828585D18E6346B0001E
:102B1000639D051A638B061A0356C9021582330595
:102B2000D6003336C500B2956348B00063910524E2
:102B30001306F00F637DA622894663F356159307AB
:102B40008008F3B7078093F78708BED6010001001D
:102B500037170040930770052300F704930780FAA6
:102B60002300F704010001008356C702896781171B
:102B7000D58FC207C1832316F70223000704B65777
:102B8000F3A7078001000100FA506A54DA544A5949
:102B9000BA592A5A9A5A0A5BFA4B6A4CDA4C4A4D8D
:102BA000BA4D296182801308F5FF3335A800FD1561
:102BB0002E951356F5013298B336C800AA9695B9EA
:102BC000F336048093F68608B6CA0100010023801C
:102BD0009D002380AD000100010083463905CD8EA4
:102BE000A309D90423800D00D646F3A60680010070
:102BF000010035B3F336048093F68608B6CE0100A3
:102C0000010023809D002380CD0001000100834648
:102C1000390593E60602A309D90423800D00F64680
:102C2000F3A606800100010095B3F336048093F605
:102C30008608B6D20100010023809D002380CD00CC
:102C4000010001008346390593E60602A309D90471
:102C500023800D009656F3A606800100010045BBB7
:102C60009306F5FF33B5A600FD152E959355F50196
:102C7000AE96B3B5B600AA951396F501858269B5EF
:102C8000F336048093F68608B6D801000100930657
:102C900080FA23809D002380DD000100010083561F
:102CA000C9020566011693F6F60FD18EC206C182DF
:102CB0002316D90223800D00C656F3A60680010014
:102CC0000100850A93FAFA0F95B233E6B60045C2C1
:102CD0000356C9023305D0403338A000B305B040D5
:102CE000B385054115826345B000D1E16371A60843
:102CF000894663F0560593078008F3B7078093F77A
:102D00008708BEDA01000100B717004013077005FD
:102D10002380E704130780FA2380E7040100010001
:102D200003D7C7027D8B2396E70223800704D6577B
:102D300081BDF336048093F68608B6DC01000100FD
:102D4000930680FA23809D002380DD0001000100AE
:102D50008356C9020566011693F6F60FD18EC20698
:102D6000C1822316D90223800D00E656B9B7930716
:102D70008008F3B7078093F78708BEDE01000100E3
:102D800037170040930770052300F704930780FA74
:102D90002300F704010001000356C7029397560071
:102DA000B297C207C1832316F70223000704F65720
:102DB000C1BB914763EEB70217D701001307C709DC
:102DC0008A05BA959C41BA978287B717004003A736
:102DD000470B1345F5FF698F23AAE70A03A7070BE3
:102DE000698F23A8E70A03A7070A798D23A0A70AFA
:102DF0008280B717004083A6470B1347F5FFF98E73
:102E000023AAD70A83A6070B558D23A8A70A83A652
:102E1000070A758F23A0E70A8280B717004003A72F
:102E2000470B498F23AAE70A03A7070B1345F5FFB2
:102E300045BFB717004083A6470B1347F5FF758FB3
:102E400023AAE70A03A7070A598D4DB7B717004011
:102E500003A7470B498FEDB7914763EEB70217D72A
:102E600001001307A7008A05BA959C41BA9782878B
:102E7000B717004003A7470D1345F5FF698F23AA35
:102E8000E70C03A7070D698F23A8E70C03A7070C1E
:102E9000798D23A0A70C8280B717004083A6470D29
:102EA0001347F5FFF98E23AAD70C83A6070D558D7E
:102EB00023A8A70C83A6070C758F23A0E70C82809C
:102EC000B717004003A7470D498F23AAE70C03A7B4
:102ED000070D1345F5FF45BFB717004083A6470D03
:102EE0001347F5FF758F23AAE70C03A7070C598D2D
:102EF0004DB7B717004003A7470D498FEDB779715C
:102F000022D43714004026D24AD0035924028354D5
:102F1000040206D64209C2044ECE52CC56CA1359F8
:102F20000901C1802DE11379F9F793F4F49F420967
:102F3000C20413590901C18093078008F3B70780C1
:102F400093F787083EC40100010093077005230032
:102F5000F404930780FA2300F40401000100231114
:102F600024032310940223000404A247F3A707803C
:102F700001000100B250225492540259F249624AAF
:102F8000D24A45618280B7F5070081463000B1051D
:102F9000194597000020E7806081A2471397270119
:102FA000E34A07FC1369090893E404409309800885
:102FB000F3B7098093F787083EC001000100930A28
:102FC000700523005405130A80FA2300440501000C
:102FD00001002311240323109402230004048247D8
:102FE000F3A7078001000100294597F0FF1FE78044
:102FF0006034F3B9098093F989084EC201000100D9
:1030000023005405230044050100010083570402F6
:1030100093E707202310F402230004049247B9B772
:10302000B71700408847420541819377050491EB2B
:103030009377F5013755E801130505803345F5020F
:1030400082809377050C130700046397E70093775A
:10305000F50137459C1CCDB72165130505D082804D
:1030600037E700E01C435443A183E206D58F1CC11F
:10307000FD572320F7182322F718828013178500A5
:10308000B7E700E023A0E710618123A2A7108280A8
:10309000B7F700E08847CC47828081473737004048
:1030A000A14663C4C700328582800345B740E38EE2
:1030B000A6FE3385F5000345050085072304A740D8
:1030C000CDB7970700209387E7EE9C431737002082
:1030D0001307C7063E95636EE500173700201307F8
:1030E00067526368A700170700202325A7EC3E85D9
:1030F0008280FD57EDBF8280411122C406C62A841A
:1031000097000000E78000F22947B307E502B240CC
:103110008D83B3D7870222449507B3D7E7023737A9
:103120000040C207C1832316F7004101828041118C
:1031300037150E0006C697000000E78020FCB73761
:103140000040130770F82381E7000D47A381E700D3
:1031500013070004A380E70005472387E700B24078
:103160004101828037370040834727001A0593F7D3
:10317000F703C98F93F7F70F2301F7008280B73762
:10318000004003C7170019C9D98DA380B70003C732
:103190000700136787002380E700828093C5F5FF4F
:1031A000F98DA380B7008280AE872A87B7360040AA
:1031B00021463738004089E7170300006700E3F332
:1031C00083C8B600E30916FF05078348F7FFFD171C
:1031D000C20723041801C183F9BF411122C406C6E6
:1031E0002A8497000000E780E0E32947B307E5025F
:1031F000B2408D83B3D7870222449507B3D7E70245
:1032000037370040C207C1832316F740410182804F
:10321000716541111305052006C697000000E7807F
:1032200000FCB7370040130770F82381E7400D47D3
:10323000A381E74013070004A380E74005472387E5
:10324000E740B24041018280CC41411106C632853F
:1032500003C6150083C5050022064D8E42068D6506
:103260004186138875A2630C0611634BC80413884A
:1032700045A26300060D634AC800938535A2630129
:10328000B6082390060029464DA0138855A2630571
:10329000060D938565A2E316B6FE8D451D4663E6D1
:1032A000E5081146198E63F3C7003E86B7E70400B0
:1032B0002390C600FC4797D50100938565BD9DA06E
:1032C000138895A263030611634E060D1388A5A209
:1032D00063000613938505A5E315B6FA99451D46C7
:1032E00063E5E504198E63F3C7003E86B7E7040083
:1032F0002390C600FC47970500209385E5D51DA0C7
:103300009D451D4663E3E5022146198E63F3C70020
:103310003E86B7E70400FC472390C60097050020CF
:103320009385C533BA9582970146B24032854101F3
:103330008280AD451D46E3EAE5FE3146198E63F312
:10334000C7003E86B7E704002390C600FC4797D528
:103350000100938565B6F9B7B1451D46E3E7E5FC85
:103360003546198E63F3C7003E86B7E70400239005
:10337000C600FC4797D50100938505B565B78D4517
:103380001D46E3E4E5FA1146198E63F3C7003E8655
:10339000B7E704002390C600FC4797D5010093854A
:1033A000E5AF49B78D451D46E3E1E5F81146198EB5
:1033B00063F3C7003E86B7E704002390C600FC47CE
:1033C00097D50100938505B2B1BFA5451D46E3EE33
:1033D000E5F42946198E63F3C7003E86B7E704007B
:1033E0002390C600FC4797D501009385E5AB1DBF30
:1033F000B5451D46E3EBE5F23946198E63F3C70088
:103400003E86B7E704002390C600FC4797D501002D
:10341000938505A701BFB7E7040003A30713970629
:103420000020938666C24146A54517050020130576
:10343000A5B802832D455DE703C505000947631F55
:10344000E50803A84500411106C603471800328568
:103450000346080022074168518F930828FE63073E
:10346000170563E9E80005186303070323900600C6
:10347000294591A8130648FE630AC7041518E317E7
:1034800007FF15463E87637BF600154701A8130624
:1034900000023E876374F60013070002B7E70400DA
:1034A0002390E600FC471316070111A83E8691C33E
:1034B0000546B7E70400FC472390C6004206CC450A
:1034C000418282970145B240410182801306000883
:1034D0003E87E375F6FC13070008C9B72390060082
:1034E000054582808280416779176304E5044111B4
:1034F00022C406C685472A84639FF500B7E7040007
:1035000022852244B24003A38713970500209385A8
:10351000252F4101028389476399F500B7E704002D
:1035200083A7070B8545829771D9B2402244410198
:1035300082808280797122D452CC2E842A8A97D5B7
:1035400001009385259C17D501001305259E06D6FD
:103550003AC626D24AD0B68432894ECE97B0010000
:10356000E78040EFA68517D501001305259D97B08C
:103570000100E78020EE294597B00100E78060F266
:103580008347840093F70702E1E7834904008947F2
:10359000054532476396F908544083C7160083C631
:1035A0000600A207D58FC166138616FE638CC7027C
:1035B0008D16638FD7068D66938626902945639175
:1035C000D706B7E70400A285225403A34714B250DC
:1035D000F249A6864A86925402595285624A854724
:1035E000456102832D450DEF93070002354563E9E0
:1035F0009702B7E70400FC47484413060002CA8557
:103600008297814997070020938747209C43014573
:1036100081CB9C4391C74E852686CA8582970145FA
:10362000B250225492540259F249624A4561828052
:103630002D457DF79307700F3545E3E397FEB7E718
:103640000400FC4748441306700FCA8582975DBF8B
:103650002145F9B7411122C437E4040083278413BC
:1036600026C2AA84416506C69705002093854519A0
:103670007D1582978327C40A170500001305E5E628
:103680008588829795C0032304132244B240924454
:10369000970600209386C6AD4146C5451705002014
:1036A0001305059C41010283B24022449244014526
:1036B0004101828019C59707002023A9A71401455D
:1036C0008280454582801147636AA70A97D6010028
:1036D000938606820A0536951841411106C636972B
:1036E000AE87B2850287130700026145639DE7003C
:1036F000B7E70400FC471306000217050020130576
:1037000065F682970145B2404101828005476145D7
:10371000E39BE7FEB7E70400FC47054617050020DA
:10372000130545F6F9BF1307700F6145E39DE7FCEC
:10373000B7E70400FC471306700F170500201305B8
:10374000A5F4C1B7130700086145E39EE7FAB7E7A0
:103750000400FC4713060008170500201305450266
:103760004DB715476145E390E7FAB7E70400FC471A
:103770001546170500201305E50861B70945828045
:10378000411126C2B7E4040083A7C41322C44AC06F
:1037900006C62E8497050020938585062A89829780
:1037A000058905C5970700209387878B83D7A70BCB
:1037B000A28503A3440D2310F4002244B240924496
:1037C0004A850249014641010283B24022449244A3
:1037D000024949454101828097070020238A070258
:1037E0009707002023A80702B717004003A7070C7C
:1037F000B706C0FFFD16758F23A0E70C03A7070DC2
:10380000B7064000558F23A8E70C03A7070C3D9B84
:1038100023A0E70C03A7070D1367070123A8E70CF4
:103820008280B717004003A5470C83A7470C598136
:1038300013451500C18B058999E31365250097078A
:10384000002083C7E7FC6380A7029707002023813D
:10385000A7FC11C9970700209387C7FB03A30700A4
:103860006303030002838280114517F3FFFF6700A3
:1038700043C8411193962500AA852D4506C697F0A9
:10388000FF1FE780A0F2B240014541018280011193
:1038900022CC06CE3714004026CA4AC84EC652C4AF
:1038A00083447405034AB405834984050349940598
:1038B00097F0FFFFE780C09E8347A40593F4F40FC1
:1038C000137AFA0F93E71700230DF40493F9F90F15
:1038D0001379F90FB717004003C7A705058B6DFFD4
:1038E00003D5C705A38D4705238C3705A38C270572
:1038F000A38B9704F2406244D2444249B249224A1F
:103900000561828041119397050122C406C626C233
:10391000C1872E8463DC0700B7E40400FC5482975F
:1039200019C1BC5482972165218D15A893F7150004
:1039300013C515008DE793F725009DC7970000007C
:10394000E78060EEB7E70400BC4F1306000A894524
:1039500017050020034585EC829713452400B240EB
:1039600022449244410182809397250163D8070243
:10397000B7E4040083A7C41E829797000000E78085
:10398000E0EEBC4C37560700130606308965170574
:1039900000200345A5E88297096579B7939715013B
:1039A0000145E3DE07FA17C501001305256197B04D
:1039B0000100E78000C2B7E70400BC4F13060064B3
:1039C000916517050020034565E582971165A9BF3C
:1039D0002D71232A9110FD74E98C232C811023284A
:1039E0002111232631112A84AE89328993060010D1
:1039F0000A86A6852D45232E111097F0FF1FE7801C
:103A0000E0DA13154401B7E70400FC4751810A05C9
:103A100013962900CA850A958297A6858566014670
:103A2000254597F0FF1FE78060D80A86A685930694
:103A30000010294597F0FF1FE78040D78320C11170
:103A40000324811183244111032901118329C11009
:103A500015618280B7F7070003C70701411106C649
:103A600022C426C24AC0A547631DF7009700000084
:103A7000E78040F6B24022449244024901454101A8
:103A8000828013942500AA843289A286AA850146E1
:103A9000254597F0FF1FE78060D1A2864A86A6855C
:103AA000294597F0FF1FE78060D0E9B71D71A2CCD0
:103AB00037E404005C5C485886CE494697C501004F
:103AC0009385454B829711E917C501001305C54B36
:103AD00097B00100E780E0AF01A0B7F600E07957AA
:103AE00098CAFD57DCCA0567B7E700E023A0E710D6
:103AF0001306F00290C223A0E71801000100370767
:103B0000002018471306000481459706002023A5CE
:103B1000E6D04157A38AE7403C44080882979707BC
:103B200000209387676C3EC8856713870740231A78
:103B3000E1001D673ACC37070105130707103ACE9D
:103B4000938757D11307B00F2310E1022312F1021C
:103B5000054797F7FFFF9387E7532301E1023ED81C
:103B600017070000130727D197070000938767D234
:103B7000B7F50700BAC23EDC170700001307C7ED10
:103B800097070000938787CE81463000E1051945ED
:103B9000BAC43EDE97F0FF1FE78040C11808814796
:103BA000994630003E960346060085070507A30B9D
:103BB000C700E398D7FEC24791C703574101856705
:103BC0006373F70001A0B7E7040083A7470A08085A
:103BD0008297AA8511C917C501001305253C97B026
:103BE0000100E780208701A0F640664425618280BD
:103BF000411126C2B7E4040083A7040806C622C404
:103C000017050000130545D0829717040020130400
:103C1000E4C02300A40097000000E7808002970022
:103C20000000E780A0BB03450400224403A38405F1
:103C3000B2409244130600328965410102837971D2
:103C400006D622D413078008F337078093F7870836
:103C50003EC201000100B7170040930570052380A4
:103C6000B704130680FA2380C7040100010083C64D
:103C7000F70293F6A60FA387D70223800704924684
:103C8000F3A60680010001007337078013778708C9
:103C90003AC4010001002380B7042380C704010057
:103CA000010003C7F70213672700A387E7022380F9
:103CB0000704A247F3A7078001000100054597E02C
:103CC000FFFFE780206197000000E78020BA0147EE
:103CD00081468147054685451305407E97E0FFFFF5
:103CE000E780206437E404003C4468005146814585
:103CF0008297B707C0A83EC8B787E803938707D065
:103D00003ECA97E7FF1F9387876B3EC67C586800C3
:103D10008297B250225445618280411197D50100AB
:103D20009385059017C501001305452006C697A089
:103D30000100E780207217D50100130525A797A081
:103D40000100E7802071B2402945410117A301001D
:103D500067002375411197D501009385A58D17C57F
:103D600001001305A51C06C697A00100E780806E20
:103D700017D50100130545A297A00100E780806DCB
:103D8000B2402945410117A3010067008371411129
:103D900022C406C6834705002A849DC797D5010023
:103DA0009385058F17C501001305451897A00100DD
:103DB000E780406A4C4017D50100130565AD97A018
:103DC0000100E78020693DA058410DEF97D5010023
:103DD0009385058C17C501001305451597A00100B3
:103DE000E780406717D50100130505AC97A00100D7
:103DF000E78040662244B2402945410117A30100F3
:103E00006700236AA1679386D7036313D70297D508
:103E100001009385E58717C501001305251197A0BB
:103E20000100E780206317D501001305E5A87DBFD9
:103E3000ED0797D501009385A58517C501001305EA
:103E4000E50E631BF70097A00100E780A06017D57F
:103E500001001305A5A759BF97A00100E780805F67
:103E60004C4017D50100130565A891BF411197C5B6
:103E700001009385657D17C501001305250B06C656
:103E800097A00100E780005DB2402945410117A3DA
:103E9000010067000361797122D426D24AD02E84B2
:103EA0002A898145B2844800714606D697E0FFFF13
:103EB000E780A02297F7FF1F9387474CDC4783D703
:103EC0000700231421012313F10097500000E7801D
:103ED000A0809547A305F1009307401F3EC6FD57FC
:103EE0002305A100230AF10097500000E78000930A
:103EF0002686A285480097500000E780C080B25017
:103F000022549254025945618280971700202390D1
:103F1000077E971700202389076CB7E70400BC478A
:103F2000411106C641468145170500201305451A73
:103F3000829797200000E780A05697200000E78036
:103F4000C031014597500000E780A02517070020E9
:103F50000347071A9307F00A6315F7029307F0F86F
:103F60008945170500201305A51817070020230110
:103F7000F71897070020A38D071697500000E780D9
:103F8000E04C97500000E780A059814537050400B8
:103F90009707002023AC07129707002023960712EB
:103FA0009707002023830712970700202394070A0E
:103FB00097070020239207089707002023950710F2
:103FC00097070020239E071097300000E780A0C4C9
:103FD000014597500000E780605097C50100938528
:103FE000256917C50100130565F497A00100E78056
:103FF000604617D501001305A59597A00100E7803D
:104000006045B2402945410117A30100670063499B
:10401000411122C406C626C293F715002E84638F71
:104020000710814617F6FF1F1306863285451705D0
:1040300000200355250097C00000E78060B315C934
:1040400097C501009385856317C50100130505EE2B
:1040500097A00100E780004017C501001305C504C3
:1040600097A00100E780003F294597A00100E78065
:10407000404397C501009385656017C5010013058E
:10408000E5EA97A00100E780E03C17C501001305B1
:10409000E50297A00100E780E03B294597A00100D9
:1040A000E780204017F5FF1F1305452D5C450547A8
:1040B0002390E70097300100E780E06397C5010097
:1040C0009385C55B17C50100130545E697A0010060
:1040D000E780403817C50100130585FF97A0010050
:1040E000E7804037294597A00100E780803B930790
:1040F00010F817070020230DF7FE9707002083D73D
:1041000027F317070020A305F7FE17050020130566
:1041100025FEA183914517070020230CF7FC970784
:104120000020A38807FC97500000E7802032134549
:104130001400B240224492444101828093F725004A
:10414000E1C317070020035727F845CB9706002047
:104150009386C6F7944297D7010093876781170625
:104160000020034686F6814517050020130545F615
:1041700097700000E78020BFAA8441C197C5010065
:104180009385855617C50100130545DA97A00100F0
:10419000E780402CA68517C501001305E5F497A01C
:1041A0000100E780202B294597A00100E780602FC0
:1041B00097070020239A07F0930710F817070020AD
:1041C0002308F7F29707002083D787E61707002018
:1041D000A300F7F2A18317070020230CF7F0914505
:1041E0008D47170500201305A5F017070020A3022F
:1041F000F7F097500000E78060251345240015BFB5
:1042000093F74500D1C397C501009385E54D17C5C8
:1042100001001305A5D197A00100E780A02317C5D1
:104220000100130525EE97A00100E780A022294593
:1042300097A00100E780E026930720F817070020E9
:104240002308F7EA9707002083D7C7E01707002065
:10425000A300F7EAA18317070020230CF7E885479E
:1042600017070020A307F7E897400000E780005BEE
:10427000170500201305C5E7914597500000E7801A
:10428000E01C1345440075B593F78500A9C797C591
:1042900001009385654517C50100130525C997A041
:1042A0000100E780201B17C501001305E5E697A074
:1042B0000100E780201A294597A00100E780601ED1
:1042C00097070020239207E097700000E78080B9ED
:1042D00013458400B9BD93F70501D1C38545170582
:1042E0000020035525D797500100E780A06B97C5A4
:1042F00001009385653F17C50100130525C397A0ED
:104300000100E780201517C50100130525E297A0DD
:104310000100E7802014294597A00100E78060187C
:10432000930730F8170700202304F7DC97070020D5
:1043300083D747D217070020A30CF7DA1705002010
:10434000130505DBA1838D45170700202303F7DA4A
:1043500097500000E780800F13450401D9BB93F705
:104360000502D1C797C501009385053817C501001F
:104370001305C5BB97A00100E780C00D17C501005C
:10438000130505DD97A00100E780C00C294597A023
:104390000100E7800011930740F817070020230968
:1043A000F7D49707002083D727C917070020A30158
:1043B000F7D4A18317070020230DF7D285471707ED
:1043C0000020A308F7D297070020239707C697403D
:1043D0000000E780A04417050020130565D1914532
:1043E00097500000E78080061345040299B393F7C5
:1043F0000504FDC397C501009385052F17C501006E
:104400001305C5B297A00100E780C00417C50100DD
:10441000130585D597A00100E780C003294597A023
:104420000100E78000089707002083C767CC1307C7
:10443000700A6386E7061307800A638CE708130790
:10444000600A6393E704930760F8170700202301CD
:10445000F7CA9707002083D707C717070020A309CB
:10446000F7C8A183170700202305F7C8854717075A
:104470000020A304F7C8B14517050020130545C760
:1044800097500000E78080FC97400000E7800039EB
:104490001345040497070020239707C259B99307CF
:1044A00070F8170700202305F7C49707002083D76B
:1044B00087C117070020A30DF7C2A18317070020AB
:1044C0002309F7C2854717070020A305F7C29945BE
:1044D00065B7930780F8F1B793F705080145E38ABC
:1044E00007C497C501009385252017C50100130552
:1044F000E5A397A00100E780E0F517C501001305CB
:1045000025C897A00100E780E0F4294597A00100A5
:10451000E78020F99307A0F817070020230AF7BCCB
:104520009707002083D7C7BB17070020A302F7BC5B
:10453000A18317070020230EF7BA8547170700202D
:10454000A309F7BA97070020239C07B897400000FB
:10455000E780C02C17050020130585B991459750B9
:104560000000E780A0EE13450408E1B6411122C423
:1045700097C50100938505132A8417C5010013050B
:10458000E59A06C697A00100E780C0EC4C4017C52D
:1045900001001305652D97A00100E780A0EB2945D8
:1045A00097A00100E780E0EF034704009307F00FB6
:1045B000631FF70297C501009385C50E17C501005B
:1045C0001305C59697A00100E780C0E84C4017C5C9
:1045D00001001305652A97A00100E780A0E72244A7
:1045E000B2402945410117A30100670083EBB240A7
:1045F000224441018280B1C1411122C417C501008A
:104600001305C5922E8497C501009385A50406C69F
:1046100097A00100E78000E4A28517C501001305FB
:10462000E53097A00100E780E0E22244B24029454E
:10463000410117A301006700C3E68280411122C433
:1046400026C22E84AA8497C501009385650117C5EB
:1046500001001305A58D06C697A00100E78080DF45
:1046600017C501001305452D97A00100E78080DEE6
:10467000294597A00100E780C0E297C50100938516
:1046800025FE970700202397979A17C50100130569
:10469000E589854497070020239C87989707002089
:1046A00023999798971700202393870497A00100D8
:1046B000E78040DA9715002083D5650317C5010010
:1046C0001305052897A00100E780C0D8294597A0C9
:1046D0000100E78000DD97170020238797F09720DF
:1046E0000000E78080B7228597500000E78060AB2C
:1046F000054597500000E78060DE97F7FF1F93871E
:10470000E7C7DC4703D70700C167FD176312F7024D
:104710002244B7E70400B240924403A3870517F58B
:10472000FF1F034525101306000A8545410102833A
:10473000B2402244924441018280011122CC37E4EC
:1047400004005C5C06CE354697C50100938545079D
:1047500017D50100130545C1829711E917C501005E
:104760001305858297A00100E780A0E601A097F7D6
:10477000FF1F9387E70B3EC4B7F507008567938754
:104780000780814617F6FF1F1306060AE105194543
:104790003EC697E0FF1FE78060017C44194697F50D
:1047A000FF1F93856508170500201305E58A82978A
:1047B000340017F6FF1F1306260797C501009385DF
:1047C000255217C501001305255397600000E780A7
:1047D000802E2A841DCD97C501009385E5EF17B57E
:1047E00001001305A57497A00100E780A0C6A2856B
:1047F00017C501001305C5FD97A00100E78080C51E
:10480000294597A00100E780C0C9F24062440561D4
:10481000828097E00000E780E09017C50100130553
:1048200025F297500000E780C02297A00000E780A3
:1048300020E597500100E780A04917F5FF1F1305F9
:1048400065B097500100E780403217C5010013059D
:1048500025F097500100E780204A2A8497600000E5
:10486000E780008997000100E780802197800100A0
:10487000E780A0BA97700000E78040E197600000F1
:10488000E78000FF97300100E780E0E297C5010074
:10489000938585E417B501001305456919C897A0EC
:1048A0000100E78020BBA28517C50100130585F430
:1048B000A1B797A00100E780E0B917C50100130573
:1048C000A5F597A00100E780E0B8294597A0010071
:1048D000E78020BD97300100E780C0BE97F0000060
:1048E000E78080DD55C98545370504009720000025
:1048F000E780603297C50100938505DE17B501009A
:104900001305C56297A00100E780C0B417C5010078
:10491000130505F297A00100E780C0B3294597A0D1
:104920000100E78000B897F7FF1F9387E79483D7CC
:10493000070017170020231CF7DA854717170020F8
:104940002304F7CA97200000E78000B097200000FA
:10495000E780A09017150020035565D997500000F7
:10496000E7802084054597500000E78020B797C571
:104970000100938565D617B501001305255B97A047
:104980000100E78020AD17C501001305A5EC97A035
:104990000100E78020ACADB597C501009385C5D374
:1049A00017B501001305855897A00100E78080AA7C
:1049B00017C501001305C5F997A00100E78080A97C
:1049C000294597A00100E780C0AD014569BF4111AD
:1049D00022C437E404008327041A06C6829797404E
:1049E0000000E780C07F8327040817F5FFFF130549
:1049F0006562829797F7FF1F2386A7E217F5FF1FCF
:104A00001305C59797400000E780E0132244B240A9
:104A1000410117030000670083D2B7E70400FC4799
:104A20001171A2DDCAD986DFA6DBCED72E843289EA
:104A30002E86AA8517F5FF1F1305856B829717F73A
:104A4000FF1F1307E76A83470700930680029387D7
:104A5000E70793F7F70FE3ECF610BA898A0717B761
:104A600001001307E755BA979C43BA9782878D4791
:104A700097C50100938585C817B501001305054B3F
:104A8000630FF40097A00100E780C09C17C50100E8
:104A90001305858597A00100E780C09BBDA497A062
:104AA0000100E780209B17C501001305658597A0CD
:104AB0000100E780209A294597A00100E780609EC9
:104AC000930720F8114697F5FF1F938565624A8585
:104AD00017F7FF1F230EF76097F7FF1FA38B0760E1
:104AE00097F0FFFFE780603B2A841DC997C501004E
:104AF0009385C5C017B501001305454397A0010074
:104B0000E7804095A28517C501001305258397A06E
:104B10000100E7802094294597A00100E780609874
:104B200097C50100938585BD17B5010013050540A4
:104B300097A00100E780009217C501001305458189
:104B400097A00100E7800091294597A00100E78028
:104B500040954165930730FA054697F5FF1F938509
:104B600025597D1517F7FF1F2304F75897F0FFFF0E
:104B7000E780A0322A841DC997C50100938505B836
:104B800017B501001305853A97A00100E780808CD6
:104B9000A28517B501001305657A97A00100E7808B
:104BA000608B294597A00100E780A08FB7E704003C
:104BB000BC4F0566130606C8A14517F5FF1F034540
:104BC00065C68297FE506E54DE544E59BE5911612F
:104BD000828091476303F40297C50100938505B273
:104BE00017B501001305853497A00100E780808682
:104BF00017B501001305057971BDB7E70400FC4F37
:104C0000914517F5FF1F0345E5C1829797C5010040
:104C10009385C5AE17B501001305453197A0010076
:104C2000E780408317B501001305857797A0010041
:104C3000E7804082294597A00100E7808086974061
:104C40000000E780A0BD914535A485476303F402C9
:104C500097C50100938585AA17B501001305052D99
:104C600097900100E780007F17B501001305C57418
:104C700015B597F7FF1F239F273DB7E7040005668B
:104C8000BC4F130606C8C1450DBF8D476303F40230
:104C900097C50100938585A617B501001305052961
:104CA00097900100E780007B17B50100130585721E
:104CB000D5B3930740F8114697F5FF1F93854543F9
:104CC0004A8517F7FF1F2305F74297F7FF1FA382B7
:104CD000074297F0FFFFE780401C2A84E30405EEBB
:104CE00097C50100938585A117B50100130505241B
:104CF00097900100E7800076A28517B501001305A3
:104D0000E56397900100E780E074294597900100E2
:104D1000E780207945BD9147E31CF4F6B7E704002E
:104D2000FC4F9305000217F5FF1F0345A5AF8297BF
:104D300097C501009385859C17B501001305051FD4
:104D400097900100E780007117B501001305056A0F
:104D5000F1BD894763E3870297C501009385059AF2
:104D600017B501001305851C97900100E780806E40
:104D700017B501001305C56831BB97F4FF1F83C445
:104D8000443797F7FF1F83C7B73697C50100938550
:104D9000E596A20417B5010013054519DD8C97901F
:104DA0000100E780206BA28517B501001305856619
:104DB00097900100E780006AC2042945979001009E
:104DC000E780206EC1849305D4FF93960401C182CD
:104DD0004A8693F5F50F17F5FF1F130595319720B8
:104DE0000000E78000E7E35F90DC930750F817F7D7
:104DF000FF1F230FF72E83C73900228697F5FF1F69
:104E00009385052F85074A8517F7FF1FA303F72E04
:104E100097F0FFFFE78060082A84E30505DA97C56D
:104E200001009385A58D17B50100130525109790F6
:104E30000100E7802062A28517C50100130505AEB9
:104E4000C9B5894763E3870297C501009385058B40
:104E500017B501001305850D97900100E780805F6D
:104E600017B501001305C55C35B197400000E78018
:104E7000E09AA28517F5FF1F1305852797400000CC
:104E8000E780C05C81B38D476303F40297C50100DE
:104E90009385C58617B50100130545099790010054
:104EA000E780405B17B501001305455AE5B6B766C4
:104EB00002000146B7750200054597E0FF1FE78035
:104EC000E08E930760F817F7FF1F2303F72297F789
:104ED000FF1FA38007229307000617F7FF1F230B6E
:104EE000F720894717F7FF1FA306F72097F7FF1F43
:104EF0002383072097F7FF1FA38F071EC14717F7CC
:104F0000FF1F230BF71E930720F917F7FF1FA305B9
:104F1000F71E314697F7FF1FA381A71E97F5FF1FC6
:104F20009385051D4A8597F7FF1F2388071C97F077
:104F3000FFFFE78080F62A84E30605C897B50100E5
:104F40009385C57B17B50100130545FE97900100B9
:104F5000E7804050A28517B501001305A55055B351
:104F6000B1476303F40297B501009385257917B51E
:104F700001001305A5FB97900100E780A04D17B530
:104F800001001305E54F39B6B7E70400FC4F930560
:104F9000000417F5FF1F0345E5888297974000003E
:104FA000E780C087B145F9B5914763E3870297B5BC
:104FB00001009385A57417B50100130525F7979097
:104FC0000100E780204917B501001305254DD9B42C
:104FD00097F4FF1F83C4041297F7FF1F83C777114D
:104FE000A204DD8C8E04B77702006D14BE94228675
:104FF000A68517B501001305A54B97900100E78022
:105000006045B7E70400FC47228697F5FF1F9385AC
:10501000750E2800829793160401C1823000A68580
:10502000094597D0FF1FE78060782A8409C917B522
:1050300001001305A54997900100E7808059930767
:1050400070F8194697F5FF1F9385850A4A8517F76B
:10505000FF1F230FF70897F7FF1FA38D870897F00F
:10506000FFFFE78080E32A84E30E05B497B50100D3
:105070009385C56817B50100130545EB97900100AE
:10508000E780403DA28517B501001305254595B978
:105090009947630BF41297B501009385256617B500
:1050A00001001305A5E897900100E780A03A17B525
:1050B000010013052544F9BA914763E3870297B5C8
:1050C00001009385A56317B50100130525E69790A8
:1050D0000100E780203817B50100130525435DBAAC
:1050E00097F4FF1F83C4040197F7FF1F83C777005E
:1050F000A204DD8C8E04B77702006D14BE94228664
:10510000A68517B501001305A54197900100E7801A
:105110006034B7E70400FC47228697F5FF1F9385AC
:1051200075FD2800829793160401C1823000A68580
:105130000D4597D0FF1FE78060672A8409C917B51E
:1051400001001305A53F97900100E7808048930771
:1051500080F8194697F5FF1F938585F94A8517F75B
:10516000FF1F2307F7F897F7FF1FA38587F897F02E
:10517000FFFFE78080D22A84E30605A497B50100EB
:105180009385C55717B50100130545DA97900100BF
:10519000E780402CA28517B501001305653B95B645
:1051A00099476303F40297B501009385255517B518
:1051B00001001305A5D797900100E780A02917B536
:1051C00001001305653AF9B0B7E70400FC4F9305F9
:1051D000000417E5FF1F0345E56482979730000040
:1051E000E780C063994579B18D476303F40297B5B1
:1051F00001009385A55017B50100130525D397909D
:105200000100E780202517B501001305653759B067
:1052100017B501001305C53797900100E780603B83
:105220001305C01297D0FF1FE780A011014597E03A
:10523000FFFFE78020E30D4597100000E780009F07
:10524000294597D0FF1FE780C00F97D0FF1FE78049
:1052500020008DBA99476303F40297B50100938546
:10526000E54917B50100130565CC97900100E7806B
:10527000601E17B501001305653229B817F7FF1F27
:10528000034757E797F7FF1F83C7C7E622075D8FDE
:105290009166BA96C2061166C1821306F6EF8D4773
:1052A0006365D60297E7FF1F9387470D9C4B17F660
:1052B000FF1F034616E49386C7002DC203D60700DE
:1052C00069CA8907E39CD7FE89471307A0F81146EE
:1052D00097F5FF1F9385C5E14A8597F6FF1F238940
:1052E000E6E017F7FF1FA306F7E097F0FFFFE78060
:1052F000C0BA2A84E308058C97B501009385054060
:1053000017B50100130585C297900100E78080144E
:10531000A28517B501001305A529E5B203D607003C
:10532000630EE60A8907E39BF6FE8D4779BF914736
:105330006304F40297B501009385453C17B501005D
:105340001305C5BE97900100E780C01017B5010096
:10535000130585276FF00FF4B7E70400FC4F9305A2
:10536000000817E5FF1F0345E54B8297C9B897B5BD
:1053700001009385A53817B50100130525BB97904B
:105380000100E780200D17B50100130565256FF0BA
:105390006FF02390E70017E5FF1F130525FE972008
:1053A0000100E780A03797B501009385253517B533
:1053B00001001305A5B797900100E780A00917B574
:1053C00001001305E52297900100E780A008294518
:1053D00097900100E780E00C8147C5BD239007004E
:1053E00017E5FF1F130585F997200100E7800033BB
:1053F00097B501009385853017B50100130505B3F6
:1054000097900100E780000517B501001305C51F3F
:105410005DBF411122C406C6834705002A849DC78B
:1054200097B501009385452917B50100130505B00F
:1054300097900100E78000024C4017B5010013056A
:10544000255497900100E780E000E1A05841B7079C
:10545000CF009387777D631DF70697B5010093858D
:10546000A52517B50100130565AC97900100E780ED
:1054700060FE1C448356E4008355C40003C6070045
:1054800017B501001305455197900100E78080FC96
:10549000294597900100E780C0000357E400970773
:1054A000002083D7C7246309F7008355C40008444C
:1054B00097E0FFFFE78080CF0356E4008355C400E8
:1054C00008442244B240410117F3FFFF670023550F
:1054D000B707CC009387777D6315F70497B5010074
:1054E0009385851D17B50100130545A4979001000C
:1054F000E78040F61C448356E4008355C40003C68D
:10550000070017B501001305254997900100E780B2
:1055100060F42244B240294541011793010067001D
:1055200043F8B707CE009387777D6304F70297B5FA
:1055300001009385651817B501001305259F979005
:105540000100E78020F14C4017B501001305053A32
:10555000CDBDB240224441018280B7E70400FC4740
:1055600041112E8606C622C426C24AC02E842A892C
:10557000AA8517F5FF1F1305A5B7829797B50100F8
:105580009385851917B501001305459A9790010079
:10559000E78040EC97F5FF1F83C585B517B501007F
:1055A000130585BF97900100E780C0EA29459790D1
:1055B0000100E78000EF97F4FF1F938464B383C773
:1055C000040041479387070693F7F70F636AF75C78
:1055D00017B70100130707A98A07BA979C43BA9720
:1055E00082879D476307F40297B501009385C51232
:1055F00017B501001305859397900100E78080E5BA
:1056000017B501001305C5B997900100E78080E444
:10561000ADAC97F7FF1F83C7B7ADDDCB17F7FF1F03
:10562000034737AD97F7FF1F83C7A7AC22075D8FEE
:1056300097F7FF1F83C707ACC2075D8F97F7FF1F60
:1056400083C757ABE207D98F17F7FF1F2320F7A8AF
:1056500083C7640097B501009385050C17B5010059
:105660001305C58C17F7FF1F2301F7A697900100BC
:10567000E78040DE97F7FF1F938747A58C4317F617
:10568000FF1F034686A417B50100130525B39790A5
:105690000100E78020DC294597900100E78060E069
:1056A00097F7FF1FA38607A42244B2409244024901
:1056B000930700F817F7FF1F230CF7A29D4517F576
:1056C000FF1F1305E5A2410117430000670003D83F
:1056D00097600000E780808897F7FF1F238BA7A0C3
:1056E0009357850017F7FF1FA305F7A093570501F0
:1056F0002A8417F7FF1F230FF79E93578501014553
:1057000017F7FF1FA308F79E97600000E780C0858A
:1057100097F7FF1F2381A79E97B501009385C5FFCB
:1057200017B501001305858097900100E78080D2AE
:1057300017F6FF1F0346269CA28517B50100130527
:1057400065A9B1B7CD476303F40297B5010093850E
:10575000A5FC17A501001305657D97900100E78062
:1057600060CF17B50100130565A879BD37E40400C3
:105770007C44414697F5FF1F9385959717F5FF1FCA
:1057800013050595829717F5FF1F1305659497106C
:105790000000E78080C497100000E78000AC97F716
:1057A000FF1F83C7079617F7FF1F03477795A207C9
:1057B00003238405D98F17F7FF1F2317F7901306CC
:1057C000000A89452244B2409244024917E5FF1F6E
:1057D00003454505410102838D476303F40297B5F4
:1057E0000100938565F317A50100130525749790B3
:1057F0000100E78020C617B501001305E5AE29B505
:1058000017F4FF1F0344E48E97F7FF1F83C7578EDB
:1058100097B50100938545F0220417A501001305F3
:10582000E5705D8C97900100E780C0C2A28517B536
:1058300001001305259D97900100E780A0C129452F
:1058400097900100E780E0C50D4697F5FF1F93850F
:10585000258A228597E0FFFFE7802064AA8421C182
:1058600097B50100938545EB17A501001305056C5D
:1058700097900100E78000BEA68517B501001305CB
:10588000A59997900100E780E0BC2244B240924481
:1058900002492945410117930100670083C097E73A
:1058A000FF1F2399877AB7E70400116603A38705D2
:1058B000130606E8914539B78D476303F40297B59F
:1058C0000100938565E517A50100130525669790EE
:1058D0000100E78020B817B501001305A5AF2DB36F
:1058E00017F4FF1F0344E48097F7FF1F83C7578017
:1058F00097B50100938545E2220417A50100130521
:10590000E5625D8C97900100E780C0B4A28517B571
:1059100001001305A59197900100E780A0B32945E8
:1059200097900100E780E0B70D4697E5FF1F93854C
:10593000257C228597E0FFFFE7802056AA841DC1C1
:1059400097B50100938545DD17A501001305055E98
:1059500097900100E78000B0A68517B501001305F8
:10596000258E05B797E7FF1F2398876CB7E70400DC
:10597000116603A38705130606E89305000299B58F
:10598000894763E3870297B501009385E5D817A59A
:1059900001001305A55997900100E780A0AB17B54A
:1059A00001001305E5A58DB197E4FF1F83C464745E
:1059B00097E7FF1F83C7D77397B501009385C5D5B8
:1059C000A20417A5010013056556DD8C9790010010
:1059D000E78040A8A68517B501001305E5879790D5
:1059E0000100E78020A7294597900100E78060AB80
:1059F000228697E5FF1F9385A56F268597E0FFFF19
:105A0000E780A0492A84630E051A97B501009385A3
:105A1000A5D017A501001305655197900100E780F7
:105A200060A3A28517B501001305458499BD85477C
:105A300063F98718834519002244B2409244024911
:105A4000B335B00097E7FF1F2380B76217B5010099
:105A5000130505834101179301006700A39FA285E9
:105A60002244B24092444A85024941011703000092
:105A70006700032299476303F40297B501009385F9
:105A8000A5C917A501001305654A97900100E78095
:105A9000609C17B50100130565B0BDB617E4FF1F84
:105AA0000344246597E7FF1F83C7976497B50100F8
:105AB000938585C6220417A50100130525475D8C33
:105AC00097900100E7800099A28517A501001305B2
:105AD000A57C97900100E780E09729459790010009
:105AE000E780209C194697E5FF1F93856560228516
:105AF00097E0FFFFE780603AAA841DC197B50100D7
:105B0000938585C117A501001305454297900100B3
:105B1000E7804094A68517A501001305E57895B3A5
:105B200097E7FF1F239E875AB7E70400116603A378
:105B30008705130606E89305000869B1854797B500
:105B40000100938565BD17A501001305253E630B74
:105B5000F40097900100E780E08F17A5010013057E
:105B6000E5755DB497900100E780C08E17A5010030
:105B70001305457697900100E780C08D29459790E1
:105B80000100E78000922244B2409244024997E724
:105B9000FF1F239B07524101175300006700832C0E
:105BA00097B50100938545B717A501001305053882
:105BB00097900100E780008A17B50100130545A200
:105BC000A1B4B24022449244024941018280411171
:105BD00006C622C497E0FFFFE780202C9377F50FDD
:105BE000A1C32A8497B50100938585B417A5010048
:105BF0001305C53397900100E780C0859375F40FB6
:105C000017B50100130585D197900100E7808084C6
:105C10002244B2402945410117930100670063887F
:105C2000B240224441018280411122C491462A841B
:105C300017E6FF1F1306065A9D652D4506C697D029
:105C4000FF1FE780A0B6B7F7070003C70701A54706
:105C50006313F70001A09306001001469D652545DA
:105C600097D0FF1FE78080B497E7FF1F23848756F4
:105C70002244B240914617E6FF1F1306A6559D65C4
:105C80002945410117D3FF1F670043B25171CAD1A3
:105C900037E904008327C904A2D52E8686D7A6D368
:105CA0002E84AA8517E5FF1F13058544829797E781
:105CB000FF1F83C7E7431307700A6387E710636C0E
:105CC000F7001307600A6384E704BE502E549E5405
:105CD0000E596D6182801307800A6388E7161307E7
:105CE000900AE394E7FE8D476309F41C97B5010021
:105CF000938505D617A5010013054523978001005C
:105D0000E780407517B501001305C5D125A08D4763
:105D1000630CF40297B50100938585D317A50100A4
:105D20001305C52097800100E780C07217B50100F8
:105D3000130585C897800100E780C07129459780C9
:105D40000100E780007651B7854717B501001305BC
:105D500065C817E7FF1F2309F73097900100E78018
:105D60004087B7750200B76602000146054597D027
:105D7000FF1FE780A0A3930760F817E7FF1F230921
:105D8000F73697E7FF1FA38607369307002617E726
:105D9000FF1F2321F736E5779387072117E7FF1FBA
:105DA000231CF734B14597E7FF1F2388073497E793
:105DB000FF1FA384A73417E5FF1F13056533973032
:105DC0000000E780A06811B7914763E3870297B5A9
:105DD00001009385E5C717A50100130525159780D8
:105DE0000100E780206717B501001305A5C099B72A
:105DF00097E4FF1F83C4043097E7FF1F83C7772F03
:105E0000A204DD8C8327C9046D14228697E5FF1F49
:105E10009385552E280082978E0493160401B7753A
:105E20000200C1823000A695094597D0FF1FE78088
:105E3000E097930770F817E7FF1F230BF72A9945A0
:105E400097E7FF1FA388A72ABDB7914763E387029F
:105E500097B501009385C5BF17A501001305050D72
:105E600097800100E780005F17B50100130505BAB0
:105E7000D1B597E4FF1F83C4E42797E7FF1F83C7CB
:105E80005727A204DD8C8327C9046D14228697E569
:105E9000FF1F93853526280082978E0493160401F0
:105EA000B7750200C1823000A6950D4597D0FF1F3F
:105EB000E780C08F930780F8BDBF17B501001305B9
:105EC000A5B797800100E780C0701305C01297C086
:105ED000FF1FE7800047014597D0FFFFE78080184C
:105EE0000D4597000000E78060D4294597C0FF1F4B
:105EF000E780204597C0FF1FE7808035F9B3411147
:105F00004AC097F6FF1F83D6867E328917D6FF1FB9
:105F10000356E64822C426C206C62A84AE849700E9
:105F20000000E780C05F35C12DC0994763FF97042B
:105F30008347140003470400A207D98F13978700F3
:105F4000A183D98FC2073167C1831307C755639EE9
:105F5000E70297D7FF1F83D78744A301F400A183EB
:105F60002302F40097F7FF1F83D7677891C7A30236
:105F7000F400A1832303F400A68517B501001305DF
:105F800025B197800100E780E04C97F7FF1F83C79A
:105F9000A765B9CF97D5FF1F83D5654017B5010019
:105FA0001305C5B097800100E780C04A2686A28508
:105FB00017D5FF1F0355A53E97000000E78060C17D
:105FC0006301090497E7FF1F83C7C7219DCB95C8CD
:105FD00097E7FF1F83C747098DE722852244B24018
:105FE0000249A68592444101173300006700034629
:105FF00017B50100130585AC97800100E780605D4F
:10600000C1B7B24022449244024941018280834791
:1060100055008345450017B50100130525A6A207C5
:10602000DD8D178301006700E34217B501001305FA
:10603000E5A3178301006700C3598D4763FBB70AC7
:10604000011126CA06CE22CC0344350097E4FF1F77
:1060500083C4541997B50100938505A7B337800011
:1060600017E7FF1FA300F71809C497B50100938530
:1060700065A617B50100130565A697800100E780A6
:10608000603D97E7FF1F83C7F7156386970097006A
:106090000000E780802697E7FF1F83C7B7148DC7EE
:1060A00085472306F100B7E7040083A74717700070
:1060B000854513055030829717B50100130505A3D8
:1060C00097800100E780E0509967938757EE231689
:1060D000F100680085479145A30781002307F1007F
:1060E00097300000E7808036F2406244D244056178
:1060F00082808280894763F7B708011122CC06CEDF
:1061000026CA8344250085472A84639DF404914769
:1061100063F5B704034545008347340022055D8DD0
:1061200097D7FF1F239DA72697000000E780004810
:106130009967938767EE2314F100834734002305A2
:106140009100A305F10083474400954528002306EC
:10615000F10097300000E780602FF2406244D244A3
:1061600005618280FDF89967938767EE2314F1003B
:1061700097D7FF1F83D7A722A305F10023050100AE
:10618000A183E1B782800111996722CCD51717F45A
:10619000FF1F130464452314F1008347040026CA3B
:1061A00097F4FF1F9384A4542305F10083D70400C0
:1061B00028009545A305F100A18306CE2306F10032
:1061C00097300000E780802803D604008345040050
:1061D00017B501001305059397800100E78080271C
:1061E000F2406244D244056182809D677971D9177B
:1061F0002316F10097F7FF1F83C7073F06D6230733
:10620000F100A9C3B7E70400FC47414697E5FF1F2B
:10621000938505EC1305F10082976800CD45973012
:106220000000E780A02297F5FF1F83C5E53B17B567
:1062300001001305259097800100E780A021B2504E
:1062400045618280B7E70400BC474146814513059C
:10625000F1008297D9B7B76702045D71938757AA97
:106260003EC08567938707F02312F10097F7FF1F61
:106270009387873783C70700A2C4A30301002303C2
:10628000F10097F7FF1F9387874683D7070037E40E
:10629000040086C62314F10097D7FF1F93872710A9
:1062A00083D70700414668002315F1007C4497E539
:1062B000FF1F9385E5E18297F1450A85970000006D
:1062C000E780E021231EA1007C448A8508107946DE
:1062D00082973C441305E1030946814582971010DB
:1062E00093050002014597D0FFFFE780003EB640CE
:1062F000264461618280B7C7A55A01119387C733CD
:106300003EC497E7FF1F83C7F7ED3EC6B7F7070008
:1063100003C7070106CE22CCA5476313F70001A0EF
:106320001164930504F0930600100146254597C0BB
:10633000FF1FE780A0473000930504F0A1462945E0
:1063400097C0FF1FE780804697E5FF1F83C595E94B
:1063500017B501001305C58E97800100E780800FF7
:10636000F24062440561828001119165A1463000CE
:10637000938505F02D4506CE97C0FF1FE7800043AB
:106380002247B7C7A55A9387C7336314F702B245AC
:1063900017A501001305057EB335B00097E7FF1F71
:1063A000A382B7E497800100E780C00AF24005614C
:1063B0008280814517A501001305057E97E7FF1F21
:1063C000A38207E297800100E780C00897000000E1
:1063D000E780A0F2E1BFB7C7A55A79719387F73577
:1063E0003EC6B7E70400FC47AA8506D622D441463C
:1063F00008088297B7F7070003C70701A54763138B
:10640000F70001A01164930504E89306001001460B
:10641000254597C0FF1FE78060397000930504E8A9
:10642000D146294597C0FF1FE780403817B50100C6
:106430001305C58497800100E780A019B25022544B
:106440004561828079719165D1467000938505E838
:106450002D4506D697C0FF1FE78040353247B7C7A6
:10646000A55A9387F73517A501001305E57A631040
:10647000F702B7E70400FC4717E5FF1F130545C502
:1064800041460C08829717A501001305E576978011
:106490000100E7800014B25045618280B7F7070021
:1064A00003C70701A5476313F70001A091654111D8
:1064B000930600100146938505E8254506C697C05A
:1064C000FF1FE780A02EB24017A501001305C56885
:1064D0004101178301006700C30FC16769768146D8
:1064E000FD1705061397060141836364B7003E85D7
:1064F00082803307D50003470700B98F214713F87F
:106500001700858363050800B18FC207C1837D171B
:106510001377F70F6DF78506F1B741C5A547054716
:1065200063F2B70883471500034705003168A207E7
:10653000D98F13978700A183D98FC207C18313080E
:10654000C855054763900707411106C622C426C2F5
:1065500003442500914763F087049307540063ECDC
:10656000F502A301C50021822302C5009304340073
:1065700091C6A302D500A1822303D5002A84A68553
:1065800097000000E780A0F526942300A400218155
:10659000A300A4000147B240224492443A8541013D
:1065A000828005473A858280B7C7A55A0111938733
:1065B000E7343EC42AC6B7F7070003C7070106CE73
:1065C00022CC26CAA5476313F70001A091642A8450
:1065D000938504EE930600100146254597C0FF1FE2
:1065E000E780C01C3000A146938504EE294597C082
:1065F000FF1FE780A01BA28517A5010013054566B4
:1066000097800100E78000E597000000E780E0C484
:10661000F2406244D2440561828001119165A14635
:106620003000938505EE2D4506CE97C0FF1FE7800D
:10663000E0172247B7C7A55A9387E7346318F702D4
:10664000B24517A501001305255797D7FF1F2398BB
:10665000B7D4C205C18197800100E780A0DF970011
:106660000000E78080BFF24005618280D147D145BC
:1066700017A501001305455617D7FF1F2311F7D2A1
:1066800097800100E78000DD17D5FF1F035525D156
:1066900097000000E78080F1F9B721C1411126C2BF
:1066A00006C622C4AE848DC52A8497200000E780E8
:1066B00040BB97E7FF1F83C7E7B299CB22852244EF
:1066C000B240A6859244410117330000670003D809
:1066D000B2402244924441018280828079714AD042
:1066E00006D622D426D24ECE93F715002E899DCB06
:1066F000AD67371700409387A7AA1CC3B7E704000C
:10670000BC4F13060019854517D5FF1F034505C962
:10671000829713451900B250225492540259F249FB
:106720004561828093F725006383071E2D4697A558
:1067300001009385A558480097800100E78020C696
:1067400097F6FF1F83C686FA139706014183954784
:1067500063F9E70C014417F5FF1F130525E913063C
:10676000300513085004930810041303B004130EEB
:1067700090059307640063F4F6043A84FD5997F496
:10678000FF1F83C4A4E697F7FF1F83C737E6A20461
:10679000DD8CAD679387B7556387F41463E3970A7D
:1067A000A9679387A755638AF414A28517F5FF1F7D
:1067B0001305C5E397000000E78060EE11A2B30760
:1067C000850083C50700639AC50483C517006396D7
:1067D000050583C527006392150583C53700639EB1
:1067E000C50283C54700639A650283C75700639655
:1067F000C703A2890DE897F5FF1F83C525EFB38571
:106800003541C20517F5FF1F130545DEC1814E95C1
:1068100097000000E780A0E8C1A005044204418081
:1068200089BF3A84FD598547E3EB87F45DC0854510
:1068300017F5FF1F130585DB97000000E78020E6B2
:1068400049A8B1679387C7556380F404B5679387F8
:10685000D755E39CF4F4A28517F5FF1F130505D95E
:1068600097300000E78080BE8947630BF4049305EE
:10687000E4FFC205C18117F5FF1F130545D7972017
:106880000000E780009E2DA80546A28517F5FF1F92
:106890001305C5D597F0FFFFE780A06697F7FF1FA8
:1068A00083C787D491EF480097800100E78020DB01
:1068B00093150501C181480097D0FFFFE780008F45
:1068C000A68517A501001305653D97800100E780A7
:1068D00060B8FD57E391F9F297F7FF1F238807E0AF
:1068E000134529000DBDA28517F5FF1F130505D01F
:1068F00097F0FFFFE780E071E1B7A28517F5FF1F72
:106900001305C5CE97F0FFFFE780607255BF93F780
:1069100045000145E38107E017A50100130545394E
:1069200097800100E780E0CA97300000E78000C14F
:1069300013454900CDB3411122C437E404005C5C27
:1069400006C6354697A50100938585E717B5010072
:10695000130585A1829711E917A501001305C53616
:1069600097800100E780E0C601A08327041C82977E
:106970002A84054597B00000E780207A97600100DF
:10698000E78040FF97600100E78040D497B00000A7
:10699000E780A08B2285B2402244410182801567A6
:1069A000B71700401307575598C3D8439D66558FB6
:1069B000D8C3D843FD76758FD8C3D8431367F70F74
:1069C000D8C335671307C7CC98C3828041110545EA
:1069D00006C622C426C297C0FFFFE7808052130577
:1069E000800497B0FF1FE780806C757585457D1525
:1069F00097C0FFFFE780203C7D7585451305F53680
:106A000097C0FFFFE7808045371400408327840A42
:106A10008D451305002093E707202324F40A97C02F
:106A2000FFFFE7804039B7E4040097C0FFFFE7802D
:106A3000607EC85897800100E780A0B917B50100B3
:106A40001305859297800100E780A0B88327840C06
:106A50008545414593E707082324F40C97C0FFFFC1
:106A6000E780C03F8D451305000897C0FFFFE78012
:106A7000E03E97C0FFFFE780C06B014597C0FFFF76
:106A8000E780806E85450545894717F7FF1F23017D
:106A9000F7C697C0FFFFE780C06E37070004B7E76F
:106AA00000E023A0E71097D0FFFFE780600097D0B9
:106AB000FFFFE780201497000000E78000E89700C0
:106AC0000000E780A08A97000000E78040B597E0CB
:106AD000FFFFE78000F097000000E780601097005C
:106AE0000000E780600B83A704081705000013056A
:106AF00025BF829797D7FF1F2382A78ABC4C130616
:106B000000648545829797000000E78080E997C080
:106B1000FF1FE780E08D01458280B7F7070003C7BC
:106B20000701A547AE866316F7009397450191C309
:106B300001A0AA850146254517C3FF1F670003C7AB
:106B40004111B2862E86AA852D4506C697C0FF1F25
:106B5000E780C0C5B240014541018280930700042F
:106B600063E8C7021D71A2CC2A84080886CE32C60B
:106B700097800100E780A082B2461008A2852945CF
:106B800097C0FF1FE78080C2F6406644256182807F
:106B90003955828041110D658D4506C697C0FFFFAE
:106BA000E7806021B71700408D6623A6D70A17F546
:106BB000FF1F130525B41387C70A9387870A1CC1D3
:106BC0005CC5856689675CC958C114C518C9B7E733
:106BD0000400B24003A3871E4101028397F7FF1F01
:106BE00083C7C7B299EF411106C697100000E7802E
:106BF0006061B240854717F7FF1F2309F7B04101D5
:106C00008280828011C589C517C3FFFF6700035AC0
:106C10008280411126C2AE848D4522C406C62A84D4
:106C200097C0FFFFE7808023B717004099C803A5EE
:106C3000C70C418D23A6A70CB240224492444101C7
:106C4000828003A5870C418D23A4A70CF5B7834749
:106C5000050003471500A207D98FC2076177C187D6
:106C600013072720639AE7008345250037050400B2
:106C700017030000670023FA828017F6FF1F130630
:106C800026A98147B2861303F00FA9483308F600FE
:106C90000348080013F7F70F6307A80C63066800A2
:106CA0008507E39517FF2947B387E6002380A700F0
:106CB00097F7FF1F938787A65DA8411113D765003B
:106CC0001347170006C693F63500058B954791CA02
:106CD000054699476387C60009469D476383C600FA
:106CE000A14713F645003336C00093F68503050629
:106CF00085C2A145638BB604E145638AB60493055A
:106D000080026388B604930580036393B6009146BE
:106D100097F5FF1F2389F5C697F5FF1F2384C5C686
:106D200097F5FF1FA380D5C6BE8517A501001305E3
:106D3000250397700100E780E071B240854717F79F
:106D4000FF1FA302F7C4410182808546D1B789465F
:106D5000C1B78D4675BF17A501001305E50217736E
:106D600001006700236F17F7FF1F1307279BBA97D0
:106D70002380B700E147E302F5F493077002E30CC8
:106D8000F5FC82802A8723800500814717F5FF1FC5
:106D9000130505981308F00F2946B306F50083C6BE
:106DA00006006396E60297F6FF1F93862697B6972E
:106DB00083C7070005452380F5009947636EF702F6
:106DC0009D4763FDE700E147630DF700828063851F
:106DD00006018507E393C7FC0145C5B7238005007D
:106DE0008280B737004003C7370083C7050093F799
:106DF0000704D98F2380F5008280797126D24AD08A
:106E000097F4FF1F83C404CA17F9FF1F1309C9C8E9
:106E100006D622D44ECE52CC56CA5AC8B3079900D1
:106E200083C7070093F7F70FA5C79387140093F75D
:106E3000F70F0D476361F70C17F7FF1F2304F7C621
:106E400097F7FF1F9387C7C5A69783C70700130748
:106E5000100293F7F703638FE7286363F70A05448B
:106E600063808720E389076E09476389E714130766
:106E70000002E38EE758B7E700E03707400023A0A1
:106E8000E71801000100CA942380040023A0E71042
:106E9000B787004003C76700058BE30F077897F6B5
:106EA000FF1F83C646C00547E39AE676294723813C
:106EB000E70209472383E7022385E70297F7FF1FCD
:106EC000A38407AC97F7FF1FA38F07BCB7870040C9
:106ED000A381070017F7FF1FA30A07AA054723830B
:106EE000E700B250225492540259F249624AD24AFF
:106EF000424B4561828097F7FF1F238507BA89B708
:106F0000130730026386E70A63E6E71413074002BB
:106F1000638AE70813070003E39FE7F497F7FF1F6F
:106F20009387C7B7A69703C70700A1471377F70F43
:106F3000E31AF71C17EAFF1F130A0A7F83476A0048
:106F400097F6FF1F2388F6A297E7FF1F83C7377EB8
:106F500091C7FD5797F6FF1F238EF6A097E5FF1FF9
:106F600083C5957C97F7FF1FA386B7A097E7FF1F00
:106F700083C7877B93F907089306000493F70706F6
:106F80006393D7529307A009638DF51A63EAB71686
:106F90009307F005638AF54E930750096388F52E31
:106FA000014479ABFD5717F7FF1F2304F79CE1B5A8
:106FB000FD5717F7FF1F230DF79A75BD17A50100A1
:106FC000130505EE97700100E780A06097F7FF1F9B
:106FD0009387C7ACA69703C40700814917FAFF1F20
:106FE000130A0A8D1374F40F97AA0100938ACAEB4F
:106FF00063C78904294597700100E780804A854767
:1070000017F7FF1FA304F78A17F7FF1F2301878ACB
:1070100017F7FF1F230AF79637E700E0B70640008F
:107020002320D71801000100378600408347A602BD
:1070300093F7370F2305F6022320D7102DBDB30792
:107040003A0183C507005685850997700100E780DE
:10705000604079BF854717F7FF1F2309F78421BDDB
:1070600017A501001305C5E397700100E78060567E
:1070700097F7FF1F938787A2A69703C4070081494C
:1070800017EAFF1F130A8A761374F40F97AA0100F8
:10709000938A8AE163C58904294597700100E780D6
:1070A0004040854717E7FF1FA300F77417E7FF1F4E
:1070B000230D877217F7FF1F2308F78C37E700E0CF
:1070C000B70640002320D718010001003786004092
:1070D0008347660293F7370F2303F602B1BFB30766
:1070E0003A0183C507005685850997700100E7803E
:1070F00060364DB7854717E7FF1F2307F76EA5BB1F
:107100009307400A638DF5349307200B6388F536A7
:107110009307100AE396F5E883072A00014463D138
:10712000074297E7FF1F83C7576093F63700638EC8
:10713000061A0546638EC62209466399C61A1D477C
:1071400075A217E5FF1F0345455EC94717EAFF1FF4
:10715000034ABA5D97E5FF1F83C5455D17E4FF1F2E
:107160000344D45C6319F510CD476316FA109307F6
:107170007008639CF5021307300FB7170E00630801
:10718000E4001307900DB7B704006314E40817E791
:10719000FF1F2327F77EBE8517A50100130545D1E4
:1071A00097700100E780002BE5BB93078008639D83
:1071B000F50033048040B77746001374F40F9387CB
:1071C00087CDB3D78702E1B793079008639AF5009C
:1071D0003304804091671374F40F9387C766D5B763
:1071E0009307A008639BF50033048040B7173D0068
:1071F0001374F40F93870790E9B79307B008639A65
:10720000F5003304804091671374F40F938797D08F
:107210004DBF93F5F5078D47639BF5003304804020
:10722000B7975B001374F40F938707D859BF89474A
:10723000639BF50033048040B7770B001374F40FA1
:107240009387071BBDBF8547639AF50033048040D1
:10725000DD671374F40F938767E3A5B789E93304F7
:1072600080408D671374F40F938777DC99BFF167C3
:107270009387072029BF97000000E78040A0A285E0
:10728000528597000000E780809F19BB930561003D
:1072900017E5FF1F0345654917E4FF1F0344F44842
:1072A00097000000E78040AE9305710022859700AB
:1072B0000000E78060AD3C0017E7FF1F232CF77C40
:1072C000834761002304F10083477100A304F100A8
:1072D000894717E7FF1F230FF7688357810017E7D8
:1072E000FF1F2313F7440944A1AC154793F6470049
:1072F000B336D00093F78703850685C32146638B99
:10730000C7066146638AC706130680026388C706FC
:10731000130680036393C700914717E6FF1F2303FB
:10732000D66697E6FF1FA38FF66497E7FF1F238CAF
:10733000E76417E7FF1F0347673F9376070497E764
:10734000FF1F83C7B73E8DEE1377770C9306700847
:10735000630CD7021377F7078D46631ED70AB3076E
:10736000F040B7955B0093F7F70F938505D881A898
:107370001947ADBF854755B7894745B78D4771BF99
:10738000930670086311D7021307300FB7150E006C
:107390006389E7021307900DB7B504006383E70222
:1073A0001307700845BF9306800C6311D702B3071B
:1073B000F040B775460093F7F70F938585CDB3D5A9
:1073C000F50297E7FF1F23ADB75AF9B39306900C68
:1073D000631AD700B307F040916593F7F70F9385D1
:1073E000C566F1BF9306A00C631BD700B307F0403E
:1073F000B7153D0093F7F70F93850590C9B793062E
:10740000B00CE319D7F4B307F040916593F7F70F89
:10741000938595D06DB78946631BD700B307F040BD
:10742000B7750B0093F7F70F9385051B49BF85468A
:10743000631AD700B307F040DD6593F7F70F938524
:1074400065E3B5BF09EBB307F0408D6593F7F70F20
:10745000938575DCADB7F165938505209DB78347AE
:107460002A00C18B99C7854717E7FF1F2307F750ED
:1074700005BE97E7FF1F238207501DB6854717E714
:10748000FF1FA302F75029BE3C0017E7FF1F23236D
:10749000F7600947930700032314F10097E6FF1FE5
:1074A000238AE64C2DBD639A0758A94763ECB7447D
:1074B00017A70100130707888A05BA959C41BA9758
:1074C000828717E4FF1F03445426094A630C440FC4
:1074D000636C8A0885476309F40A9307F00F17E77E
:1074E000FF1F0347274963F6E70017E7FF1F230342
:1074F000F74817EAFF1F034AEA479307000413748B
:10750000FA0F63F447011304000497E7FF1F938702
:10751000675883AA0700228617E5FF1F1305C520B9
:10752000D685330A8A40A29A97700100E78020E747
:1075300097E7FF1F2380474597E7FF1F23AC575569
:1075400097E7FF1F83C717431547639AE762B7E7BB
:1075500000E03707400023A0E71801000100B786CC
:107560000040238086028DA58D47630CF40A99475D
:10757000E315F4F697A701009387478217E7FF1FEB
:10758000232AF750A947A1BF17E7FF1F0347A751B9
:1075900097E7FF1F93870740494697A5010093850A
:1075A000E5886306870097A50100938525843E85BD
:1075B00097700100E780A0DE17E7FF1F232CA74C80
:1075C000C94731BF97E6FF1F83C6E64D054797E7DA
:1075D000FF1F9387273C6394E6023E8513067002E3
:1075E00097A501009385058297700100E78020DB55
:1075F00017E7FF1F2320A74A93077002CDB53E85EA
:1076000013063004979501009385057A9770010061
:10761000E780E0D817E7FF1F232EA7469307300423
:107620007DBD97E5FF1F83C5451017A50100130514
:10763000658997700100E780E0E1854A17EBFF1F3D
:10764000034B6B4697E5FF1F83C5250E17A5010069
:107650001305458763185B0B97700100E78080DF97
:1076600097E7FF1F83C7670CB5CBE368F4E6179471
:1076700001001304E47F638C670117940100130475
:10768000A47F6386470117A4010013046480228548
:1076900097700100E780A0FC1375F50F93071500A4
:1076A000860717E7FF1F2307F72E8D4717E7FF1FF2
:1076B000A302F72E97E7FF1F9387C72D0147BE86CA
:1076C0001376F70F89076365A60297E7FF1F23A3C9
:1076D000D73C97E7FF1F83C7E72B11B597970100AA
:1076E0009387077217E7FF1F2326F73A9147C5BB19
:1076F0003306E40003460600A38007000507238045
:10770000C7007DBF97700100E780C0D497E7FF1FD7
:1077100083C7A701E1D7E362F4DC179401001304E7
:107720002472638C5701179401001304E47163867B
:107730004701179401001304A47222859770010079
:10774000E780E0F11375F50F93071500860717E73B
:10775000FF1F2301F7248D4717E7FF1FA30CF72214
:1077600097E7FF1F938707230147BE861376F70F1E
:107770008907E37CA6F43306E40003460600A380F1
:10778000070005072380C700D5B797E5FF1F83C50E
:10779000C5F9179501001305A57397700100E780DF
:1077A00060CB97E7FF1F83C7B71E93E7470017E734
:1077B000FF1FA30FF71C83472A0017E7FF1FA3072C
:1077C000F71C6FF0EFFD179501001305A571977079
:1077D0000100E78000E097E7FF1F9387271B83C71F
:1077E000070017E7FF1F2301F7F417E4FF1F034407
:1077F000641833348000A9B3179501001305C56FD1
:1078000097700100E780E0DC97E7FF1F83C75718F8
:1078100093E7070117E7FF1FA30CF71683472A001A
:1078200017E7FF1F2304F7166FF08FF71795010076
:107830001305C56D97700100E780A0D903470A00C2
:107840007D8B51EFB787004003C767021377C70BE3
:10785000136727002383E70203C7A7021377C70B29
:10786000136727002385E70203C7E7021377C70BD7
:10787000136727002387E70203C727031377C70B84
:10788000136727002389E702854717E7FF1F230DAA
:10789000F7F417E7FF1F230BF70017E7FF1F230974
:1078A000F70C17E7FF1F2306F70C97E7FF1FA38DC1
:1078B00007F297E7FF1FA38B07FE97E7FF1FA38938
:1078C000070A97E7FF1FA386070A97E7FF1FA38D05
:1078D000070A97E7FF1FA388071C6FF06FEC894723
:1078E0006312F70297E7FF1F83C747E49146638C53
:1078F000D70863E0F604638EE70C6369F70A05476F
:107900006380E70EFD5717E7FF1FA305F70637074C
:107910004000B7E700E023A0E71801000100B786A8
:1079200000401306F0FC2381C60223A0E7106FF08D
:107930008FD4130720086382E7086362F7021307F6
:107940001008E391E7FC378700408347670293F70D
:10795000C70B93E727002303F7026FF06FE41307C9
:1079600030086389E70213074008E39DE7F837878B
:1079700000408347270393F7C70B93E727002309AA
:10798000F7026FF0EFE1378700408347270393F753
:107990003707F5B7378700408347E70293F7C70BF0
:1079A00093E727002307F7026FF08FDF3787004048
:1079B0008347E70293F73707F5B7378700408347D8
:1079C000A70293F7C70B93E727002305F7026FF091
:1079D0002FDD378700408347A70293F73707F5B7B6
:1079E000378700408347670293F73707ADB717958E
:1079F00001001305A55297700100E78080BD97E74D
:107A0000FF1F238307D2D5B3179501001305055235
:107A100097700100E780E0BB97E7FF1F239607D030
:107A200097E7FF1F938707F503C40700894763F3B0
:107A3000870009441374F40F21B613070002E3937F
:107A4000E7EC6399090A638FF500930720026381CD
:107A5000F508179501001305E55097700100E780C0
:107A6000609F4DB5179501001305054D97700100F6
:107A7000E78020B60144179B0100130B2B4DA14A50
:107A8000B3078A0083C507005A8505049770010073
:107A9000E780409CE31654FF179501001305C5AF1E
:107AA00097700100E780E0B217E4FF1F034404C8A9
:107AB00011E497E7FF1F238C07C459B48947E313E8
:107AC000F4E4854717E7FF1F2303F7C46FF04FCD9A
:107AD00017E6FF1F034676C597E5FF1F83C5E5C47C
:107AE000179501001305054797700100E780809600
:107AF0006FF00FCB638FF50493071002E39BF5F44F
:107B000097E5FF1F83C585C21795010013058546BC
:107B100097700100E780009497E7FF1F23AC47F7B9
:107B200097E7FF1F9387C7E5944383D7470017E77D
:107B3000FF1F034747E517E6FF1F2327D6BE1D4457
:107B400097E6FF1F2394F6BE97E7FF1F2381E7BE4A
:107B5000C5BA97E5FF1F83C565BD179501001305DD
:107B6000E54297700100E780E08E97E7FF1F2380D2
:107B700007BA97E7FF1F239907BA6FF0CFF625479B
:107B8000E387E79C19476391E702B78600402380AB
:107B90008602B7E700E03707400023A0E71801009E
:107BA0000100130600FC41B31307100A6391E702BA
:107BB000B786004023808602B7E700E03707400021
:107BC00023A0E71801000100130680FCA9BB1307DE
:107BD000A009E38FE7FC1307400AE38BE7FC1307D8
:107BE0002002E386E7960547E383E796B7E700E0E0
:107BF0003707400023A0E718E39109960100010030
:107C0000B786004023808602130620FC29BB17E7B5
:107C1000FF1F034737D66308F71E63E7E702954760
:107C2000630EF70E99476308F704B7860040238078
:107C30000602B7E700E03707400023A0E71801007D
:107C400001001306A0FCC5B19307F005630AF70015
:107C5000930750096306F70093071002E317F7FC38
:107C6000B7E700E03707400023A0E7180100010054
:107C7000B786004051BF97E9FF1F83C9A9CF93077B
:107C80000004CE8A63F43701930A000497E7FF1FCC
:107C9000938747E003AA070013F4FA0F2286D285E0
:107CA00017E5FF1F130545A897600100E780206FC7
:107CB000B3878940529417E7FF1F230DF7CA97E750
:107CC000FF1F23A987DC638E0902B787004023804A
:107CD0005703B7E600E03706400023A0C6180100AE
:107CE000010003C72702134707042381E70203C7E4
:107CF00027021377C70F2381E70223A0C6106FF076
:107D00008F97B786004023800602B7E700E0370769
:107D1000400023A0E71801000100FDB537870040AF
:107D20008347370097E6FF1F83C656C693F70708B9
:107D3000D58FA301F700B7064000B7E700E023A006
:107D4000D718010001001306A0FC2301C70223A0DD
:107D5000D7106FF04F9297E7FF1F938727D4A6970E
:107D600083C7070093F7F70FD9CF97E7FF1F83C7A4
:107D700087D3D1EB17E7FF1F0347D7BF9307000255
:107D80006313F70897E7FF1F9387079A03AB070072
:107D900097EAFF1F83CA8A9917EAFF1F034A1A99B5
:107DA00097E9FF1F83C9A998D2875687CE865A863E
:107DB00097E5FF1F83C5A595179501001305851E3F
:107DC00097600100E780006997E7FF1F23AA67BB60
:107DD00097E7FF1F238857BB97E7FF1FA38447BB85
:107DE00097E7FF1F238137BB97E7FF1FA380879289
:107DF000B7E700E03707400023A0E71801000100C3
:107E0000B7860040D1B3B7E700E03707400023A0B2
:107E1000E71801000100B786004025B529472381F6
:107E2000E70209472383E7022385E7022387E70266
:107E30002389E7026FF08F8803C76700118B630205
:107E4000078A83C75700918BB5CF17E7FF1F0347FA
:107E500087C585476313F70697E7FF1FA385E7B23A
:107E600097E7FF1F2382079897E7FF1F238007A448
:107E700097E7FF1F238E07AE97E7FF1F238B07AE01
:107E800097E7FF1FA382079697E7FF1FA38007A22C
:107E900097E7FF1FA38E07AC97E7FF1FA38B07ACE5
:107EA00097E7FF1FA38207AE97E7FF1FA38D07BECB
:107EB000B787004011476FF08F8217E7FF1FA307B6
:107EC000F78479BF854717E7FF1F230FF79017E760
:107ED000FF1F230DF79C17E7FF1F230BF7A817E7DA
:107EE000FF1F2308F7A869BF854717E7FF1F230D6A
:107EF000F78E17E7FF1F230BF79A17E7FF1F2309DA
:107F0000F7A617E7FF1F2306F7A617E7FF1FA30D26
:107F1000078C17E7FF1FA30B079817E7FF1FA3099D
:107F200007A497E7FF1FA38607A48280411106C616
:107F300097000000E78080FBB787004023800700A0
:107F4000130740FC2386E7001307C004A386E7005D
:107F500017D7FF1F1307477D2398E70017E7FF1F79
:107F600013078780239AE70017E7FF1F1307078C83
:107F7000239CE70017E7FF1F13078797239EE7005F
:107F800029472381E70209472383E7022385E70284
:107F90002387E7022389E702A3810700930600F8FD
:107FA000A380D700930690022380D700FD56238339
:107FB000D7002381E700B706400037E700E0232021
:107FC000D71003C7170013671700A380E700B2405C
:107FD00097E7FF1F239C079A41018280411106C643
:107FE00097000000E78080F0B787004023800700FB
:107FF000130700FC2386E7003147A386E70017D765
:10800000FF1F130767722398E70017D7FF1F130797
:10801000A775239AE70017E7FF1F13072781239C03
:10802000E70029472381E70209472383E7022385E5
:10803000E702A3810700930600F8A380D700930608
:1080400090022380D700FD562383D7002381E700C9
:10805000B706400037E700E02320D71003C717001A
:1080600013671700A380E700B24097E7FF1F239F25
:10807000079041018280F1679387072017E7FF1F70
:108080002320F790854717E7FF1F231DF78EA14791
:1080900017E7FF1F2309F78E97E7FF1FA385078EBA
:1080A00097E7FF1F2382078E97D7FF1F238107665D
:1080B00097D7FF1FA38C0764814717D5FF1F1305B0
:1080C0002565FD5517D6FF1F130646652947B306DC
:1080D000F5002380B600B306F6002380060085076E
:1080E000E397E7FE97E7FF1F2388079A97E7FF1FAD
:1080F000A384079A97E7FF1F2381079A97E7FF1F3B
:10810000A38B078697E7FF1FA389078697E7FF1FC3
:108110002384078697E7FF1F238F078497E7FF1FB6
:10812000238E078497E7FF1FA388078497E7FF1F25
:108130002385078497E7FF1FA3810796828017E7AF
:10814000FF1F0347479685476316F7001703000094
:10815000670003E917030000670083DD411122C4B3
:1081600006C617E7FF1F0347079485472E8613F4BB
:10817000F50FAA856317F70417D5FF1F1305056FC1
:1081800097600100E780A02197D7FF1F2380077227
:10819000B787004023848702B7E600E03706400037
:1081A00023A0C6180100010003C7A7021377C70F59
:1081B0002385E702B240224423A0C61001454101B5
:1081C000828017D5FF1F1305255E97600100E780A9
:1081D000001D97D7FF1F23890760B78700402382C0
:1081E0008702B7E600E03706400023A0C61801006A
:1081F000010003C767021377C70F2383E7025DBF40
:10820000411106C697000000E78020E7B240410117
:10821000170300006700E3F2411106C697F0FFFF65
:10822000E780E0BD97D7FF1F83C7175C95C797D539
:10823000FF1F83C5855B89C917D5FF1F1305055B24
:1082400097F0FFFFE780409C97D7FF1FA38E07584A
:1082500097D7FF1F238A0772B2404101828041C92C
:10826000D9C597D7FF1F83C76772D1C3011122CC2D
:108270004AC84EC656C25AC006CE26CA52C42E8915
:10828000AA890144930A0004371B0300637724037F
:10829000B3078940C207C183BE8463F4FA00930424
:1082A0000004C204C180130A1BD497D7FF1F83C7E1
:1082B000A7539DE37D1A631C0A00F2406244D24436
:1082C0004249B249224A924A024B0561828097F0A4
:1082D000FFFFE780C0B2D1BF338589002694A68511
:1082E000420497000000E780A0E7418045B7828004
:1082F00097D7FF1F9387C77E18429C4383D64500BC
:108300000345070083C5C700035646006396A500D2
:1083100083D5E700638DD502011106CE2386A70021
:108320002397D700B705CF00DC4B9385757D0507F4
:108330007D162EC2230001003AC42316C100231764
:10834000D10099C30A858297F240056182808280BC
:10835000DC4DDC4B81CFB7E70400904503A38705D4
:10836000914517D5FF1F0345E577028382806D7124
:108370003C083EC6B707E500232291103EC8AA84F8
:108380003C083285232611103ECA23248110232065
:1083900021112E8997300000E78020562A84979576
:1083A00001009385A5C317850100130525B89760C3
:1083B0000100E780200AA28517950100130585D2E8
:1083C00097600100E7800009294597600100E78078
:1083D000400DB705CB009385757D680097100000B0
:1083E000E780405FA285680097300000E780404347
:1083F000014781467000CA85268597200000E780E6
:10840000C08205CD2A8497950100938525BD1785E7
:1084100001001305A5B197600100E780A003A285C4
:10842000179501001305C5CC97600100E780800215
:10843000294597600100E780C0068320C11003240E
:10844000811083244110032901105161828097D744
:10845000FF1F9387E76818429C43797122D406D6A0
:108460000348070083C807012A8483D645000355C3
:1084700046006396080183D82701638DD8022388BC
:10848000070105072399D7003708CC00DC4B1308F8
:10849000787D3ACC1307F5FF42CA23080100231E5A
:1084A000E100231FD10099C7080832C62EC4829765
:1084B0003246A245228597000000E78080EBB2504B
:1084C0002254456182806D713C083EC0B707E500CB
:1084D0003EC23C083EC423261110232481102322CF
:1084E0009110231701002318010023190100231AFA
:1084F0000100231B010097B7FF1F83D7A7EC99E367
:10850000C167FD172316F10097B7FF1F83D7A7EBAD
:1085100091EB97D7FF1F9387A75C9C439C43DC4755
:1085200083D7070017B4FF1F1304C4E9584C23175F
:10853000F10083574400484B2318F10031E197952F
:1085400001009385A5B0178501001305259E97604E
:108550000100E78020F017950100130565B09760D2
:108560000100E78020EF294597600100E78060F374
:108570008320C11003248110832441105161828023
:1085800097B7FF1F83C777E489EBB7E70400BC57B1
:1085900082975C4C23AA0700E1BFFD1797B6FF1F27
:1085A000A385F6E203560701834704014C470A8579
:1085B000230BF10097300000E780A02397D7FF1F1F
:1085C000938707529C430147814688430A866C0083
:1085D00097100000E7806065AA8429C19795010083
:1085E0009385C5A617850100130545949760010082
:1085F000E78040E6A68517950100130525A797603B
:108600000100E78020E5294597600100E78060E9E7
:10861000584CB7E70400BC57484B9DBF97B7FF1FA6
:1086200083C7B7DAF5D7B7E70400BC4F10448545D8
:1086300017D5FF1F0345054B82971DBF5C4EDC4BD2
:10864000B9CFB1CD411122C4178501001305058EA4
:108650002E84979501009385A59D06C6976001001D
:10866000E78040DFA285179501001305E5A297601A
:108670000100E78020DE294597600100E78060E285
:10868000B7E704002244B24003A3870517D5FF1FB4
:10869000034545451306400691454101028382800A
:1086A000411122C417B4FF1F130484CF1C4C06C60B
:1086B00089C7DC4399C34C488297584CB7E70400FC
:1086C000BC57484B82975C4CB240224423AA070017
:1086D0004101828017B7FF1F130787CE834707002A
:1086E0009306F00B850793F7F70F63E9F60097B64B
:1086F000FF1F2387F6CC034507008280930700F80D
:10870000FDB7835745006386071001114AC817B9A2
:10871000FF1F130929CB52C4032AC90106CE22CC5C
:1087200003274A0126CA4EC656C2F15735E313073E
:10873000D00DFD57636EC704B7E9040083A709078E
:108740002A841305860042054181B284AE8A82974D
:10875000232AAA000325C9015C49A9E797950100CE
:108760009385058B177501001305457C9760010003
:10877000E78040CE179501001305459A97600100E8
:10878000E78040CD294597600100E78080D1DD5723
:10879000F2406244D2444249B249224A924A3E855A
:1087A0000561828093874400B705CF002319F50047
:1087B0009385757D310597100000E780A021032582
:1087C000C90183456400310597300000E78040050A
:1087D0000325C9012686D685310597300000E7803C
:1087E00040017146A2854A8597600100E78020BB61
:1087F000504419CA83A78905854517D5FF1F03452E
:10880000652E8297814769B797000000E780E0CB2B
:10881000D5BFFD573E858280411126C297B4FF1F08
:10882000938444BAD84C22C437E404003C54484BE7
:1088300006C68297DC4C0323C4052244B24092440E
:1088400023AA070017D5FF1F0345C5298545410108
:108850000283411126C297D4FF1F938464289C4051
:1088600006C622C44AC0D5C3DC43C5C35CC12300CD
:10887000B5002A84978501009385C574177501009A
:108880001305C56A97600100E780C0BC2945976061
:108890000100E78000C19C4023A4070023A2070039
:1088A00097B7FF1F9387C7AFDC4FDC4B91C72955A4
:1088B00097000000E78000DF97B7FF1F938787B01E
:1088C000DC4FDC4B89C797000000E78020F537E9D3
:1088D00004008327C905894517D5FF1F0345852057
:1088E00082978327C905914517D5FF1F0345851F2B
:1088F00082979C4003A34701630903002285224419
:10890000B2409244024941010283B240224492445F
:108910000249410182800111328506CE22CC26CA4D
:108920002E8497300000E78040FDAA8497850100DF
:108930009385856C177501001305455F97600100ED
:10894000E78040B103078400035664008355440068
:10895000A686178501001305257697600100E7803C
:1089600060AF294597600100E780A0B397B7FF1F6C
:1089700083C767A3639D9700014597000000E780C8
:1089800060D281450A8597000000E780C0ECF24084
:108990006244D244056182806D71232481102326B4
:1089A00011102322911093F745002E84638707143A
:1089B0003C083EC0B707E5003EC23C083EC4231752
:1089C00001002318010023190100231A0100231BB1
:1089D000010097B7FF1F83D7A79C99E3C167FD17D5
:1089E0002316F10097B7FF1F83D7A79B91EB97D76B
:1089F000FF1F9387E70E9C439C43DC4783D7070008
:108A000017B7FF1F1307C7992317F100544F835758
:108A100047002318F100DC4AA1E797850100938500
:108A2000E561177501001305655097600100E78047
:108A300060A2178501001305A56297600100E78019
:108A400060A1294597600100E780A0A51345440077
:108A50008320C1100324811083244110516182803E
:108A600097B7FF1F83C737942555D9C3FD1717B68E
:108A7000FF1FA30AF69203D6060183470701CC46DF
:108A80000A85230BF10097300000E78080D697D746
:108A9000FF1F9387E7049C4317B7FF1F13074790F7
:108AA000978601009386C65E88430A866C009710FD
:108AB0000000E7808017AA8451D99785010093852B
:108AC000E557177501001305654697600100E780BB
:108AD0006098A68517850100130545599760010028
:108AE000E7804097294597600100E780809B2685B5
:108AF00097000000E78000BB91BF93F725009DC75A
:108B0000B7E70400BC4741468145280882972555B0
:108B100097000000E78000B928089305F00F970040
:108B20000000E78040D3134524001DB793F71500DC
:108B3000014599DF97000000E78020991345140054
:108B400001BF5C4D411106C688C317D7FF1F2329FB
:108B5000F7F8B7E7040083A7070817050000130517
:108B6000E5E38297B24097D7FF1F238DA7F6014513
:108B70004101828001113335A000A307A100B7E7AE
:108B8000040083A7471706CE1306F1008545130599
:108B900050308297F240056182808280411122C468
:108BA00006C697D7FF1F83C767F5014489EF97B7BC
:108BB000FF1F83C73763054499E717D4FF1F03449A
:108BC000A4A213441400228597000000E780C0FA95
:108BD000178501001305456009E417850100130599
:108BE000A5602244B24041011763010067008386FB
:108BF000797122D4A30F010037E40400832784177E
:108C000026D24AD006D6AA842E8913055030930561
:108C1000F10132C6829732468347F101931506016E
:108C2000C18185CB01452EC697000000E780C0F4C6
:108C300083274417B2454A862685829705459700C3
:108C40000000E78060F3B25022549254025945610B
:108C50008280832744174A8626858297EDB7411183
:108C60009397050122C406C626C2C1872E8463D409
:108C70000702B7E40400FC5417A5FF1F03458577DE
:108C8000829719C1BC5482972165218DB24022443C
:108C900092444101828093F715008DC7B7E7040025
:108CA00083A7471A17A6FF1F1306C67397D5FF1F82
:108CB000938505E417A5FF1F0345C57382971345E8
:108CC0001400E9B793F7250099CFB7E70400BC4F2C
:108CD00013060064894517A5FF1F0345A5718297F8
:108CE0001345240065B793F785009DC7B7E70400D7
:108CF00003A8871A1307401F97A7FF1F83C7876F13
:108D0000814613064006994517D5FF1F035545DFD9
:108D10000298134584009DBF93F745000145BDD7D8
:108D2000B7E4040083A7041817D5FF1F035545DDDA
:108D30008297BC4C13060064914517A5FF1F03459D
:108D4000656B82971345440091B797D7FF1F83D770
:108D500027DB6398A70217D7FF1F2314B7DA17D7AB
:108D6000FF1F2311C7DA17D7FF1F231ED7D82E8660
:108D7000178501001305854CBE8517530100670058
:108D8000636D178501001305E54C1763010067004B
:108D900043840357450097D7FF1F83D767D6631ACD
:108DA000F704C1674111F91722C417D7FF1F232900
:108DB000F7D437E4040097D7FF1F23A507D497D72C
:108DC000FF1FA38D07D27C4C06C6894517A5FF1F40
:108DD0000345456282977C4C914517A5FF1F0345CB
:108DE000656182972244B240410117030000670089
:108DF00023DB178501001305E545175301006700C4
:108E0000437D7D15954763E2A71C17870100130773
:108E1000673A0A053A951C41011122CC06CEBA9751
:108E20002E84828717850100130545439750010062
:108E3000E780207AA1A203C7250099476311F702B2
:108E40002E8597000000E78000F5834564001785B4
:108E500001001305A54197500100E780A05F97B777
:108E6000FF1F23810738178501001305E5417DBFEA
:108E700003C7250095476319F702C16717D7FF1F7E
:108E8000035707C8F91703D5A5006309F702B7E729
:108E9000040083A7C7178297178501001305C53FF4
:108EA00097500100E780E072854717B7FF1F230B3B
:108EB000F732178501001305A5408DBF97D7FF1F17
:108EC0002390A7C483D7E50097D6FF1F239BF6C244
:108ED00083D7050197D6FF1F2396F6C283D72501B6
:108EE00097D6FF1F2391F6C297D7FF1FA38807C00D
:108EF000631BE502B7E70400BC4F09661306069042
:108F0000A14517A5FF1F0345E54E82970356E400D0
:108F10008355A400178501001305453997500100BA
:108F2000E780405351B79307700F2316F100B7E75E
:108F3000040083A7870D17A6FF1F0346A64B6C00EE
:108F400082974DF9854717D7FF1FA309F7BA5DB779
:108F50001785010013058537D1BD83C525009147CD
:108F60006392F502178501001305C537975001007C
:108F7000E780206697000000E78080C2F2406244EC
:108F80000561828099476392F5022285970000006F
:108F9000E78060E083456400178501001305052D17
:108FA00097500100E780004BD1BF9547639AF500C9
:108FB00083471400E1F3178501001305E534BDB5BF
:108FC000178501001305C534E1BF82806D7123242C
:108FD00081102326111023229110328401CD89475C
:108FE000630AF5028320C1100324811083244110F9
:108FF000516182801785010013054532AE84975078
:109000000100E780005DA285268597C0FFFFE7800D
:109010000055C9BFB7E70400FC47280082971785B1
:1090200001001305653097500100E780805A83479F
:10903000810039C41307000B6380E7021387A7057B
:109040001377F70F8D4663EDE602A285280097D0CF
:10905000FFFFE780E0C379B78547E3F587F88345ED
:109060009100177501001305A521B335B00097B71E
:10907000FF1F238BB7FE97500100E780A03D9DB7EF
:1090800003479100A207D98F35671307D75563852A
:10909000E7086368F7022D671307B7556387E7068C
:1090A00031671307C755638AE70429671307A75574
:1090B0006394E702A285280097D0FFFFE78020F79E
:1090C00015B739679306E765638DD70663E9F60040
:1090D0001307E7556380E706A28528003DB73D6783
:1090E0009306F7556386D7061307F766E396E7FE00
:1090F00097D0FFFFE780A00FF5B50146A2852800B5
:1091000097D0FFFFE780E0DFF1BDA285280097D070
:10911000FFFFE78000F0F9B58947E3F587EC930599
:10912000E4FFC205C1811305A10097A0FFFFE780FE
:10913000E0074DBDA285280097D0FFFFE78020F013
:1091400055B5A285280097D0FFFFE780E0FA59BD0A
:1091500097D0FFFFE780600371B5411122C417A4C7
:10916000FF1F1304642AAA86178601001306060649
:109170002285C14506C697500100E780C0460357C7
:10918000440097A7FF1F938727292393E7000357DE
:1091900064002394E700B2402244410182804111DF
:1091A00006C697000000E78080FBB7E7040083A7AE
:1091B000871417A6FF1F13062625D545014582975C
:1091C000B2404D4697A5FF1F9385052513057030C6
:1091D0004101170300006700E3A161712324811A94
:1091E00037E40400832704082326111A2322911A46
:1091F0002320211B232E311917050000130565A616
:10920000829717A9FF1F1309E91E99478544230078
:10921000A900231CF10097850100938525FF930782
:10922000400617750100130565D0231CF1082308BB
:10923000910097C9FF1F9389894B97500100E780E0
:10924000602183D5090017850100130525FB975080
:109250000100E7802020294597500100E780602425
:1092600003D50900856997000000E78040EF832758
:1092700044171008854513055030829783274417FB
:1092800017A6FF1F13064619CD45130570308297A8
:109290008327441717A6FF1F13060616B5451305A7
:1092A00060308297832744173008894513051031B1
:1092B0008297832744173009894513052031829707
:1092C00083274415938509C80D4582978327441544
:1092D000938509C811458297A30591002306910043
:1092E0002308910002CD230C010083278416300946
:1092F0009145130570408297832784161306B100A9
:1093000085451305004082978327841670008545A4
:10931000130510408297832784163008854513056E
:1093200020408297832784161008854513055040F6
:109330008297832704157D558297832744137D5593
:1093400082977D5597A0FFFFE78000318327440C6B
:10935000829797A0FFFFE780400C8327841417A60D
:10936000FF1F1306660AD5450145829789471306F4
:10937000700F814528092306F1009790FFFFE780D1
:10938000C0D58D471306000881452808230CF10835
:109390009790FFFFE78060D49147230CF100977707
:1093A0000100938727AA984383C747003AC8230A36
:1093B000F10097D0FFFFE78040EA70008545054542
:1093C00097A0FFFFE780603030099305700F0945D3
:1093D00097A0FFFFE780602F3008930500080D4538
:1093E00097A0FFFFE780602E10089545114597A0D4
:1093F000FFFFE780802DC16717C7FF1F1307477066
:10940000F9171CC32322070017A5FF1F130545FEEC
:1094100097A0FFFFE780402A8327C41D17C5FF1FC1
:109420001305856C82973C48034509008545829762
:109430008320C11A0324811A8324411A0329011AA3
:109440008329C1195D618280C16717C8FF1F035856
:10945000286BF9176301F8083DCDB5CD011126CA77
:10946000B7E4040083A7841222CC2E862315B10012
:1094700006CE2A8401478146ED45428582972AC659
:1094800011ED17850100130565D997500100E7809C
:109490004014F2406244D24405618280FC44035689
:1094A000A100A28582972C0017C5FF1F03554565B3
:1094B00097A0FFFFE780002D69DD178501001305E8
:1094C00025D797500100E780C01083A7C412ED454F
:1094D000280082977DBF8280411106C61DC985473D
:1094E00017A7FF1FA30FF7F0354697A5FF1F93851A
:1094F000A5F01305603097A7FF1F238507F097F0AD
:10950000FFFFE780206FB240410117F3FFFF6700C4
:10951000236997A7FF1FA38607EEF9B7C16717C591
:10952000FF1F0355E55DF9176307F500B7E7040072
:1095300003A3C71702838280854717C7FF1F230F26
:10954000F75A014517F3FFFF670003631793FFFF07
:10955000E70203B42A8408452E89B28919C900C1DB
:10956000971500009385A586610597300100E78077
:10957000800181447D5A97100000E780E03963C77D
:10958000A404814497100000E780003A63C8A40453
:1095900097C7FF1F938747579C43DC47B307F940A2
:1095A00091872302F400638309048327C900B3076A
:1095B000F4409587A302F4001C4C89C79C4799C3CB
:1095C000228582971793FFFF6700C3AF5C44139710
:1095D00014008504BA972390470171BF1C48139764
:1095E00014008504BA972390070069BF8327890078
:1095F0000547B307F4409587A302F400835704009E
:10960000638EE7028DC309476384E7040D47E39542
:10961000E7FA978701009387E7231CCC978701001F
:109620009387472411A897870100938727EA1CCCCA
:1096300097870100938787EA5CC8BDBF97870100C1
:109640009387C7D51CCC97870100938727D6EDB7A2
:10965000978701009387C7241CCC978701009387C5
:109660002725D9BF95E51793FFFFE70203A400461E
:1096700018448347940075839D8B6317F7009710F8
:109680000000E78060B448C41793FFFF670023A47D
:1096900082801793FFFFE702A39F13893500C164FF
:1096A00042094111AA890144F11413590901054ADB
:1096B0002EC697100000E7802026B2456348A4001C
:1096C000014541011793FFFF6700C39F83A709006E
:1096D00013171400BA9783D707006388B700639401
:1096E000970063742A010504E1B70545D9BF1793B4
:1096F000FFFFE7020399AA892E89328BB6843A8A42
:10970000BE8A97A00000E78020FB71C926859720BC
:109710000000E78020098D4763E7A7007D55179378
:10972000FFFF6700839983DB440097100000E78008
:10973000A0242A8497100000E78040259307740036
:1097400031443305850263CDA70297100000E780FE
:10975000A02297100000E78020222A8497100000A2
:10976000E780C0229307740031443305850263C348
:10977000A70497100000E78020209307450029A840
:1097800097100000E7808020330585021307F0174B
:109790009307C017E35FA7FA2D55E3C277F9630477
:1097A0000B02D6865286A6854A8597200100E7805F
:1097B00020BAB5B797100000E780401D3305850239
:1097C0009307C5FFD1BF832749001385C90083D5FF
:1097D000270097000000E78000EC61F581B769552C
:1097E0003DBF97C7FF1F2393A73297C7FF1F9387DC
:1097F000A731904381470C463307F5004207418368
:109800006393B70082805446139847008507C29639
:109810002390E600D5B797C7FF1F9387E72E9C4399
:1098200003C58700828017C5FF1F0355252E828040
:109830001793FFFFE7026387C1671387D7FF630BA7
:10984000E502636AA700F1176300F502014517936B
:10985000FFFF6700C3871387E7FF6302E502FD1779
:109860001D8D13351500E5B797500000E780C02621
:109870007D15C5BF97500000E78040FBD5BF9750CE
:109880000000E78060F9EDB71793FFFFE702E3817F
:109890004111AA8401442EC697100000E780C00839
:1098A000B2456348A400014541011793FFFF6700DB
:1098B00003829C48131514003E9583570500E385E9
:1098C000B7FE0504C9BF03485500814693F7F60F5C
:1098D00063E5070181473E8582805845939756008E
:1098E000BA9703D727006316B70003D70700E3042E
:1098F000C7FE8506E1BF8346450001479377F70F12
:1099000063E4D700814711A81C45131657000507CB
:10991000B29703D60700E313B6FE3E858280178315
:10992000FFFFE702E37693170501C18797CAFF1F80
:10993000938A8A1D635BF00883A70A00C0479C478F
:1099400003570400198D420541816368F500014405
:1099500022851783FFFF6700E37612052A94CDBFA7
:10996000DC4713944900014A3E9483474400634115
:10997000FA02014A834754006349FA028509C20981
:1099800093D9090183A70A009847E3EBE9FCC1B723
:109990001C4413195A00A6853E994A859700000079
:1099A000E780C0EE05E1050AC9B75C4413195A0007
:1099B000A6853E994A8597000000E78020ED19E1D1
:1099C000050A4DBFE30C09FA61B7AA8481495DBF5E
:1099D0001783FFFFE702636D1C452A8481E7930725
:1099E000C5001CC51C44231204001CC09307F00FC3
:1099F00063EDB70093F5F50F228597200000E7800F
:109A000020E21783FFFF6700836C93940501C16711
:109A1000C18063F9F500A685228597200000E780C4
:109A200040E5C5B7C18193F5F50F22859720000069
:109A3000E78000DFA685228597200000E78040E0D0
:109A4000C9B797C7FF1F9387270C884382801C459F
:109A500099C797C7FF1F23A9A70A014582807D5593
:109A6000828097C7FF1F9387270A98438347450043
:109A7000484792073E9582801783FFFFE702E36223
:109A8000617100451C183EC6B70780013EC81C180E
:109A90003ECA8357440002CE02D002CC231EF100FE
:109AA000834784002A8902D22301F1023C083ED474
:109AB00002D697000000E78000FB835705002316BD
:109AC000F10297500000E78060C42307A1025C40C8
:109AD00003556400F18313F717008347F102520521
:109AE0005181F99BD98FA307F10297100100E780FC
:109AF000807539CDAA840355050097A00000E78042
:109B000080BC83D704002AD26800231CF10083D7CD
:109B10002400231DF1001C4803D647008C439720E6
:109B20000000E78000CD8347B400CA861786010095
:109B3000130646808117A305F4006C004810972097
:109B40000100E780E0805D611783FFFF6700235815
:109B50002155D5BF1C45B1CF03C5A7008946135772
:109B60006500630BD7028D46630ED70285466300FE
:109B7000D702130740063305E50203C7B700418B40
:109B800015CB83C7B700BD8B3355F5408280137565
:109B9000F5031307803EC5B709671375F50313076F
:109BA0000771D1BF372709001375F5031307077C29
:109BB000D9B7014582801783FFFFE702034F03A94E
:109BC0008500630C09048347B900AE8493F7070E40
:109BD00085C303459900930520030D810505B30551
:109BE000B5028844610597300100E780E0A935A0FF
:109BF0002E8597000000E78020F62A8419CD970073
:109C00000000E780605C8325C900B307B54063FAB4
:109C100087002E94B305A440E9F51783FFFF670082
:109C2000034B85457DBF1783FFFFE70203482A8466
:109C300003D50500011132C636C43AC22EC002CA8D
:109C400002CC02CE97A00000E780E0A782452ACA96
:109C500022852ECC97000000E780E0E00357050046
:109C6000231EE10097500000E78040AAA24632463A
:109C70009247230FA10036874C08B2862285014601
:109C800097000000E780E0A605611783FFFF6700EB
:109C900003441783FFFFE702434161711C183EC66E
:109CA000B70780013EC81C183ECA3C0800453ED498
:109CB000AA8402CC02CE02D002D202D697000000C3
:109CC000E78060DA8357050035592316F102975073
:109CD0000000E780A0A32307A10209C48357440022
:109CE00081EB21594A855D611783FFFF6700233EA1
:109CF000035564005205518197100100E780A0547C
:109D00002A8965D18347B40093F7070E99C71305D5
:109D1000840197300100E780609983574400231E37
:109D2000F100834784002301F1025C4003550900E0
:109D3000D98313F7070883471102231CA10093F767
:109D4000F707D98FA300F10283572900231DF100E3
:109D50005C40F18313F717008347F102F99BD98F19
:109D6000A307F10297A00000E780E0952AD235D939
:109D7000834794006800139757008347B400FD8B16
:109D8000D98FA305F4001C4803D647008C439720C5
:109D90000000E78000A6A687177701001307875900
:109DA000740005464C10268597000000E7806094FB
:109DB0002A890DD98347B400A685FD8BA305F4003D
:109DC00097000000E78060DF31BF1783FFFFE702E5
:109DD000C32D832485FE2A84411126859700000027
:109DE000E78080D7834734FF93F7070E8DCB2AC6D1
:109DF000268597000000E78060C809CD834734FFBF
:109E0000B245FD8BA309F4FE91C522859730010070
:109E1000E780808741011783FFFF6700432B7DD9CF
:109E20008327C4FF2685829775F5834734FF93F710
:109E3000070E91C7228597300100E7802087032510
:109E400084FE97000000E78000E5E9B71783FFFF75
:109E5000E702A3229C4141112A8903C707008947D1
:109E60002E84935667006380F6040D466388C6040B
:109E70009307F0076304F7022E8597200000E78020
:109E8000C0A7AA848149C16B130C490097C7FF1F63
:109E9000938787C79C43984763E4E904410117838C
:109EA000FFFF6700432103D745008547E3F8E7FE3E
:109EB0002E8597200000E780A0A9E1B703D74500D1
:109EC000E3FEE7FC2E8597200000E78000A3AA842C
:109ED000228597200000E78060A4C204C98C5DB78A
:109EE000DC470355A900139A49003E9A93170501D0
:109EF000C187635DF00083570A006397A70263E799
:109F000074038327CA00034D5A002DA0A16721675F
:109F1000A98F1307F7EFE374F7FE63970900970023
:109F20000000E780209161FD85098DB783278A00B5
:109F3000034D4A00835DA90003576900216A138B12
:109F4000C7003AC6814A33CA4D01631E5D0197C7F7
:109F5000FF1F9387E7BB9C43E1DBA28662868145B6
:109F600026858297D1B7A1679387F7EF930C4BFFB4
:109F700063F24703B2455A8597F0FFFFE780A0716F
:109F80000DC103278B00104709CE10436382C40222
:109F90003107D5BFEE85668597000000E780008F0A
:109FA00071F993861A0093FAF60F130B0B0271BF27
:109FB000835644005C43E3E9F6F622853AC69710DF
:109FC0000000E780807DA1679387D7042A8A035D1C
:109FD0004400324763E897008347D90093E707F8C6
:109FE000A306F9001C4766852286E2858297C16731
:109FF0000844FD17337AFA00529508C02312A401D1
:10A0000025B797C7FF1F938727B09843814715C38C
:10A010001447814763FFD500939745004C47BE9591
:10A0200019C903C7550081476375E600DC4516066C
:10A03000B2973E85828003C745008147E37BE6FEF9
:10A0400016069C45F5B71783FFFFE7026304AA894C
:10A050002E8A814497CAFF1F938A0AAB83A70A00FE
:10A06000984763E6E4001783FFFF6700A305DC471A
:10A070001394440001493E9413BB140083474400E9
:10A08000634BF900014913BB140083475400634F2D
:10A09000F9008504E1B70844931759005287DA861E
:10A0A0000146A2853E9582990509C9BF4844931788
:10A0B00059005287DA860546A2853E9582990509A0
:10A0C000E9B71783FFFFE70243FE814517F5FFFF5E
:10A0D0001305054897C7FF1F239A07A297000000A2
:10A0E000E780A0F61783FFFF670063FE97C7FF1F97
:10A0F000938787A19C4395C31783FFFFE702E3FA89
:10A10000814517F5FFFF1305A54497000000E78080
:10A11000C0F31783FFFF670083FB82801783FFFF75
:10A12000E70203F737E40400832784124111231563
:10A13000E100AE893289368A3A8681460147ED458B
:10A14000AA8482972AC621C90356A100D2859740C6
:10A150000100E780C0248327C413CE85268582971B
:10A16000058905C98327440D2314210101462C00CC
:10A17000268582972A8401C9B7E7040083A7C712FE
:10A18000ED4528008297228541011783FFFF670074
:10A1900063F34944D5B76554FDB75C41FD175CC115
:10A1A00082801783FFFFE70243F0B7E70400FC5FFC
:10A1B000829795473305F50281450D811783FFFF8F
:10A1C0006700E3F01783FFFFE70223EEB7E7040021
:10A1D000FC5F829795473305F5020D811783FFFFDA
:10A1E0006700E3EE1783FFFFE70223ECB7E7040005
:10A1F00083A7870B0355050082971783FFFF67002E
:10A2000003ED1783FFFFE70243EA0355050032879A
:10A21000AE861796FF1F0356462697C5FF1F9385E8
:10A22000658F97000000E780A0EF1783FFFF6700AE
:10A2300003EA1783FFFFE70243E7B7E7040083A7BA
:10A24000C71782971783FFFF670063E81783FFFF35
:10A25000E702A3E5B7E7040083A7871397C5FF1FAD
:10A260009385458B829701451783FFFF670023E69F
:10A270001783FFFFE70263E3B7E7040083A7C71F65
:10A2800081451795FF1F0355451B82971783FFFFD5
:10A290006700E3E31783FFFFE70223E1B7E704006A
:10A2A00083A7871397C5FF1F9385C58782970145AD
:10A2B0001783FFFF6700A3E11783FFFFE702E3DED9
:10A2C000B7E7040083A7C71F81451795FF1F0355F4
:10A2D000C51C82971783FFFF670063DF1783FFFFAB
:10A2E000E702A3DC2E8597800000E780E0AF97802F
:10A2F0000000E780E0EC1783FFFF670043DD178372
:10A30000FFFFE70283DA97800000E780E0F617831B
:10A31000FFFF6700C3DB5C49E1175CC95CC583577D
:10A320002501A1072319F50083570501A10723186B
:10A33000F5008280F1473305F50297C7FF1F938729
:10A3400067809C433E9582808D476315F60803D74E
:10A350004600854763F0E7081783FFFFE702E3D471
:10A36000368536842E8997100000E780005929C968
:10A370008357440093140501C18063E39704228549
:10A3800097100000E7806057FD1423129400930794
:10A39000A0026300F5029307B0026307F50293077A
:10A3A0009002631FF500228597000100E780C085B9
:10A3B00001A80146CA85228597A00000E78060B009
:10A3C0001783FFFF6700A3D0228597100000E78066
:10A3D000C003FDB7828097B6FF1F9386E6769C4246
:10A3E000014599CF9843D44217B6FF1F232EE67438
:10A3F0006396D70097B6FF1F23AAE6741385C7FE9E
:10A4000082801783FFFFE70243CA97000000E780BE
:10A41000A04B714433058502914597900000E78079
:10A4200020E911E565551783FFFF670043CA97B719
:10A43000FF1F23A7A77097000000E780E0483305BF
:10A440008502914597900000E78080E661DD97B72F
:10A45000FF1F23A9A76E97000000E780E04697B78B
:10A46000FF1F2399A76C97000000E780E04597B78E
:10A47000FF1F2392A76C977701009387E7F017B728
:10A48000FF1F232DF76A97070000938707E917B787
:10A49000FF1F2323F76A014579B71783FFFFE70200
:10A4A000C3C0AA8517B5FF1F1305C5689710000024
:10A4B000E780C05B1783FFFF670063C11783FFFF5F
:10A4C000E702A3BE97000000E78060FD9710000040
:10A4D000E780405B97B7FF1F938707679C4391CF47
:10A4E0001387C7FE19CB83D5C7FF17B5FF1F130509
:10A4F000256697200100E78020191783FFFF67007A
:10A5000003BD1783FFFFE70243BA97000000E7800F
:10A51000C0EC09CD834785002A8493F7070499EBA3
:10A520000355E50097000000E78080F91783FFFFDF
:10A530006700E3B98347C5009304450117B9FF1FBE
:10A540001309896085E3832709005CC997B7FF1F5A
:10A5500023AC975E83274900F1FB97B7FF1F23A722
:10A56000975EE9B7FD172306F500610597800000A7
:10A57000E780C0D68307840063CB07048347840049
:10A5800093E707F82304F400B7E704009C5F829781
:10A590004205A94741813375F5028347840093F74B
:10A5A00007FCC98F2304F4008347D4003E951C4068
:10A5B0002318A40089CF984319CB8347C400504087
:10A5C000814585073305F5024205418102978327BE
:10A5D00009005CC897B7FF1F23A897568327490037
:10A5E00089E797B7FF1F23A397568347C4009DDFD2
:10A5F0008355040117B5FF1F1305855597200100EA
:10A60000E780800825B71783FFFFE70203AA97B703
:10A61000FF1F938727799C4701448583858B85E3BA
:10A62000AE84B2853A8697100000E780804B2A847A
:10A6300019C597100000E780C041829408CC22859C
:10A640001783FFFF6700A3A81783FFFFE70243A458
:10A6500041112E8932C6AA8997000000E780C031D7
:10A66000324713060502CA86970500009385C5CCBC
:10A6700017B5FF1F1305054C97000000E780E0F8B1
:10A680002A8425C99304C50097000000E780E041B3
:10A690001946AA85268597100000E7808015854514
:10A6A000268597100000E7806011177501001305DB
:10A6B00065CB4E9583450500268597100000E78001
:10A6C00020165C4831468145A1075CC85CC48357AD
:10A6D0002401E1172319F40083570401E11723181B
:10A6E000F4001C4C3E859780FFFFE780009FA30489
:10A6F0002501228541011783FFFF6700A39C178373
:10A70000FFFFE702839A4111AA842EC632C4971034
:10A710000000E7806036004DB24522468347840042
:10A720000CC050C093F7F70393E707042304F40029
:10A7300023180400268597100000E78080318347A6
:10A740009400A9462317A40013D737000507330741
:10A75000D7029D8B85072306F400A306E40083C778
:10A760000401D8488507230FF7FE17B7FF1F13070B
:10A77000A73D5843232A04009307440129E317B750
:10A78000FF1F2325F73C17B7FF1F232FF73A17B4F6
:10A79000FF1F1304E43B228597200100E78000E1BE
:10A7A0001C44858B5D8D19E581452285972001002C
:10A7B000E78080ED41011783FFFF670043911CC3D1
:10A7C00017B7FF1F2324F738D9B71783FFFFE70216
:10A7D000C38D97050000938565B70145970000007C
:10A7E000E78000B001451783FFFF6700438E1783A2
:10A7F000FFFFE702838B97000000E78080B017839C
:10A80000FFFF6700C38C8347C500A5E31783FFFFE5
:10A81000E702A3892A840355E50097000000E7803A
:10A8200000C821C18347840093F7F7FB2304F40099
:10A830001C4091C7DC4381C74C400145829797007B
:10A840000000E78080B917B5FF1F1305653097201A
:10A850000100E780A0E50355E40097000000E780D1
:10A8600020C61783FFFF6700838682801783FFFF60
:10A87000E702A38397B7FF1F9387072D9705000073
:10A88000938565C817B5FF1F1305852C23A0070006
:10A8900023A2070097200100E780E0CE1783FFFF87
:10A8A0006700E3821C4D91CFDC4381CF1773FFFF1C
:10A8B000E702A37F8345070082971783FFFF6700A6
:10A8C0000381828097B7FF1F9387C72A9C4303C5E4
:10A8D0000700828097B7FF1F9387C7299C4303C552
:10A8E0001700828097B7FF1F9387C7289C4303C533
:10A8F0002700828097B7FF1F9387C7279C4303C514
:10A900004700828097B7FF1F9387C7269C4303C5E4
:10A910003700828097B7FF1F9387C7259C4303C5E5
:10A920005700828097B7FF1F9387C7249C4303C5B6
:10A930006700828097B7FF1F9387C7239C4303C597
:10A940007700828097B7FF1F9387C7229C4303C578
:10A950008700828097B7FF1F9387C7219C4303C559
:10A960009700828097B7FF1F9387C7209C4303C53A
:10A97000A700828097B7FF1F9387C71F9C4303C51B
:10A98000B70011E11D45828097B7FF1F9387871E8F
:10A990009C4303C5C700828097B7FF1F9387871D1D
:10A9A0009C4303C5D700828097B7FF1F9387871CFE
:10A9B0009C4303C5E700828097B7FF1F9387871BDF
:10A9C0009C4303D50701828097B7FF1F9387871A9F
:10A9D0009C4303C52701828097B7FF1F9387871980
:10A9E0009C4303D54701828097B7FF1F9387871841
:10A9F0009C4303D56701828097B7FF1F9387871712
:10AA00009C4303D58701828097B7FF1F93878716E2
:10AA10009C4303C5A701828097B7FF1F93878715C3
:10AA20009C4303C5B701828097B7FF1F93878714A4
:10AA30009C4303C5C701828097B7FF1F9387871385
:10AA40009C4303C5D701828097B7FF1F9387871266
:10AA50009C438857828097B7FF1F9387A7119C4319
:10AA600003D5C702828097B7FF1F9387A7109C4327
:10AA700003D5E70219E11305800C828097B7FF1F09
:10AA80009387470F9C4303C50703828097B7FF1F37
:10AA90009387470E9C43C85B828097B7FF1F9387BD
:10AAA000E70C8843828097B7FF1F9387670C884322
:10AAB000828019E17D558280F5DE984265DFFDD9FF
:10AAC00017B7FF1F1307072E1847AA877155058B65
:10AAD000631D072403C507001547E37DA7FC03C7D3
:10AAE00037001305F0057D171377F70FE364E5FCD6
:10AAF00003C35700E30003FC83C86700E38C08FA34
:10AB000003C77700494579171377F70FE364E5FA30
:10AB100003C7A70011481305F7FF1375F50FE36B83
:10AB2000A8F803CE97000D481305FEFF1375F50F27
:10AB3000E362A8F803C8B700630908006518137832
:10AB4000F80F1305600DE36705F703C5C7007948E3
:10AB500079151375F50FE36FA8F403C8D7000D45F9
:10AB60007D181378F80FE36705F503D80701930EF6
:10AB700040175118420813580801E3ED0EF303C8BB
:10AB8000E7007D181378F80FE36605F303C8270183
:10AB90007D181378F80FE36F05F103C88700C54EE1
:10ABA00075181378F80FE3E70EF103D86701856E87
:10ABB000938EBEE06D18420813580801E3EC0EEFC7
:10ABC00003D847016D18420813580801E3E40EEF5B
:10ABD00003D887017918420813580801E36C05ED82
:10ABE00003C8A7017D181378F80FE36505ED03C5C9
:10ABF000B7011D487D151375F50FE36DA8EA03C570
:10AC0000D701714879151375F50FE365A8EA03D5E7
:10AC1000E7011308E00F7D1542054181E36CA8E8C8
:10AC200003C50702494879151375F50FE364A8E8D1
:10AC3000C85301C937C834005915130858BFE36B0E
:10AC4000A8E603A8870237C53400130555BF591875
:10AC5000E36205E717B5FF1F232CC5F003C6050106
:10AC600017B5FF1F2328F5F00545E375C5E403D8A4
:10AC70002501D04933760603E31E06E203C615011B
:10AC8000E30A06E217B6FF1F2322B6EE83C52700AC
:10AC900001466387A50003C61700F1453306B602D7
:10ACA00083C707039305C00272971A071307C705E6
:10ACB00016031A9796084697B387B70241553E97F1
:10ACC0003297420741836362E8061773FFFFE7028A
:10ACD000C33D368597800000E780A068970001009B
:10ACE000E78020482A8497A00000E780805A2A94B1
:10ACF00097F00000E78060262A9497900000E78094
:10AD0000A0812A9497F0FFFFE780E06F2A94974094
:10AD10000000E78060932A9497700000E780A09C71
:10AD200022951773FFFF6700833A82801773FFFF36
:10AD3000E702A3374111A307A10097A00000E78015
:10AD4000A0C59305F100170500001305E5B597F0C0
:10AD5000FFFFE780802F014541011773FFFF670068
:10AD600003371773FFFFE702C33117B4FF1F130444
:10AD700064030328840079599368180097B4FF1F6F
:10AD800023A614031378180063100802BA84BE893E
:10AD9000368B328A2E89AA8A97F0FFFFE780E0A7D8
:10ADA0007D15269519E531594A851773FFFF670010
:10ADB000C33097F0FFFFE78040A67D152695A16779
:10ADC000E353F5FE97B7FF1F9387C73498433E8C34
:10ADD000814B01CB014597F00000E7802044933B75
:10ADE00015004A85DA865686D28597900000E7805E
:10ADF000C04D2A8911CD1C44F99B17B7FF1F23278B
:10AE0000F7FA83270C00CDD3E3800BFA829769BF52
:10AE1000268597B7FF1F23A907F897F0FFFFE78064
:10AE2000809C4146CE8517B5FF1F1305250197303D
:10AE30000100E780C05697D00000E78040990325C5
:10AE4000040B97D00000E780009D054597D00000D7
:10AE5000E78000A4054597000000E78060EDA9B7F2
:10AE600097B7FF1F938707F49C47858BEDC7177330
:10AE7000FFFFE702832317B5FF1F130565FA97B796
:10AE8000FF1F23A107F297B7FF1F23AF07F097B764
:10AE9000FF1F23AD07F097200100E7802081975026
:10AEA0000000E780E0F597100100E780A04C9710C4
:10AEB0000100E780A05297B7FF1F938727ED9C43BF
:10AEC00091C7054597800000E780402097B7FF1F96
:10AED000938787D59C4399C741657D15977000007E
:10AEE000E78040A297F00000E780E03D97D00000A7
:10AEF000E780808F97B7FF1F9387C7FF9C43139707
:10AF000017016356070097F00000E78000AD97B780
:10AF1000FF1F23A507F297B7FF1F23A307F297B7D9
:10AF2000FF1F23A107F297B7FF1F23AF07F097007A
:10AF30000000E780008C97000000E780007297F027
:10AF4000FFFFE780401897F00000E78040D61773B6
:10AF5000FFFF6700C317828097B7FF1F938787E4BF
:10AF6000884382801773FFFFE70223149780000055
:10AF7000E780607597800000E780C0771773FFFF58
:10AF80006700E3141773FFFFE70283102A8493041A
:10AF9000140201112E85B289A685214636C63A894A
:10AFA00097300100E780403D0DE9B246380826861B
:10AFB000CE851305940497500000E7806041214638
:10AFC0002C084A8597300100E780003B13351500B7
:10AFD00005611773FFFF6700E30E0145D5BF1773C7
:10AFE000FFFFE702830C9305450617B5FF1F130506
:10AFF000A5B897100100E78020691773FFFF67006D
:10B00000030D1773FFFFE702430A41112EC697F0A5
:10B01000FFFFE780601BB24588C141011773FFFF46
:10B020006700E30A1773FFFFE7028306AA842E84F2
:10B0300097800000E780006CAA89854522859700EB
:10B040000000E780E07D83C7E4011389940899E359
:10B0500013890403CE85228597000000E780407C99
:10B06000214693051902228597000000E780607849
:10B0700097B7FF1F938707D38C4322859710000053
:10B08000E780C082214693858402228597000000D4
:10B09000E78020761773FFFF6700C3021773FFFF77
:10B0A000E70223FE397197F00000E780E0B49305D2
:10B0B000400661E997800000E780006063020514A4
:10B0C00097B7FF1F83C707AD13B7170097B6FF1FCA
:10B0D0002382E6AC014499CFC16417B9FF1F13095D
:10B0E00069CC9309400EFD1497000000E780C086EC
:10B0F0006342A40A97F0FFFFE780000D4169B7297A
:10B100000900096AFD7A2A8B81447D199389F97BAC
:10B11000130A0A71938A8AC797000000E780C083E8
:10B1200063D7A4041304400EB387840217B7FF1F2C
:10B13000130747C70324070B3E948357C401638258
:10B14000270B18403307EB4063EAE90083474400CC
:10B150008507B3874703D6976365F708014681459E
:10B16000094597F0FFFFE780604EAA8B29E59740DD
:10B170000000E780808385476317F506896593851E
:10B18000057117B5FF1F1305259F97100100E78074
:10B19000A04F95A0B30734030327090BBA9703D731
:10B1A000C7016308970003C75700A38207002382E3
:10B1B000E700050415BF9305C50022859700000030
:10B1C000E78080E65E852286976501009385C51A33
:10B1D00097F0FFFFE780E0525E8597100000E78060
:10B1E000608A850415BF97B7FF1F9387A7BB9C474D
:10B1F0008D83858BC1F721611773FFFF6700E3EB38
:10B2000001468545094502D002D202D402D697F004
:10B21000FFFFE780A043AA8479DD97F00000E78074
:10B22000E09C1389C4002A8481454A859700000068
:10B23000E780005F0C4041464A8597000000E780A8
:10B24000405B832944006385090C4E8502D802DAED
:10B2500002DC02DE97300100E78060402ACE141045
:10B2600005462C0808184ECC97500000E780E00AED
:10B270001375F50F51ED8355840093E525004A853C
:10B2800097000000E780E05E11460C104A859700A9
:10B290000000E78000560146976501009385450E42
:10B2A000268597F0FFFFE780C045268597000000C0
:10B2B000E780407D5C40A1D3014685450D4597F070
:10B2C000FFFFE780A038AA841DD548401389C40039
:10B2D00097300100E780A0382AC64A859700000011
:10B2E000E780404C3246636FC5004C404A8597006A
:10B2F0000000E780005001468145268597F0FFFF5A
:10B30000E7802040268597000000E780A077E5B51C
:10B3100083558400ADB71773FFFFE70203D997B7D2
:10B32000FF1F938727A89C471DC193E7870017B588
:10B33000FF1F1305658417B7FF1F2329F7A6971072
:10B340000100E78040321773FFFF670043D8DD9BA1
:10B3500017B7FF1F232CF7A497300000E780E064A5
:10B360007DF117B5FF1F1305258197100100E780B8
:10B37000E033D1BF1773FFFFE702A3D04169AA8969
:10B380002E8AB28A368BBA8B814417BCFF1F130CEE
:10B390006CA1930C400E7D1997F0FFFFE780C05B16
:10B3A00063C4A40001443DA03384940383270C0BA1
:10B3B0003E948357C401638627055A87D6865286F2
:10B3C000CE851305040397000000E780E0BB01C9A8
:10B3D00023800B0022851773FFFF670003CE83478E
:10B3E000F40185C35A87D6865286CE851305940804
:10B3F00097000000E78040B909C585472380FB001E
:10B40000D1BF850451BF835745006380071E177362
:10B41000FFFFE702E3C701112A8497000000E780DD
:10B42000C04D09C985476309F50605611773FFFF1C
:10B43000670043C997E00000E780007C7DF58357F3
:10B4400044004947ED9BE392E7FEC1452285970002
:10B450000000E7804033AA84228597000000E7803F
:10B46000204F0357440002CE91472A89631AF70000
:10B47000228597000000E780A0513C082ACC3ECEF0
:10B4800097E00000E78080765C55C5D374084A8653
:10B49000A6850545829751BF03574400D147E3F67F
:10B4A000E7F8032A0400C169014997BAFF1F938A8C
:10B4B0006A8F130B400EFD1997F0FFFFE780C0491C
:10B4C000634FA90E2285032A040097000000E7803D
:10B4D000C042A1452A89228597000000E780A02A62
:10B4E000AA84228597000000E780804A14402A86BB
:10B4F000AA8978082685CA8597000000E780C0E7FA
:10B50000AA8405D503C7F40189476315F70083476B
:10B51000C10181DF5546D285138564009730010053
:10B52000E780E0E7014597800000E780C01901C58A
:10B5300083D7C401A5E797B7FF1F9387A7869C47CA
:10B5400093551900858913D73700058B01CF89835F
:10B55000858B6399B70001452EC697000000E780F0
:10B56000C0DBB2454E8597800000E780601F034630
:10B57000C1012A8493751900268597900000E78001
:10B58000E03935C1268597800000E780E0182685E0
:10B5900011C0014597800000E780004C9730000003
:10B5A000E780A0408547E312F5E883C754001307FE
:10B5B000F00FE38CE7E68507A382F400BDB5B30482
:10B5C000690383A70A0BBE9483D7C401638B370139
:10B5D0005546D2851385640097300100E780C0D9B5
:10B5E00055DD0509D1BD5DD86DB782801773FFFFAA
:10B5F000E70203AA97800000E780000C05C1C16440
:10B60000014417A9FF1F1309E9799309400EFD149E
:10B6100097F0FFFFE7804034634EA40017A5FF1F9B
:10B620001305855597100100E780E0031773FFFFAE
:10B63000670043A9330534038327090B3E958357DD
:10B64000C501638897002312050097800000E780FA
:10B65000A00C050475BF97A7FF1F9387A7749C478D
:10B660008D83858B8DE31773FFFFE70203A417A576
:10B67000FF1F1305655097100100E7802003177323
:10B68000FFFF6700C3A482801773FFFFE702E3A1F7
:10B69000970500009385C5A017A5FF1F1305C54D8D
:10B6A00097100100E78020EE1773FFFF670023A2C9
:10B6B0001773FFFFE702639F8841B7E70400BC5B95
:10B6C000050542054181829709C585472300F5009C
:10B6D00005051773FFFF6700839F83C7F5FF2E855E
:10B6E0008507A38FF5FE828083C7F5FFFD1793F7CB
:10B6F000F70FA38FF5FE99EF1773FFFFE702E39AA9
:10B70000B7E70400BC571385F5FF82971773FFFF57
:10B710006700E39B82801C41035745008D8FBA95DB
:10B720001CC12312B5003E85828093D78500A205F7
:10B730001441DD8D835745001387E6FF18C1890743
:10B740002312F50013D685004111238FB6FEA38F77
:10B75000C6FE4101828018419307F7FF1CC1835741
:10B76000450085072312F500A30FB7FE828083579B
:10B7700045008D8F2312F5001C41BE950CC12E850E
:10B780008280AA8703D7470008410D8FAA9523928C
:10B79000E7008CC38280184108453305A7408280AA
:10B7A00083574500035765001D8F1C4108453385AD
:10B7B000A7403305A74082801773FFFFE702E38E9F
:10B7C00041112EC62A8497000000E780A0FDB245F3
:10B7D0006373B50001A0835744000840BE9523124F
:10B7E000B4003E9541011773FFFF6700438E177346
:10B7F000FFFFE702838B41112E84B28532C697008A
:10B800000000E780A0FB3246A28597300100E78068
:10B8100000B941011773FFFF6700638B1773FFFFC8
:10B82000E702A3882E84854597000000E78000F991
:10B83000230085001773FFFF670063891773FFFFFD
:10B84000E702A38641112317B10089459700000044
:10B85000E780C0F68347E1002300F5008347F1004D
:10B86000A300F50041011773FFFF670043861773BC
:10B87000FFFFE702838393D78500A2054111DD8D89
:10B880002317B100894597000000E78020F3834724
:10B89000E1002300F5008347F100A300F50041011A
:10B8A0001773FFFF6700A3821763FFFFE702E37FC1
:10B8B0001397850193D78501C166938606F0D98FCA
:10B8C00013D78500758FD98FA2053707FF00F98D33
:10B8D0004111DD8D2EC6914597000000E78000EEF6
:10B8E0006C00114697300100E78060AB410117639F
:10B8F000FFFF6700C37D1763FFFFE702037B1C4167
:10B90000854503C4070097000000E78080E6228594
:10B910001763FFFF6700A37B1763FFFFE702E3786E
:10B920001C414111894503C7070083C7170023073E
:10B93000E100A307F10097000000E78080E30355D2
:10B94000E10041011763FFFF670063781763FFFFA2
:10B95000E702A3751C414111894503C7070083C74E
:10B9600017002307E100A307F10097000000E7801C
:10B9700040E08357E100410113D58700A2075D8DA8
:10B98000420541811763FFFF670063741763FFFF80
:10B99000E702A3710C4141112A84114668009730D7
:10B9A0000100E780C09F9145228597000000E78055
:10B9B00040DCB247C166938606F01397870113D522
:10B9C0008701598D13D78700758F598DA2073707C7
:10B9D000FF00F98F5D8D41011763FFFF6700236F43
:10B9E0001C45BE950CC18280AE87944391E65841B8
:10B9F00001EF0CC15CC1828003C7570013671700B9
:10BA0000A382E700B687D5B70CC3EDB7AA87084174
:10BA100019CD1841D44398C36313D500D8C32A87DE
:10BA2000034657009376160081E6232007008280A4
:10BA3000944381CA8C4203A847008CC363930601D8
:10BA4000CCC3799A14C3A302C7003687D1BF1C4563
:10BA5000DC471D8DB777DBB6938777DB0985330528
:10BA6000F502420541818280F147B385F5024845E0
:10BA70002E9582808347450085072302F50082804A
:10BA80001763FFFFE70263622A8409E41763FFFF7D
:10BA90006700E36383474400F5DBFD1793F7F70F77
:10BAA0002302F400E5F71C4403D727000507239180
:10BAB000E700DC4399C3228582974C4889CD8347B0
:10BAC0005400898B99E71C4422859C479C439C47E2
:10BAD0008297232A04000040232004007DB71763C7
:10BAE000FFFFE702835C8357250041112EC681EBDF
:10BAF0000144228541011763FFFF6700435D03573F
:10BB000005008147F146E305F7FEB385D7024045BE
:10BB100085072E948345440008C4F5F5B247AA84EE
:10BB200081E7232A040009A81C456C0022859C4358
:10BB30009C43829748C84DDD85472312F400B247E5
:10BB400023200400231804002319F4005C485CC47B
:10BB500083D72400FD172391F40061BF1763FFFF13
:10BB6000E702A35497A7FF1F938707038843232661
:10BB7000050023240500410597100100E78000B36C
:10BB80001763FFFF6700A3541763FFFFE702E3514A
:10BB900017A4FF1F130444001C40411199CF9C4778
:10BBA0002300B5002AC65CC197000000E78040FB77
:10BBB0001C40DC4399C33245829741011763FFFF64
:10BBC0006700E3500347450029E3584DAA877D5598
:10BBD0001DCF1763FFFFE702434D1CC3DC4797A649
:10BBE000FF1F23ABE6FAF156130507012390D70098
:10BBF000970500009385050297100100E780A09843
:10BC000001451763FFFF6700834C7D55828082806A
:10BC10001763FFFFE7026349011161468145280070
:10BC20009760FFFFE780604B97A7FF1F9387C7F6DA
:10BC30009C4328009305F00FDC473EC697000000A8
:10BC4000E780C0F405611763FFFF6700434897A7CB
:10BC5000FF1F938767F49C43D847A1679387C70268
:10BC6000631EF70A397106DE22DC26DA80004AD824
:10BC70004ED652D456D23285B28497000000E78067
:10BC8000C0C7AA89268597000000E78020C923182D
:10BC9000A4FC268597000000E78040C82319A4FC77
:10BCA000268597000000E78060C783D744000A8A92
:10BCB000231AA4FC858393F7F70F230EF4FC860761
:10BCC000BD0793F7073F3301F1408A8A0149834753
:10BCD000C4FD6367F902CE85130584FC232C54FD53
:10BCE00097000000E78080EA5281130104FCF250C3
:10BCF0006254D2544259B259225A925A21618280D6
:10BD0000268597000000E78060C193171900D69739
:10BD100005092390A7001379F90F55BF828097A7D3
:10BD2000FF1F938767E79C43D847A1679387A702C4
:10BD3000631AF70A397106DE22DC26DA80004AD857
:10BD40004ED652D456D23285B28497000000E78096
:10BD5000C0BAAA89268597000000E78020BCFD575D
:10BD60002318A4FC26852319F4FC97000000E78023
:10BD7000E0BA83D744000A8A231AA4FC858393F788
:10BD8000F70F230EF4FC8607BD0793F7073F330137
:10BD9000F1408A8A01498347C4FD6367F902CE8571
:10BDA000130584FC232C54FD97000000E78000DE7F
:10BDB0005281130104FCF2506254D2544259B259D8
:10BDC000225A925A21618280268597000000E780DE
:10BDD000E0B493171900D69705092390A7001379AB
:10BDE000F90F55BF828097A7FF1F9387E7DA9C431F
:10BDF000D847A16789076310F70A397106DE22DC8C
:10BE000026DA80004AD84ED652D456D232853289AC
:10BE100097000000E78060AEAA894A85970000007D
:10BE2000E780C0AF835749000A8A2318A4FC8583A2
:10BE300093F7F70F230CF4FC8607BD0793F7073F32
:10BE40003301F1408A8A8144834784FD63E7F40229
:10BE5000CE85130584FC232A54FD97000000E7805B
:10BE6000E0D25281130104FCF2506254D254425980
:10BE7000B259225A925A216182804A859700000065
:10BE8000E780C0A993971400D69785042390A70054
:10BE900093F4F40F55BF828097A7FF1F9387C7CFF6
:10BEA0009C43D847A1679387E704631EF70A39715B
:10BEB00006DE22DC26DA80004AD84ED652D456D28C
:10BEC0003285B28497000000E78020A3AA892685E6
:10BED00097000000E78080A42318A4FC2685970023
:10BEE0000000E780A0A3231AA4FC26859700000089
:10BEF000E780C0A283D744000A8A2319A4FC858363
:10BF000093F7F70F230EF4FC8607BD0793F7073F5F
:10BF10003301F1408A8A01498347C4FD6367F9020E
:10BF2000CE85130584FC232C54FD97000000E78088
:10BF3000E0C55281130104FCF2506254D2544259BC
:10BF4000B259225A925A21618280268597000000B8
:10BF5000E780C09C93171900D69705092390A70086
:10BF60001379F90F55BF828097A7FF1F9387C7C228
:10BF70009C43D847A1679387C704631AF70A3971AE
:10BF800006DE22DC26DA80004AD84ED652D456D2BB
:10BF90003285B28497000000E7802096AA89268522
:10BFA00097000000E7808097FD572318A4FC2685A2
:10BFB000231AF4FC97000000E780409683D74400E2
:10BFC0000A8A2319A4FC858393F7F70F230EF4FC48
:10BFD0008607BD0793F7073F3301F1408A8A01497D
:10BFE0008347C4FD6367F902CE85130584FC232CC7
:10BFF00054FD97000000E78060B95281130104FCF2
:10C00000F2506254D2544259B259225A925A216182
:10C010008280268597000000E780409093171900E2
:10C02000D69705092390A7001379F90F55BF828091
:10C0300097A7FF1F938747B69C43D847A167DD07A3
:10C040006317F7041763FFFFE70223067971328550
:10C05000328497000000E780408A2AC62285970034
:10C060000000E780A08B2311A10222859700000029
:10C07000E780A088B2452300A102280897000000AD
:10C08000E780C0B045611763FFFF6700430482800B
:10C0900097A7FF1F938747B09C43D847A167938713
:10C0A00087046317F7041763FFFFE7020300797142
:10C0B0003285328497000000E78020842AC62285DA
:10C0C00097000000E78080852311A1022285970058
:10C0D0000000E7808082B2452300A1022808970073
:10C0E0000000E780A0AA45611763FFFF670023FEF9
:10C0F000828097A7FF1F938727AA9C43D847A167F1
:10C100009387A7046312F7021763FFFFE702E3F9BF
:10C1100001112800814597000000E78020A70561F4
:10C120001763FFFF6700A3FA828097A7FF1F93871B
:10C13000A7A69C43D847A167938757026319F702C4
:10C140001763FFFFE70263F60111328597F0FFFFE7
:10C15000E780A07A2308A10081452800970000000D
:10C16000E780C0A205611763FFFF670043F6828086
:10C1700097A7FF1F938747A29C43D847A167938740
:10C18000E702631BF7041763FFFFE70203F20111E5
:10C190003285328497F0FFFFE7804078AA842285B9
:10C1A00097F0FFFFE7808077854709E9228597F0C0
:10C1B000FFFFE78080744205B337A0002800814567
:10C1C000231891003ECA97000000E780209C05617B
:10C1D0001763FFFF6700A3EF828097A7FF1F938776
:10C1E000A79B9C43D84799476313F7081763FFFF42
:10C1F000E702A3EB79713285328497F0FFFFE78085
:10C20000C06F2AC6228597F0FFFFE78020712310B8
:10C21000A102228597F0FFFFE780206E2301A10293
:10C22000228597F0FFFFE780406DA301A1022285E0
:10C2300097F0FFFFE780606C2302A102228597F050
:10C24000FFFFE780806B2313A102228597F0FFFF99
:10C25000E780A06AB2452314A102280897000000D5
:10C26000E780C09245611763FFFF670043E6828065
:10C2700097A7FF1F938747929C43D847A16793874F
:10C28000C7036313F7081763FFFFE70203E279713F
:10C290003285328497F0FFFFE78020662AC6228528
:10C2A00097F0FFFFE78080672310A102228597F0B7
:10C2B000FFFFE780A0662311A102228597F0FFFF10
:10C2C000E780A0632302A102228597F0FFFFE780A9
:10C2D000C062A302A102228597F0FFFFE780E06120
:10C2E0002303A102228597F0FFFFE7800061B2459A
:10C2F000A303A102280897000000E7802089456178
:10C300001763FFFF6700A3DC82801763FFFFE7026C
:10C31000C3D901112A8497F0FFFFE780005EAA8449
:10C32000228597F0FFFFE780605F228597F0FFFF8F
:10C33000E780C05E035744008D4763F7E70022851E
:10C3400097F0FFFFE780805D228597F0FFFFE78091
:10C35000E05C2800A68597000000E7802083056147
:10C360001763FFFF6700A3D697A7FF1F9387C782B6
:10C370009C43D847A167FD07631FF7001763FFFFC2
:10C38000E702A3D2328597000000E78040F81763E8
:10C39000FFFF6700C3D382809797FF1F9387C77FF4
:10C3A0009C43D847A167E5076315F7081763FFFFAC
:10C3B000E702A3CF79713285328497F0FFFFE780DF
:10C3C000C0532AC6228597F0FFFFE78020552285BB
:10C3D00097F0FFFFE78080542310A102228597F099
:10C3E000FFFFE780A053520551812311A10222854E
:10C3F0002302010297F0FFFFE7802050A302A10271
:10C40000228597F0FFFFE780404F2303A10222859A
:10C4100097F0FFFFE780604EB245A303A102280812
:10C4200097F0FFFFE780807645611763FFFF6700A5
:10C4300003CA82809797FF1F938707769C43D8474C
:10C44000A1679387E703631FF7001763FFFFE70206
:10C45000C3C5328597000000E78060EB1763FFFFDC
:10C460006700E3C682809797FF1F9387E7729C431C
:10C47000D847A16793874704631EF7021763FFFF3E
:10C48000E702A3C279713285328497F0FFFFE7801B
:10C49000C0462AC6228597F0FFFFE7802048B245B4
:10C4A000280897F0FFFFE780606E45611763FFFF84
:10C4B0006700E3C182809797FF1F9387E76D9C43D6
:10C4C000D847A167938787026310F7041763FFFFBC
:10C4D000E702A3BD79713285328497F0FFFFE780D0
:10C4E000C0412AC6228597F0FFFFE7800041B24590
:10C4F0002300A102280897F0FFFFE780206945612B
:10C500001763FFFF6700A3BC82801763FFFFE7028A
:10C51000C3B9011197F0FFFFE780203EAA852800EC
:10C5200097F0FFFFE780806605611763FFFF6700F4
:10C5300003BA9797FF1F938727669C43D847A16745
:10C54000D107631FF7001763FFFFE70203B63285C9
:10C5500097000000E780A0FB1763FFFF670023B789
:10C5600082809797FF1F938727639C43D847A167D3
:10C57000C507631FF7001763FFFFE70203B33285A8
:10C5800097000000E780A0F81763FFFF670023B45F
:10C5900082809797FF1F938727609C43D847A167A6
:10C5A000B907631FF7001763FFFFE70203B0328587
:10C5B00097000000E780A0F51763FFFF670023B135
:10C5C00082809797FF1F9387275D9C43D847A16779
:10C5D000AD07631FF7001763FFFFE70203AD328566
:10C5E00097000000E780A0F21763FFFF670023AE0B
:10C5F00082809797FF1F9387275A9C43D847894784
:10C600006318F7021763FFFFE70223AA01113285BF
:10C6100032C897F0FFFFE780402EAA85280097F0E8
:10C62000FFFFE780A05605611763FFFF670023AA9D
:10C6300082809797FF1F938727569C43D847A1670F
:10C640008D076311F7041763FFFFE70203A60111CB
:10C650003285328497F0FFFFE780202A13066100BD
:10C66000AA844C00228597300000E780C023280070
:10C67000A68597F0FFFFE780605105611763FFFF14
:10C680006700E3A482809797FF1F938727519C43FD
:10C6900081CFDC4391CB1763FFFFE70203A18297B1
:10C6A0001763FFFF6700A3A282801763FFFFE70203
:10C6B000C39F79713C08AE843ED2A165B7070A00DA
:10C6C0002A843ED448103C08DD053ED636C432C626
:10C6D0003AC297D0FFFFE780E02F12474810BA8593
:10C6E00097F0FFFFE780C01332464810B28597F0FD
:10C6F000FFFFE780E014A2464810B68597F0FFFFE1
:10C70000E7800012501001478146A685228597D008
:10C71000FFFFE780805145611763FFFF6700239BA0
:10C720001763FFFFE702639801117C000329C5012D
:10C73000AE843ECAA165B70707002A843ECC4808EC
:10C740007C00C5053ECE97D0FFFFE780A02883453B
:10C75000D900480897F0FFFFE780800C5008014798
:10C760008146A685228597D0FFFFE780004C0561B2
:10C770001763FFFF6700A3951763FFFFE702E392CC
:10C7800083C7950093F7F707A384F500970000008F
:10C79000E78040F91763FFFF670063931763FFFFAC
:10C7A000E702A39079713C08AE843ED2A165B70739
:10C7B00009002A843ED448103C08938545043ED69F
:10C7C00032C636C497D0FFFFE780C020A24648108B
:10C7D000B68597F0FFFFE780A00432464810B28587
:10C7E00097F0FFFFE780C005501001478146A685FE
:10C7F000228597D0FFFFE780404345611763FFFF25
:10C800006700E38C1763FFFFE702238A83C7950065
:10C8100041112A8493F7F707A384F50032852EC6C9
:10C8200097F0FFFFE780800F85672AC46370F502E9
:10C8300097700000E78020E92246B24509ED1147D4
:10C840008146228597000000E78060E6410117637A
:10C85000FFFF6700C38701478346F501DDB7176314
:10C86000FFFFE702E38201113C003ECAB7070A005E
:10C870003ECC3C003ECE83C79500AA89328593F713
:10C88000F707A384F5002E8497F0FFFFE7800009E7
:10C890008567637DF504A165AA84938585044808AE
:10C8A00097D0FFFFE7800013268597700000E78090
:10C8B00080E12A8929E19145480897F0FFFFE78048
:10C8C00020F6A685480897F0FFFFE78060F7CA8545
:10C8D000480897F0FFFFE780A0F401478146500821
:10C8E000A2854E8597D0FFFFE7802034056117535E
:10C8F000FFFF6700237D8145480897F0FFFFE78031
:10C9000020F20349090275BF1753FFFFE70243787E
:10C9100079711C103ECAB7070F003ECC404D1C1069
:10C92000AA84AE894808994532C636893ECE97D04A
:10C93000FFFFE780200A32464808B28597F0FFFFE4
:10C94000E78000EE630C0902A545480897F0FFFF59
:10C95000E780C0E62546CA8597200100E78020A42D
:10C96000500801478146CE85268597D0FFFFE78096
:10C97000C02B45611753FFFF6700C3748355C40282
:10C98000480897F0FFFFE780A0EB0355E4028145DC
:10C9900005C5854785456301F502C167FD17930508
:10C9A000F00F630BF5007D1597700000E780208E77
:10C9B0009305150093F5F50F480897F0FFFFE78002
:10C9C00020E683450403480897F0FFFFE78040E531
:10C9D00083451403480897F0FFFFE78060E4835520
:10C9E0002403480897F0FFFFE78080E58355440360
:10C9F000480897F0FFFFE780A0E49DB71753FFFFBB
:10CA0000E702A36A83C795008146014693F7F707BB
:10CA1000A384F50097000000E78040EF1753FFFF65
:10CA20006700E36A1753FFFFE702236879713E84CA
:10CA30001C103ECA2E89B7070F00A1653ECCFD052C
:10CA40001C10AA84480842C03AC23ECE36C432C640
:10CA500097D0FFFFE78000F832464808B28597F08C
:10CA6000FFFFE780E0DBA2464808B68597F0FFFFAE
:10CA7000E78000DD12474808BA8597F0FFFFE7809E
:10CA800020DC0248630C08029145480897F0FFFF3C
:10CA9000E780C0D21146A28597200100E780209050
:10CAA000500801478146CA85268597D0FFFFE78059
:10CAB000C01745611753FFFF670063618945480848
:10CAC00097F0FFFFE78080CF834704002300F50045
:10CAD00083471400A300F500E1B71753FFFFE702F7
:10CAE000235B83C7950001112A8A93F7F707A38474
:10CAF000F5003285AE8432C697F0FFFFE78000E292
:10CB000032462A89328597F0FFFFE78000DF85678C
:10CB10006373F902AA894A8597700000E780A0BA7A
:10CB20002A8419ED114781464A86A68552859700C9
:10CB30000000E780C0B705611753FFFF6700835807
:10CB40009387E9FF93F7F70F0547E366F7FE8347FF
:10CB5000F50195EB8947E380F9FE8346F4015285A0
:10CB600001474A86A68597000000E78040B4A16788
:10CB7000D90748083ECC230A010002CE97000000E6
:10CB8000E780A0B04DBF639EE7008947639EF90030
:10CB900093071020231FF50097700000E780C0B7AF
:10CBA0006DBF0947E39BE7FA8D47E398F9FA2285C1
:10CBB00097700000E78080DF9797FF1F9387071D1E
:10CBC0009C4399E79797FF1F938707069C4399C754
:10CBD00003D5040097800000E780A0CE231F040047
:10CBE00022855DBF1753FFFFE702234C01113C0074
:10CBF0003ECAB7070B003ECC3C003ECE83C7950033
:10CC00002A89328593F7F707A384F500AE8497F05D
:10CC1000FFFFE780A0D093170501C187635AF00694
:10CC2000A1652A849385E502480897D0FFFFE78035
:10CC300060DAA285480897F0FFFFE78060C0979709
:10CC4000FF1F938767FE9C43A9EB01449375F40F84
:10CC5000480897F0FFFFE780A0BC9355844093F508
:10CC6000F50F480897F0FFFFE78080BB935504411C
:10CC700093F5F50F480897F0FFFFE78060BA01478A
:10CC800081465008A6854A8597D0FFFFE780E0F9E6
:10CC900005611753FFFF67008343416585460546DD
:10CCA000A2857D1597500000E78060BD59DD5105D4
:10CCB00097000100E780808F13044006334485020B
:10CCC00071B71753FFFFE702433E0111B707060094
:10CCD0003EC683C7950021642A8993F7F707A3848A
:10CCE000F500AE8428009305A4040AC40AC897D0AE
:10CCF000FFFFE78020CE300001478146A6854A85A8
:10CD000097D0FFFFE78060F297E0FFFFE780801594
:10CD100013049404480822CC230A010002CE970091
:10CD20000000E780809605611753FFFF6700233AF4
:10CD30001753FFFFE702C335C1642A89014497995D
:10CD4000FF1F93892906130A8002FD1497E0FFFF55
:10CD5000E78080C16347A40001451753FFFF6700C8
:10CD60006336B307440303A7C90ABA9703D707007A
:10CD70006306970083D72700638427010504F9B76A
:10CD80000545E1BF1753FFFFE70283302A8A2E894A
:10CD900099C123A0050081498144979AFF1F938A76
:10CDA0002AE0614B97E0FFFFE78040C263C7A40021
:10CDB0004E851753FFFF6700E3303384640383A776
:10CDC0000A003E948357040099E763040900232076
:10CDD00089008504C1BF4146D285130544009710E0
:10CDE0000100E780605975F5A289E5B71753FFFF89
:10CDF000E702032A39717C083ED4B7070A003ED601
:10CE00007C083ED883C795002A8A328593F7F707B6
:10CE1000A384F5002E8932C697F0FFFFE78000B0AB
:10CE200085676373F5083246AA84328597F0FFFF61
:10CE3000E780A0AC8547AA8963E8A706A16593852A
:10CE40008504281097D0FFFFE780C0B8268597702B
:10CE50000000E78040872A8429ED9145281097F04B
:10CE6000FFFFE780E09BA685281097F0FFFFE78093
:10CE7000209DCE85281097F0FFFFE780609A01473C
:10CE800081463010CA85528597D0FFFFE780E0D9F0
:10CE9000A1679387770448183EDC230A010202DE6B
:10CEA00097F0FFFFE780607E21611753FFFF670067
:10CEB00063218145281097F0FFFFE7806096A685E3
:10CEC000281097F0FFFFE780A0979797FF1F9387A1
:10CED00027249C4381CB22856389090097D00000D9
:10CEE000E78040248345040271B797D00000E780B3
:10CEF000C022CDBF1753FFFFE702831983C79500F8
:10CF00004111AA8993F7F707A384F5003285AE840F
:10CF1000328A97F0FFFFE78060A08567637FF502A4
:10CF20002A8997600000E780007A2A84914631C5FB
:10CF30008347F50105476387E70291C70D4763669D
:10CF4000F704AD461DA89305050303250A004146D5
:10CF500097100100E78040420DE941011753FFFFA0
:10CF6000670043169305950803250A00414697106C
:10CF70000100E7806040814669F54A86A6854E85B6
:10CF800097000000E780C081C9BF83250A00130510
:10CF9000940897700000E780A02919C1C146F1BF2D
:10CFA0009797FF1F938787DE9C4399E79797FF1F0B
:10CFB000938787C79C4399C7228597800000E780A5
:10CFC000208A69FD8547A30FF400228597B00000F1
:10CFD000E7806084228597600000E780E0734E85DB
:10CFE00081464A86A68597F0FFFFE780607BA167B0
:10CFF0009387570448003EC42302010002C697F0FD
:10D00000FFFFE780806891BF1753FFFFE7026307C8
:10D0100083C795004111AA8993F7F707A384F50008
:10D0200032852E89B28A97F0FFFFE780208F8567CF
:10D030006374F50EAA8497600000E780C0682A84B4
:10D040000DED416B014A979BFF1F938BABD5130CE2
:10D05000400E7D1B19A833048A0383A70B0B3E9453
:10D060008357C40163836705050A97E0FFFFE780E4
:10D07000A08EE342AAFE95460DA08357C501639694
:10D0800097029305050303A50A0041469710010086
:10D09000E780802E994611E181462686CA854E8515
:10D0A00097F0FFFFE780C06F85A883A50A001305EE
:10D0B000040397700000E780A017C14679FD228520
:10D0C000231E940097A00000E780E07422859760FB
:10D0D0000000E78060649797FF1F938767039C4376
:10D0E000A9C323000402228597D00000E78040F006
:10D0F0004E8581462686CA8597F0FFFFE780406A05
:10D10000A1679387070448003EC42302010002C6BA
:10D1100097F0FFFFE780605741011753FFFF67005B
:10D12000C3F989472300F402E1B7397106DE22DC36
:10D130004AD8800052D456D25AD026DA4ED65ECE85
:10D140002E8A32892A8B97D0FFFFE780E07D060583
:10D15000710541998A8A3301A140232224FC2314BA
:10D1600004FC97D0FFFFE780207C83479A000605E8
:10D17000350593F7F7072315A4FCA304FA004A85A5
:10D18000232624FC97E0FFFFE780407993170501F1
:10D19000C1876340F0025681130104FCF2506254CF
:10D1A000D2544259B259225A925A025BF24B21612F
:10D1B0008280AA844A8597E0FFFFE7802076AA89CB
:10D1C0004A8597E0FFFFE7806075A1659385C502FA
:10D1D0002A89130544FC97C0FFFFE780A07F2685BE
:10D1E00097C0FFFFE780E073854511C94A86CE8569
:10D1F00097C0FFFFE780606DAA8B21E98945130581
:10D2000044FC97E0FFFFE780A061A685130544FC7E
:10D2100097E0FFFFE780C062CE85130544FC97E0EE
:10D22000FFFFE780E061CA85130544FC97E0FFFF3C
:10D23000E780006101478146130644FCD2855A8588
:10D2400097D0FFFFE780609EB9B78145130544FC86
:10D2500097E0FFFFE780C05CA685130544FC97E0DC
:10D26000FFFFE780E05DCE85130544FC97E0FFFFFC
:10D27000E780005DCA85130544FC97E0FFFFE78067
:10D28000205C814497D0FFFFE780006AE3D4A4FAD2
:10D2900083A70B0113971400BA9783D5070099C58C
:10D2A000130544FC97E0FFFFE78080598504D9BF50
:10D2B000797106D622D44AD000184ECE52CC56CA26
:10D2C00026D25AC8AE893289AA8A97D0FFFFE78052
:10D2D000A0650605690541990A8A3301A140232A00
:10D2E00024FC231C04FC97D0FFFFE780E06383C786
:10D2F000990006052D0593F7F707231DA4FCA384C9
:10D30000F9004A85232E24FC97E0FFFFE7800061A7
:10D3100093170501C187634FF0005281130104FD8B
:10D32000B250225492540259F249624AD24A424BB4
:10D3300045618280AA844A8597E0FFFFE780005E0E
:10D34000A1659385A5022A89130544FD97C0FFFFB7
:10D35000E7804068268597C0FFFFE780805C8545B1
:10D3600009C9CA8597C0FFFFE78020592A8B29E1A8
:10D370008945130544FD97E0FFFFE780604AA685D5
:10D38000130544FD97E0FFFFE780804BCA85130536
:10D3900044FD97E0FFFFE780A04A0147814613065E
:10D3A00044FDCE85568597D0FFFFE7800088B5B74E
:10D3B0008145130544FD97E0FFFFE7806046A685A1
:10D3C000130544FD97E0FFFFE7808047CA851305FA
:10D3D00044FD97E0FFFFE780A046814497D0FFFF20
:10D3E000E7808054E3DBA4FA83270B011397140032
:10D3F000BA9783D5070099C5130544FD97E0FFFF51
:10D40000E78000448504D9BF1753FFFFE702E3C953
:10D4100083474500404DD5EFFD575DC483469400DA
:10D4200009476363D70A0346B400854663EEC6081E
:10D430008306E40063CA06085C45F9562390D700CA
:10D440009787FF1F83C7077699E3A304E4009787B4
:10D45000FF1F9387677D9C4381E78947A306F400FC
:10D460009797FF1F9387C7CA9C4381E78947230685
:10D47000F4009705000093854506AA84130504016E
:10D4800097F00000E7802010FD57231AF40281472F
:10D490001CDC01489787FF1F23A287709787FF1F17
:10D4A00093870770232E040304C0804397D0FFFFA7
:10D4B000E780C05161463306C502814522859750F9
:10D4C000FFFFE78080C181473E851753FFFF67005C
:10D4D00003C0FD57D5BF1753FFFFE70203BD2A84E2
:10D4E0000355450297600000E780E01D19E5231E03
:10D4F00004001753FFFF670083BD8357E401F5DB8A
:10D50000930504FF174501001305452197E000002E
:10D51000E780E014F9BF1753FFFFE70203B92E8934
:10D52000A16541119385E5032A8436C432C6BE84C1
:10D530003AC297C0FFFFE780E04912472285BA85CB
:10D5400097E0FFFFE780C02D32462285B28597E045
:10D55000FFFFE780E02EA2462285B68597E0FFFF19
:10D56000E780002E630309029145228597E0FFFFC3
:10D57000E780C0241146A68597100100E78020E2CD
:10D5800041011753FFFF670083B48945228597E067
:10D59000FFFFE780A02283C704002300F50083C7B4
:10D5A0001400A300F500E9BF1753FFFFE702E3AF44
:10D5B00083C79500444D054793F7F707A384F5000B
:10D5C0001C42411183C707006367F7062E842A892E
:10D5D000B1C003C7D400630FF7021787FF1F1307FB
:10D5E000A764184305C3A386F40097A00000E78052
:10D5F000404A83C7D40099E741657D1597400000F4
:10D60000E780403083D72403918B89C797E00000DF
:10D61000E780C0134A85A28597F0FFFFE78080105E
:10D62000A167C10748003EC42302010002C697F06B
:10D63000FFFFE780800541011753FFFF670023A923
:10D640001753FFFFE70263A603D745008D47AA845F
:10D6500041112E8432892E8563E3E70297E0FFFFB4
:10D66000E780C02BAA8523000900268597C0FFFF0D
:10D67000E780A02841011753FFFF670043A597E00B
:10D68000FFFFE780A0292AC6228597E0FFFFE780F9
:10D69000E028B24585472A862300F900268597C0F1
:10D6A000FFFFE7808022F9B7397106DE22DC26DA37
:10D6B00080004ED652D456D24AD85AD05ECEAE89C9
:10D6C000B284AA8A97D0FFFFE780002506051305DC
:10D6D000250241990A8A3301A140232224FC231404
:10D6E00004FC97D0FFFFE780202383C7990006053D
:10D6F0004D0593F7F7072315A4FCA384F9002685AD
:10D70000232624FC97E0FFFFE780402193170501C3
:10D71000C1876340F0025281130104FCF25062544D
:10D72000D2544259B259225A925A025BF24B2161A9
:10D730008280AA8B03AB040097C0FFFFE780601EC6
:10D7400051E583D7440001498544F11793B7170089
:10D75000A301F4FC834734FCA165C9C79385E504A4
:10D76000130544FC97C0FFFFE780C026A68513057C
:10D7700044FC97E0FFFFE780A00ADE85130544FC28
:10D7800097E0FFFFE780C00B834734FC114691E32D
:10D790000946DA85130544FC97E0FFFFE780600542
:10D7A0008144630A0900416B7D1B97D0FFFFE7802E
:10D7B000A01663CCA40201478146130644FCCE8523
:10D7C000568597C0FFFFE7804046B1B7A685130690
:10D7D00034FC97000000E780E0E6933415002A89C6
:10D7E00086048DBF9385C504A5BF8327C900139701
:10D7F0001400BA9783D5070063886501130544FCBC
:10D8000097E0FFFFE780C003850445B71753FFFF8C
:10D81000E702238779711C103EC4B7070F003EC68C
:10D820001C103EC883C79500AA8A328593F7F70774
:10D83000A384F500AE89328497E0FFFFE780000EF5
:10D8400093170501C187635AF0062A8A228597E05B
:10D85000FFFFE780A00C2A895285032B040097C0A4
:10D86000FFFFE780000C39ED8357440081440544F5
:10D87000F11793B71700A303F10083457100DA870E
:10D880002287CA865286280097000000E780E0C8F9
:10D89000014781463000CE85568597C0FFFFE7805F
:10D8A000C038A1679387D70348083ECC230A81007C
:10D8B00026CE97F0FFFFE78040DD45611743FFFF6D
:10D8C0006700A37FA2851306710097000000E78020
:10D8D00060D7AA84094455D13544E30055FB4A85F5
:10D8E00097F0FFFFE78000450D4441D9014497D0F0
:10D8F000FFFFE7806002634DA400C16B0144FD1B84
:10D9000097D0FFFFE7804001634EA4001544B5B7F0
:10D91000DC4413171400BA9783D7070063832703E7
:10D920000504F1B7D84493171400BA9703D707003A
:10D93000631B770123902701268597A00000E780CD
:10D9400080DB01441DBF050465BF1743FFFFE702ED
:10D95000237483C7950041112A8A93F7F707A3849C
:10D96000F50032852E89328497E0FFFFE78000FBC7
:10D9700093170501C1876353F006AA89228597E0B2
:10D98000FFFFE780A0F92311A1004E85832A040040
:10D9900097C0FFFFE780E0F839E5835744008544EE
:10D9A0000144F11793B71700A300F10003481100D9
:10D9B00003572100D6875285CE862686CA8597F0E2
:10D9C000FFFFE7806006A167F10748003EC423021D
:10D9D000910022C697F0FFFFE78020CB410117435B
:10D9E000FFFF6700236EA285130611009700000059
:10D9F000E78040C52A84894455D98357210011679F
:10DA00008544BA97C2071167C1831307F7EFE36F25
:10DA1000F7F89787FF1F938767379C4381CB85452E
:10DA20001305210097500000E780207583552100E1
:10DA30002285814497C0FFFFE78040E525D9231068
:10DA40000500228597A00000E78040CD85B71743E9
:10DA5000FFFFE702036383C7950041112A8B93F709
:10DA6000F707A384F50032852E8A328497E0FFFF02
:10DA7000E780C0EA93170501C1876351F006AA8ABF
:10DA8000228597E0FFFFE78060E92A895685832B8E
:10DA9000040097C0FFFFE780C0E831E583574400EA
:10DAA00081440544F11793B71700A301F10003481F
:10DAB0003100DE875A854A87D6862286D28597F03E
:10DAC000FFFFE78060F6A167ED0748003EC4230230
:10DAD000810026C697F0FFFFE78020BB4101174376
:10DAE000FFFF6700835DA2851306310097000000E9
:10DAF000E78040B5AA8409445DD99167CA97C207F7
:10DB00001167C1831307F7EF0544E362F7FACA858B
:10DB100097C0FFFFE78080D7014451F9814997D032
:10DB2000FFFFE78060E063DBA90098489397190046
:10DB3000BA9703D7070005EF2390270197D0FFFF7F
:10DB4000E78080DE1544E384A9F6268597A00000CF
:10DB5000E780C0BC9787FF1F938747239C430144FE
:10DB6000B9D74A8597500000E780C05889B7850922
:10DB70007DB71743FFFFE702A35179713E847C080C
:10DB80003EC82E8AB7071400A1653ECAE5057C0889
:10DB9000AA89080836C4428932C6BA8AC6843ECCED
:10DBA00097C0FFFFE78000E3CA85080897E0FFFF02
:10DBB000E78000C732460808B28597E0FFFFE7809C
:10DBC00020C8A246630A09049D45080897E0FFFFA4
:10DBD000E780C0BE1D4681459740FFFFE780E04FCC
:10DBE00063890A089145080897E0FFFFE78000BDB8
:10DBF0001146A68597000100E780607A100801476A
:10DC00008146D2854E8597C0FFFFE78000024561BF
:10DC10001743FFFF6700034BB685080897E0FFFF37
:10DC2000E78000C21C400808D8439355C701858986
:10DC300012075183B205D98D97E0FFFFE78040C0FE
:10DC40001C40080883C5870097E0FFFFE78040BDC0
:10DC50001C40080883C5A70097E0FFFFE78040BC91
:10DC60001C40080883C5970097E0FFFFE78040BB92
:10DC700085BF8945080897E0FFFFE78020B483C788
:10DC800004002300F50083C71400A300F500BDB70E
:10DC90001743FFFFE702C33F83C795004111AA89DD
:10DCA00093F7F707A384F5003285AE84328497E0BA
:10DCB000FFFFE780A0C693170501C187635DF004ED
:10DCC0002A89032A040097C0FFFFE78080C519E96D
:10DCD000835744000548F11793B71700A307F100D5
:10DCE000814631A81306F100A28597000000E78065
:10DCF00060951DC51C459DC783D647000148034755
:10DD0000F10093078500D2884A86A6854E85970044
:10DD10000000E78040E641011743FFFF6700833AB8
:10DD200009487DBF1D486DBF1743FFFFE70243361B
:10DD300065715C083EC4B7077B013EC65C083EC8FF
:10DD400083C795002A8A328593F7F707A384F500E5
:10DD5000AE8997E0FFFFE78040BA8357E100E1C753
:10DD60008945280097C0FFFFE780C0C6814528008D
:10DD700097E0FFFFE780C0AA97C0FFFFE780A0CC35
:10DD80009787FF1F9387C7389C431784FF1F03445F
:10DD900064E1AA843334800099C313642400978714
:10DDA000FF1F938767E89C4399C3136444009787D8
:10DDB000FF1F9387A7FD9C4399C31364840083D5F9
:10DDC00004002800014997E0FFFFE78060A783D5A2
:10DDD0002400280097E0FFFFE78080A683D5440059
:10DDE000280097E0FFFFE780A0A597D0FFFFE7801E
:10DDF000A0AE93150501C181280097E0FFFFE780E1
:10DE000020A4A285280097E0FFFFE78060A39C4440
:10DE10006360F902014781463000CE85528597C084
:10DE2000FFFFE78080E059611743FFFF6700832908
:10DE3000DC441314490028003E9497E0FFFFE7807C
:10DE40006096834744000347540089070607BA9742
:10DE50008607E36AF5FC835524002800814A97E091
:10DE6000FFFFE780E09D83454400280097E0FFFF27
:10DE7000E780009B83455400280097E0FFFFE78080
:10DE8000209A8347440063C9FA00814A83475400BB
:10DE900063C1FA020509A5BF1C4413975A00280064
:10DEA000BA9783D50700850A97E0FFFFE78040997E
:10DEB000C9BF032BC40093975A0028003E9B83558B
:10DEC0002B00850A97E0FFFFE780809783550B00C2
:10DED000280097E0FFFFE780A0964DBF1743FFFFA4
:10DEE000E702A31C5C4993E717005CC997A00000F8
:10DEF000E78020B61743FFFF6700631D1743FFFF4E
:10DF0000E702A31A2E84814597F0FFFFE780C0E760
:10DF100005C583570500FD172310F50009C4835775
:10DF200025002310F40097000000E78060FB014506
:10DF30001743FFFF6700A31931457DD82310040064
:10DF4000C5BF1743FFFFE702A31483C79500411124
:10DF50002A8A93F7F707A384F50032852E89328445
:10DF600097E0FFFFE780809B93170501C187635609
:10DF7000F006AA89C145228597E0FFFFE780A080CF
:10DF80002A8B4E85832A040097C0FFFFE7806099A3
:10DF900031E983574400231101000544F11793B779
:10DFA0001700A300F100814403481100035721002A
:10DFB000D6875285CE862286CA8597F0FFFFE780F6
:10DFC000A0A6A1679387170248003EC423028100E0
:10DFD00026C697E0FFFFE780406B41011743FFFF34
:10DFE0006700430E13061100A28597F0FFFFE7803C
:10DFF0006065AA8409E523110100094475B79305FA
:10E0000021005A8597000000E78080EF83572100A8
:10E010002A84D9DB9787FF1F938747D79C4381CBFF
:10E0200085451305210097500000E78000158355B2
:10E0300021002685314497C0FFFFE78020852DD53C
:10E0400023100500268597900000E780206D01448D
:10E05000A1BF1743FFFFE702430541112E896C0062
:10E06000AA8402C697F0FFFFE78000D20DC10357D4
:10E07000050005072310E50097000000E78040E653
:10E0800081473E8541011743FFFF67004304324744
:10E09000954765DBCA85268597300000E780400DEF
:10E0A000C147E34005FE3244854741462310F40052
:10E0B00083570900A685130544002311F400970037
:10E0C0000100E780C02D228545BF1743FFFFE7020F
:10E0D00023FC83C795004111AA8A93F7F707A3840D
:10E0E000F5003285AE89328497E0FFFFE780008338
:10E0F00093170501C1876356F0062A8AC145228518
:10E1000097D0FFFFE7802068AA845285032B040084
:10E1100097C0FFFFE780E08031E983574400231177
:10E1200001008544F11793B71700A300F1000144E3
:10E130000348110003572100DA875685D2862686C8
:10E14000CE8597F0FFFFE780208EA16793870702B7
:10E1500048003EC42302910022C697E0FFFFE780FB
:10E16000C05241011743FFFF6700C3F5A2851306A4
:10E17000110097F0FFFFE780E04C2A8409E52311A6
:10E180000100894475B7268593052100970000009A
:10E19000E78060ECAA8449FD83552100228597B071
:10E1A000FFFFE780A06E49F5014997C0FFFFE780B8
:10E1B000A077635DA900184893171900BA9703D791
:10E1C00007000DEF035721002390E70097C0FFFFE2
:10E1D000E7808075630625039787FF1F938707BB3A
:10E1E0009C4399C70355210097500000E78080F0B9
:10E1F000228597900000E78060521DBF050975B722
:10E2000095443DB705C19307F00F630FF500C5476F
:10E21000630CF5009307F5FF05453315F50042053E
:10E22000418182800145828041657D158280B9E906
:10E230001743FFFFE70263E70345060332849700B5
:10E240000000E78060FC9305803EB305B502C2057F
:10E25000C18181CD0357E402854763F8E7001305C8
:10E26000040197E00000E78020428357E402416701
:10E270007D176385E700FD172317F4021743FFFF9F
:10E280006700E3E482801743FFFFE70283DF004279
:10E2900083C79500444D0349140093F7F707A384FF
:10E2A000F50083470400220911673369F900A1676B
:10E2B000B347F90041112A8BAE8A63ECE70E83471E
:10E2C00024001307C00EB91793F7F70F6373F71005
:10E2D00003473400C14763EEE70E8347440013074A
:10E2E000E00793C707086371F70C834984008347ED
:10E2F0007400A209B3E9F900856763F7F90A034AD4
:10E300006400834754004E85220A336AFA0097500E
:10E310000000E780403B61C123962403834B340017
:10E32000137AFA00239A340323887403239944034D
:10E3300093890401631C090023A6040223980402A4
:10E340004E8597E00000E78060363DA00349240039
:10E350004A8597000000E78020EB2397A4028347BB
:10E3600044004E85A388F402E38D0BFCE30B09FC0B
:10E3700097E00000E780202F97900000E78000736F
:10E3800081460146D6855A8597E0FFFFE780005811
:10E39000A167938797033EC423020100480002C689
:10E3A00097E0FFFFE780602E41011743FFFF670002
:10E3B000C3D08544A2862686D6855A8597E0FFFF7E
:10E3C000E780C054A167938797033EC4230291005E
:10E3D000F1B7BD44C5B79144F1BF1743FFFFE70252
:10E3E00023CB01111C08404D3EC2B7070F003EC4AD
:10E3F0001C083EC62A89AE8997C0FFFFE780A0DAD5
:10E40000585C1C5C6346B70E6394E50063E2A70E9C
:10E410003385A740B3B7A700B305B7401306803EC6
:10E4200081469D8D97000100E78080B79314050118
:10E43000C180A1659385C503480097B0FFFFE780C1
:10E4400060598145480097D0FFFFE780603D8355C4
:10E450000404480097D0FFFFE780803E83552404E2
:10E46000480097D0FFFFE780A03D814589CCC16778
:10E47000FD179305F00F6388F40026859750000080
:10E48000E780E0E0AA85480097D0FFFFE7804039A9
:10E4900003554404814501CDC167FD179305F00F75
:10E4A0006307F50097500000E78060DEAA8548000A
:10E4B00097D0FFFFE780C03683456404480097D0BB
:10E4C000FFFFE780E03583457404480097D0FFFFE5
:10E4D000E7800035500001478146CE854A8597B0D8
:10E4E000FFFFE780807405611743FFFF670083BD6E
:10E4F000814481B71743FFFFE70223BB83C7950021
:10E5000093F7F707A384F50097000000E78020ED5C
:10E510001743FFFF6700A3BB1743FFFFE70243B7A3
:10E5200083C795004111404D93F7F707A384F50089
:10E530002A8A3285B284AE8997D0FFFFE780003EF9
:10E540002A8B268597D0FFFFE780403D2A892685C4
:10E5500097D0FFFFE780603A93170B0163CA070269
:10E56000E177CA97C207C183116763E3E7029307A4
:10E570000910C207C1831307B00F637BF70093171D
:10E580000901C187AA8A634AF000C54763FE5701A3
:10E5900041011743FFFF6700E3B297B0FFFFE78039
:10E5A000C028E31725FFD5B763080B0263060902ED
:10E5B000814463890A02B7077F0023106405231191
:10E5C00024057CC0568597000000E780E0C39304D3
:10E5D000803EB304950239A0B7077F0023200404CE
:10E5E0007CC081440355240497E00000E780A0A389
:10E5F000A1C497C0FFFFE78000BB269593D7F441E5
:10E6000033379500AE97BA9708DC5CDCCE8552852F
:10E6100097000000E780A0DC99E023220404A167B2
:10E620009387B70348003EC42302010002C697E067
:10E63000FFFFE7808005A9BF814701481CDC232E2E
:10E640000403E9B71743FFFFE70223A697C0FFFFC4
:10E65000E780C037E1473305F50291459750000048
:10E66000E78000C5E55711C59777FF1F23AAA7527A
:10E6700081473E851743FFFF670063A585471777EE
:10E68000FF1F2301F75282801743FFFFE702E3A138
:10E690009777FF1F9387875080433DC083570404BB
:10E6A0006390A70683572404639CB7043689B28419
:10E6B00097C0FFFFE78020AF5C5C63C3B70463953E
:10E6C000B7001C5C63EEA7028347640463F3F400A5
:10E6D000A6872303F4048347740463F39700A68793
:10E6E000A303F4048357440441677D176385E7005F
:10E6F00085072312F4043C4481C7CA852685829786
:10E700001743FFFF6700A39C9777FF1F9387074975
:10E710009C43014599C303C5870082801743FFFFCF
:10E72000E702A3980111B70707003EC683C795000B
:10E73000584D0AC493F7F7070AC8A384F5002A893D
:10E74000AE8411CB1C4283C707002304F7009790C7
:10E750000000E7800034216493055402280097B03C
:10E76000FFFFE780202797000000E78020FAAA85B6
:10E77000280097D0FFFFE780A00A300001478146BC
:10E78000A6854A8597B0FFFFE780204A130444021C
:10E79000480822CC230A010002CE97E0FFFFE78061
:10E7A000C0EE05611743FFFF670063921743FFFF49
:10E7B000E702A38F01117C003ECAB70707003ECCD9
:10E7C0007C003ECE83C795002E84AA8493F7F7077A
:10E7D000A384F500A16593855502480897B0FFFF13
:10E7E000E780401F97000000E78040F2AA854808B4
:10E7F00097D0FFFFE780C002500801478146A285FD
:10E80000268597B0FFFFE780404205611743FFFF71
:10E810006700E38B9777FF1F938747389C43094531
:10E8200099C303C5970082809777FF1F93870737A7
:10E830009C43094599C303C5D70082809777FF1F82
:10E840009387C7359C43014599C303C5A7008280C0
:10E850001743FFFFE702C3830111B70708003EC655
:10E8600083C79500404D0AC493F7F7070AC8A384ED
:10E87000F5002A89AE8429C41442854703C70600DF
:10E8800063E0E70A83479400094681496380C70231
:10E89000B307F740A304E400B339F00083C71600C0
:10E8A0002305F40097900000E780A01E035724037F
:10E8B000058B19C76386090097D00000E78000E93F
:10E8C000216493058402280097B0FFFFE780801041
:10E8D00097000000E78040F4AA85280097D0FFFF4A
:10E8E000E78000F497000000E78080F5AA85280003
:10E8F00097D0FFFFE780C0F2014781463000A68530
:10E900004A8597B0FFFFE78040321304740248083D
:10E9100022CC230A010002CE97E0FFFFE780E0D679
:10E9200005611733FFFF6700E3791733FFFFE70245
:10E93000C37701117C003ECAB70708003ECC7C00BB
:10E940003ECE83C795002E84AA8493F7F707A3844D
:10E95000F500A16593858502480897B0FFFFE78021
:10E96000600797000000E78020EBAA85480897D051
:10E97000FFFFE780E0EA97000000E78060ECAA85EF
:10E98000480897D0FFFFE780A0E95008014781467B
:10E99000A285268597B0FFFFE78020290561173300
:10E9A000FFFF6700C3729777FF1F9387271F9C4362
:10E9B000014599C303C5B70082801733FFFFE70203
:10E9C000C36E0111B70707003EC683C79500404DCF
:10E9D0000AC493F7F7070AC8A384F5002A89AE840E
:10E9E00005C81C42054783C707006368F70603474D
:10E9F000B400630FF700A305F40097900000E780D0
:10EA000040098347B400B9CF97D0FFFFE78040BEED
:10EA100021649305B400280097B0FFFFE78080FBD6
:10EA200097000000E78060F8AA85280097D0FFFFD4
:10EA3000E78000DF014781463000A6854A8597B010
:10EA4000FFFFE780801E2904480822CC230A01002A
:10EA500002CE97E0FFFFE78040C305611733FFFF59
:10EA60006700E36697D0FFFFE78020BF55B71733F5
:10EA7000FFFFE702836301117C003ECAB70707006E
:10EA80003ECC7C003ECE83C795002E84AA8493F7AB
:10EA9000F707A384F500A165AD05480897B0FFFF0F
:10EAA000E78040F397000000E78020F0AA8548083F
:10EAB00097D0FFFFE780C0D6500801478146A28566
:10EAC000268597B0FFFFE780401605611733FFFFEB
:10EAD0006700E35F9777FF1F9387470C9C430945C7
:10EAE00099C303C5C70082801733FFFFE702E35BCA
:10EAF00001117C00AE843ECAA165B70707002A84D5
:10EB00003ECCD1057C0048083ECE97B0FFFFE780A1
:10EB100060EC97000000E78020FCAA85480897D0A9
:10EB2000FFFFE780E0CF500801478146A685228598
:10EB300097B0FFFFE780600F05611733FFFF6700A5
:10EB400003591733FFFFE702435683C7950093F736
:10EB5000F707A384F50097000000E78020F917333A
:10EB6000FFFF6700C3561733FFFFE702635283C7F7
:10EB700095000329C501411193F7F707A384F50018
:10EB80001C4283C90700854763E637079777FF1F55
:10EB9000938707589C432E84AA8485CF9700000052
:10EBA000E78080F389476306F5026304090283471F
:10EBB000C900638037032306390197900000E7807E
:10EBC00040ED83572903898B89C797D00000E780E0
:10EBD000E0B72685A28597000000E78020F1A167B5
:10EBE000CD0748003EC42302010002C697E0FFFFA4
:10EBF000E780A0A941011733FFFF6700A34C977777
:10EC0000FF1F9387A7F99C431D4599C303C5E700E0
:10EC100082801733FFFFE70243490111B70707005E
:10EC20003EC683C79500584D0AC493F7F7070AC834
:10EC3000A384F5002A89AE8415C71C4283C7070048
:10EC400093968701E18663C4060685466381D706ED
:10EC50008346E7006388F6002307F70097900000DB
:10EC6000E78020E321649305E400280097B0FFFFCC
:10EC7000E78040D697000000E780A0F8AA8528002A
:10EC800097D0FFFFE780C0B9014781463000A685D5
:10EC90004A8597B0FFFFE78040F93504480822CC49
:10ECA000230A010002CE97E0FFFFE780009E056186
:10ECB0001733FFFF6700A3411733FFFFE702E33E6F
:10ECC00001117C003ECAB70707003ECC7C003ECE57
:10ECD00083C795002E84AA8493F7F707A384F500D1
:10ECE000A165B905480897B0FFFFE780A0CE97005F
:10ECF0000000E78000F1AA85480897D0FFFFE78071
:10ED000020B2500801478146A285268597B0FFFFB3
:10ED1000E780A0F105611733FFFF6700433B17331E
:10ED2000FFFFE702E336AA8401441779FF1F1309A6
:10ED300029E7E14997C0FFFFE78040C96344A40089
:10ED4000014519A833053403832709003E958357ED
:10ED500025006397970011051733FFFF670083367F
:10ED60000504C9BF032E8500630A0E121773FF1F27
:10ED70001303C301032303006315030029436390B6
:10ED8000061203234E01631503001D436399071008
:10ED90001733FFFFE702E32EC689428A3E89BA8A0B
:10EDA000B684328BAE8B2A84B5E103554E0019E54B
:10EDB00001431A851733FFFF67002330A167A98F2E
:10EDC000116763FBE70097000000E78080F581454D
:10EDD00097F0FFFFE780C0120844B70700E05841F2
:10EDE000F98F18455CC1B707001FF98F1CC55C4936
:10EDF00091C7610597E00000E780408BE38A09FA3C
:10EE0000228597900000E78060C65DB7328597C085
:10EE10000000E78040430D4349DD1C44116703D5E2
:10EE20004700A167A98F63FBE70097000000E78018
:10EE300040EF814597F0FFFFE780800C03238400BB
:10EE400093164B01D1828347B30003566300858834
:10EE5000FD8BA305F300FD777D8E558EFD76FD16A7
:10EE6000B204F18E83274301C58E2312730123134D
:10EE7000D3002304530123052301A3044301BDDF71
:10EE8000228597B0FFFFE78020CDAA850844B5D141
:10EE9000610597D00000E780207F8DB71D431A855C
:10EEA00082801733FFFFE702A31E0569AA84AE899B
:10EEB000328A0144FD5A7D1997C0FFFFE780C0A543
:10EEC0006347A40001451733FFFF6700A31FD84421
:10EED00093171400BA9703D70700631F37032390D3
:10EEE000570163070A00268597900000E780A080FD
:10EEF0009C449DC383D76700B3F72701639E370106
:10EF0000D2880148814701478146014681452685CF
:10EF100097000000E78040E5050479BF1733FFFF45
:10EF2000E702031779711C103EC4B7070F003EC6F5
:10EF30001C103EC883C79500AA8A328593F7F7074D
:10EF4000A384F5002E89328497D0FFFFE780009DCF
:10EF500093170501C187635AF006AA89228597D0C5
:10EF6000FFFFE780A09B2A8A4E85032B040097B001
:10EF7000FFFFE780009B39ED83574400814405443F
:10EF8000F11793B71700A303F10083457100DA87E7
:10EF90002287D2864E86280097E0FFFFE780E05761
:10EFA000014781463000CA85568597B0FFFFE7804C
:10EFB000C0C7A1679387F70348083ECC230A8100A6
:10EFC00026CE97D0FFFFE780406C45611733FFFFE7
:10EFD0006700430FA2851306710097E0FFFFE780EB
:10EFE0006066AA84094455D1528597E0FFFFE78007
:10EFF00060D40D4459D90546D28526859700000076
:10F00000E78060EA2A8451B71733FFFFE702E3097C
:10F01000835507000346270041112A842E8532C6F6
:10F020002EC497E0FFFFE780E0D001C93246A24539
:10F03000228597000000E78000E741011733FFFFBA
:10F040006700E3081733FFFFE702A30383C79500B8
:10F050004111AA8A93F7F707A384F5003285AE8998
:10F06000328497D0FFFFE780608B93170501C1873B
:10F070006357F00AC1452A8A228597C0FFFFE780BF
:10F0800080702A8D228597D0FFFFE78020892A890A
:10F09000228597D0FFFFE7804086930705F893F716
:10F0A000F70F1307E007AA8B637BF706228597D03B
:10F0B000FFFFE78080842A8C228597D0FFFFE780BE
:10F0C000C083AA8C5285032B040097B0FFFFE78012
:10F0D000408539E983574400231101008144F11729
:10F0E00093B71700A300F1000544034711008356AE
:10F0F0002100938784005685DA8822885286CE853F
:10F1000097F0FFFFE78020A7A167E90748003EC40A
:10F110002302810026C697D0FFFFE78000574101F8
:10F120001733FFFF670063F913061100A28597E00C
:10F13000FFFFE7802051AA8409E52311010009445B
:10F140006DB7930521006A8597F0FFFFE780A0F077
:10F150002A8441FD835521009356C90013164901A5
:10F1600085486688E2875E87858A51822685970072
:10F170000000E78060BF2A848DBF1733FFFFE702DE
:10F1800043F083C7950041112A8B93F7F707A384B7
:10F19000F5003285AE89328497C0FFFFE7800078A2
:10F1A00093170501C1876352F00A2A8A228597C006
:10F1B000FFFFE780A076AA8A228597C0FFFFE7803D
:10F1C000E0752A89228597C0FFFFE78000739307C7
:10F1D00005F893F7F70F1307E0072A8C6377F70614
:10F1E000228597C0FFFFE7804071AA8C228597C0D7
:10F1F000FFFFE78080702A8D5285832B040097A043
:10F20000FFFFE780007239E58357440085440144DD
:10F21000F11793B71700A301F100034731009307DB
:10F2200084005A85DE882688D6865286CE8597F059
:10F23000FFFFE78040948D4748003EC423029100C1
:10F2400022C697D0FFFFE780404441011733FFFFFC
:10F250006700A3E6A2851306310097E0FFFFE78071
:10F26000603E2A84894455D99356C9001316490132
:10F2700085486A88E6876287858A5182D6859700A5
:10F280000000E78060AEAA8449BF1733FFFFE702A2
:10F2900023E02A8981440144617A916A177BFF1F28
:10F2A000130BCBAE97B0FFFFE780006863C7A400E5
:10F2B00022851733FFFF6700E3E083270900939956
:10F2C0001400CE9703D50700330745014207418359
:10F2D0006364570305C103270B0019C785453E85A5
:10F2E00097400000E78060E9832709000504CE9776
:10F2F0002390070085047DB797000000E78060A297
:10F30000832709000504CE972390070065D5814522
:10F3100097F0FFFFE780C0BEF1BF1733FFFFE702A2
:10F3200023D783C7950041112A8A93F7F707A3844F
:10F33000F50032852E89328497C0FFFFE780005E9A
:10F3400093170501C187635AF004AA89832A040030
:10F3500097A0FFFFE780E05C31E5835744008544D8
:10F360000144F11793B71700A301F10003483100DE
:10F37000D68752850147CE862686CA8597D0FFFF5D
:10F38000E780806AA167F50748003EC42302910028
:10F3900022C697D0FFFFE780402F41011733FFFFC0
:10F3A000670043D2A2851306310097E0FFFFE78094
:10F3B00060292A8489445DD99777FF1F9387079D29
:10F3C0009C4381CF044997B0FFFFE780E055AA85B1
:10F3D000268597400000E78040DA13050401970076
:10F3E0000000E780C0EA228597800000E7800033B4
:10F3F0008144ADBF1733FFFFE702A3C883C7950061
:10F400004111AA8A93F7F707A384F5003285AE89E4
:10F4100032842311010097C0FFFFE780205093172B
:10F420000501C1876354F0062A8AC145228597C029
:10F43000FFFFE7804035AA8B5285032B040097A07D
:10F44000FFFFE780004E21E98357440085440144D3
:10F45000F11793B71700A300F100034811000357F9
:10F460002100DA875685D2862686CE8597D0FFFF83
:10F47000E780805BA1679387270248003EC4230290
:10F48000910022C697D0FFFFE7802020410117336B
:10F49000FFFF670083C2A2851306110097E0FFFFFC
:10F4A000E780401A2A8489444DD99777FF1F9387B4
:10F4B000E78D98433E8901CF044997B0FFFFE7806D
:10F4C000A046AA85268597400000E78000CB13055B
:10F4D000040197000000E78080DB97B0FFFFE78022
:10F4E000A04495443DD9930521005E8597F0FFFF28
:10F4F000E78060B6AA8435F11C48035721002285B5
:10F500002390E70097800000E780402183270900CF
:10F51000A9D70355210097400000E780A0BD35BF63
:10F520001733FFFFE702E3B583C795004111AA8AAD
:10F5300093F7F707A384F5003285AE89328497C02C
:10F54000FFFFE780A03D93170501C1876351F006D7
:10F550002A8A228597C0FFFFE780403C2A8952858E
:10F56000032B040097A0FFFFE780A03B31E5835702
:10F57000440085440144F11793B71700A301F1003B
:10F5800003483100DA8756854A87D2862686CE859B
:10F5900097D0FFFFE7804049A167F90748003EC4C4
:10F5A0002302910022C697D0FFFFE780000E4101A1
:10F5B0001733FFFF670063B0A2851306310097E0A1
:10F5C000FFFFE78020082A8489445DD99167CA97A4
:10F5D000C2071167C1831307F7EF8544E362F7FAA7
:10F5E0009767FF1F9387877A9843BE8B01CF0449A3
:10F5F00097B0FFFFE7804033AA852685974000003B
:10F60000E780A0B71305040197000000E78020C839
:10F6100097B0FFFFE780403195443DD11C482285DB
:10F6200081442390270197800000E780200F83A763
:10F630000B00B9D74A8597400000E780A0AB89B797
:10F640001733FFFFE70263A62A844105B2849700BF
:10F650000000E780C0C311C5228597800000E780C5
:10F66000E00B81460146A685228597800000E78051
:10F67000C04E1C4C89C7DC4799C32285829717333B
:10F68000FFFF6700C3A49767FF1F938727519C4321
:10F69000014599C31385070182809767FF1F9387F0
:10F6A000E74F884382801733FFFFE70203A09317D9
:10F6B000C600DD8DC2054111C1812A8432C697C0C2
:10F6C000FFFFE780E0173246228511829375F60F1F
:10F6D00097C0FFFFE780C01441011733FFFF6700A9
:10F6E000039F1733FFFFE702A39A79713C083ED2CC
:10F6F000B7070C003ED43C083ED683C79500AE84C5
:10F700002A8993F7F707A384F500A165938535044B
:10F71000481097A0FFFFE780E02BC165FD1501446D
:10F72000176AFF1F130A0A68930A400EAE892E8BD0
:10F730002EC697B0FFFFE7802022420593170401F1
:10F740004181C183B24563E9A702C167FD176387A1
:10F75000F500481097C0FFFFE780800E501001476A
:10F760008146A6854A8597A0FFFFE780004C45614A
:10F770001733FFFF670003953307540383270A0BF2
:10F78000BA9703D6C701630A3601638A3501481068
:10F7900097000000E78060F1DA85050451BFB2856B
:10F7A000EDBF1733FFFFE702C38D79717C083EC8B8
:10F7B000B70711003ECA7C083ECC83C79500AA89D2
:10F7C000328593F7F707A384F5002E8997C0FFFFD2
:10F7D000E780C01485676378F504A165AA8489056C
:10F7E000080897A0FFFFE780E01E268597400000ED
:10F7F000E78060ED133415000A04A285080897C05D
:10F80000FFFFE780E001A685080897C0FFFFE780BB
:10F81000200325CC014781461008CA854E8597A054
:10F82000FFFFE780804045611733FFFF6700E388F3
:10F83000B30754030327CA0ABA9703D70700631C08
:10F84000970003D62700638065050808970000002D
:10F85000E780A0E5DE8505042EC697B0FFFFE780B0
:10F86000A0104205931704014181C183B245E3E131
:10F87000A7FCC167FD17E38FF5F8080897C0FFFFE5
:10F88000E78000FC41BFB285F9B7C165FD150144B1
:10F89000176AFF1F130A0A51930A80022E8BAE8B40
:10F8A00065BF1733FFFFE702438018418347170006
:10F8B00083460700A207D58FD207D1832390F50096
:10F8C00083472700034717008D45A207D98F9183EF
:10F8D0002310F60097C0FFFFE780A0E91723FFFF82
:10F8E0006700E37E1723FFFFE702837AC1640144C8
:10F8F0001769FF1F1309094B93098002FD1497B084
:10F90000FFFFE78060066347A40001451723FFFF60
:10F910006700437B330534038327C90A3E95835729
:10F920000500E38597FE0504D9BF1723FFFFE70213
:10F9300023762A8AAE89B284B68A97400000E7808F
:10F9400080D819E591473E851723FFFF670083772D
:10F950002A894E8597C00000E780E08E2A84638E56
:10F960000A048D476DD103570500C547E31D47FDC8
:10F970000347F9018546AD47E317D7FC83474500A8
:10F9800081CF4146A6855D0597F00000E780C09EC7
:10F99000814755D9AD4745BF130965012302E500ED
:10F9A000CA85268597100000E780606231C1A547AF
:10F9B000E38B0AF82302040079B705C183570500D9
:10F9C000E39247F94146A685190597F00000E780C4
:10F9D000A09A81472DD99947BDB74E859700000061
:10F9E000E78080F02A84954739DD130955004DBF23
:10F9F0004146A68523104401231134011305190043
:10FA000097F00000E780A099228597800000E780AA
:10FA1000A0EA81470DBF1723FFFFE7020369797151
:10FA20007C003ECCB7070A003ECE7C003ED083C7A8
:10FA30009500B2842E8493F7F707A384F50013068C
:10FA4000A1002A892C00268597000000E780A0E508
:10FA5000A16528088D0597A0FFFFE780A0F79040DB
:10FA60008355A10003558100854697000000E7807B
:10FA700000ECAA84AA85280897C0FFFFE78040DA37
:10FA80000356A10083558100280897000000E780F5
:10FA9000C0C1300801478146A2854A8597A0FFFF73
:10FAA000E780A018854748103ED42302910202D671
:10FAB00097D0FFFFE78060BD45611723FFFF670018
:10FAC00003611723FFFFE702435E79717C003ECCA0
:10FAD000B7070A003ECE7C003ED083C79500B284B3
:10FAE0002E8493F7F707A384F5001306A1002A8953
:10FAF0002C00268597000000E780E0DAA165280841
:10FB00008D0597A0FFFFE780E0EC90408355A100B2
:10FB100003558100814697000000E78040E1AA84F8
:10FB2000AA85280897C0FFFFE78080CF0356A10071
:10FB300083558100280897000000E78000B730084F
:10FB400001478146A2854A8597A0FFFFE780E00D27
:10FB500048102302910202D402D697D0FFFFE7801B
:10FB6000C0B245611723FFFF670063561723FFFFED
:10FB7000E702A35397000000E78060DB1723FFFF35
:10FB80006700E3549767FF1F93878701884382804C
:10FB90001723FFFFE7026351835725004111AE840D
:10FBA0002A842307B10017F5FFFF130525466C00D3
:10FBB0002316F10097A0FFFFE780204991C422851A
:10FBC00097800000E780E0D6FD572310F40013066D
:10FBD00020028145130554009720FFFFE780E04F86
:10FBE00041011723FFFF6700834E1723FFFFE70242
:10FBF000234A79717C003ECCB7070A003ECE7C00D8
:10FC00003ED083C79500AA89AE8493F7F707328563
:10FC1000A384F5001306A1002C0097000000E780E4
:10FC200080C803558100114497400000E780A0A9D7
:10FC300015C50355A100014497B00000E780A060FE
:10FC400011CD035705008357810045446318F70021
:10FC5000854597000000E780E0F3014421699305A2
:10FC60003900280897A0FFFFE780C0D6A2852808A2
:10FC700097C0FFFFE780C0BA0356A10083558100FB
:10FC8000280897000000E78040A23008014781461D
:10FC9000A6854E8597A0FFFFE78020F948104AD43B
:10FCA0002302810202D697D0FFFFE780009E4561C4
:10FCB0001723FFFF670003411723FFFFE702433DC0
:10FCC0009767FF1F938787ED2A8488432E8915C580
:10FCD000035745038357C4016311F7022326050226
:10FCE00023180502410597D00000E780209C630699
:10FCF000090097800000E78060DB81449769FF1F5F
:10FD00009389490A130A800297B0FFFFE780C0C5B4
:10FD100063C4A4049767FF1F938707F19C4399C7A7
:10FD20000355C40197200000E780C0BD63070900A8
:10FD3000228597800000E780C0A01306400E814511
:10FD400022859720FFFFE7804039FD57231EF400EE
:10FD50001723FFFF670003373385440383A7C90ACE
:10FD60003E95035705008357C4016317F700CA8502
:10FD700097000000E78000E2850479B71723FFFFB2
:10FD8000E702033183C795004111AA8993F7F7076A
:10FD9000A384F5003285AE8497C0FFFFE78000B8EA
:10FDA00085676378F5042A8997400000E780A09171
:10FDB000014401CD83D70400314463882701854580
:10FDC00097000000E78080EF01444E85A2864A86B6
:10FDD000A68597D0FFFFE780A09CA16793871704B3
:10FDE00048003EC42302810002C697D0FFFFE7808F
:10FDF000C08941011723FFFF6700C32C1723FFFFB2
:10FE0000E70203299767FF1F938747D9804329C4D7
:10FE1000014597C00000E780002181470148C16487
:10FE20001CDC232E0403232004041769FF1F13097D
:10FE300069F701449309400EFD1497B0FFFFE78076
:10FE4000A0B1634FA400814517F5FFFF1305857F1F
:10FE500097A0FFFFE780601F1723FFFF670083263F
:10FE6000330534038327090B3E958357C501638708
:10FE70009700854597000000E78040E4050475BFC2
:10FE80009357050113D78700A380F5009317050149
:10FE9000C183A1832380E5002381F500A381A50010
:10FEA00082801723FFFFE70243202300050083C75A
:10FEB0001500A300F50083C725002301F50083C7C3
:10FEC0003500A301F50083C745002302F50083C771
:10FED0005500A302F50083C7650093059500A303B1
:10FEE00005002303F5002304050032859700000078
:10FEF000E78040F91723FFFF6700631D1723FFFF0B
:10FF0000E70203194111E9540DCD85CD93F9C5FFE1
:10FF10002E842A89AA84338AA900B7EA04006318C8
:10FF20009A020D88854411CCB7E704009C5F829744
:10FF30002AC622866C003305390197E00000E7806D
:10FF40000046268541011723FFFF6700A31783A7FB
:10FF50008A039104829793170501C183A183A38E1D
:10FF6000F4FE93570501238FF4FEA183238EA4FE94
:10FF7000A38FF4FE6DB763E6D5021723FFFFE702F8
:10FF8000C312B28741113686BE8536C697E000009F
:10FF9000E780E040B246410136851723FFFF670046
:10FFA0000313814636858280838705001387F50019
:10FFB0003D05FD8793F77708834607007D15860684
:10FFC000B58FA300F5006307B7007D1783471700BF
:10FFD0009D83DDB782801723FFFFE702030DB7E79C
:10FFE000040083A7070932872A863A85829713354A
:10FFF00015001723FFFF6700830D15C181478DC1D1
:020000040001F9
:100000001723FFFFE702630A414697E00000E780FD
:10001000003985473E851723FFFF6700430B814763
:100020003E8582801DCD1723FFFFE702030841466E
:1000300081452A849720FFFFE780200A41468145B9
:10004000130504039720FFFFE78020090147C167DC
:100050002322040438C87CC805451723FFFF670026
:1000600003070145828081473DCDB5CD1723FFFFB2
:10007000E702A303B2842E891306800581452A84F2
:100080009720FFFFE7806005CA8524C42685970076
:100090000000E780C0F64146814522859720FFFF9A
:1000A000E780A0033044A285228597000000E78006
:1000B000C0F293040401A285268597000000E78022
:1000C000E0EEA6851305040297000000E78000EE2D
:1000D000228597000000E78020F585473E8517239D
:1000E000FFFF6700C3FE3E8582801723FFFFE70204
:1000F00023FA4111E9540DCD85CD93F9C5FF2E8426
:100100002A89AA84338AA900B7EA040063984403C1
:100110000D88814411CCB7E704009C5F82972AC602
:1001200022866C003305390197E00000E780202724
:10013000268541011723FFFF6700C3F883A78A03C1
:100140009104829793170501C183A183A38EF4FEC6
:1001500093570501238FF4FEA183238EA4FEA38F62
:10016000F4FE6DB765CD1723FFFFE70263F2B2849B
:1001700011E605451723FFFF6700C3F42A842E8983
:100180000145EDD93C487848B3E6E700E5D69386CB
:10019000F7FFB3B7F6007D17032A4404BA9734C8B3
:1001A0007CC863050A06C14913050A03B38949419E
:1001B0002295637D3601B2862E86A68597000000C3
:1001C000E780A0DB7C40BE9464C065B7CE862E86F7
:1001D000CE8597000000E78040DAC114D2944E9992
:1001E00023220404A2879306040103C7070003C661
:1001F00007038507318FA38FE7FEE398F6FE3044AF
:10020000A285228597000000E78020DD2699C1495C
:100210003306994063EC9900A9DCA686A6851305F0
:10022000040397000000E78040D579BF8147B306FB
:10023000F4003307F6000347070083C5060085076F
:100240002D8F2380E600E39437FF3044A28522857A
:1002500097000000E78060D8C1145DBF014582802F
:100260000DC11723FFFFE70243E413068005814514
:100270009720FFFFE78060E605451723FFFF670033
:1002800003E501458280814749C5C1C51723FFFFAA
:10029000E702A3E1FC4141462E84AA846399C70486
:1002A00013860501A2878146C14503C7070003C520
:1002B00007038507298F3305D6000345050085060A
:1002C000298FA38FE7FEE392B6FE3044A2852685F0
:1002D00097000000E78060D0228597000000E7804B
:1002E00060F885473E851723FFFF670043DE1385CF
:1002F00007031D8E814522959720FFFFE780E0DDF3
:100300007C40130700F813060402A2972388E70233
:1003100051BF3E8582801723FFFFE70203D96D712D
:100320002E84B284AA859010280036899700000098
:10033000E780A0D309EDD55725A050400C402800F8
:1003400097000000E78040E27DD5FD142104F5F41C
:100350002C004A8597000000E78020F3814761DD8B
:100360003E8551611723FFFF670063D61723FFFF08
:10037000E702A3D341112EC432C62C0005469700D4
:100380000000E78080F941011723FFFF670023D4B5
:100390001723FFFFE70263D101112A842EC602C88A
:1003A00002CA02CC02CE97E00000E780402BB246A2
:1003B0002A86A285080897000000E78060FB137575
:1003C000F50F05611723FFFF670063D01723FFFFB9
:1003D000E702A3CD7971B2872A8421462308B100B0
:1003E00013051101BE853AC436C697E00000E780C8
:1003F00000FBB24693059101368597000000E78027
:1004000060A82285141035460C0897000000E7808C
:1004100020F62A84224701E921460C103A8597E00C
:100420000000E780C0F7228545611723FFFF6700C2
:1004300003CA1723FFFFE70243C77171AE84AA8581
:100440000A85328497000000E78060BB11C90A86E4
:10045000A685228597000000E78020B8814711E13A
:10046000C5473E854D611723FFFF670043C617232D
:10047000FFFFE70283C01D712A8AB289BE84354618
:100480008547130511012E8CB68A3A8BC28C468D96
:100490002308F10097E00000E78060F010100C08DE
:1004A0005285231F010097000000E780C0F82A84CE
:1004B0003DEDA1476313FD089307900591E0E547E3
:1004C0003546E2851305110113990A012308F1004D
:1004D0001359090197E00000E78060EC1357890089
:1004E00093978A00D98F90080C085285231FF1003A
:1004F00097000000E78020F42A8415E9A1E493879F
:10050000FA0091831379F9003EC66313090041494B
:10051000668B8144C14B854DB247639F970C6A86B9
:100520008C0033855C0197E00000E78040E722857E
:1005300025611723FFFF670003B893079004C9F0F4
:10054000A547BDBF834701050947C14B2308F100FB
:1005500083471105A58FA308F100938724008144E8
:1005600063E1FB04014714083386E6008C08B38678
:10057000E400BA95DA9683C6060083C50500050730
:10058000AD8E2300D600E390E7FE4147639CE7046D
:1005900090080C08528597000000E780C0E925D13B
:1005A00081A0B3069B00BA871008B305F600900837
:1005B0003E9603C506000346060085078506298E7C
:1005C0002380C500E39277FF998F90080C0852852D
:1005D000BE9497000000E78000E68947014749D1B3
:1005E0002A84B1B790083E96034606001408BE96CA
:1005F0002380C600850759BFB247850463879714D7
:1006000081471808B306F70098083E973386F9002B
:1006100003470700034606008507318F2380E60065
:10062000E39177FF90080C08528597000000E7805F
:1006300080E05DF53546E285130511012308B1011F
:1006400097E00000E780A0D51397040141839397BA
:1006500084002183D98F10180C085285231FF100C4
:1006600097000000E78020DD25FD814710183387C3
:10067000F9003E960347070003460600B306FB0059
:100680008507318F2380E600E39277FF65A818087D
:10069000B306F70098083E973386F9000347070032
:1006A000034606008507318F2380E600E3E127FF3C
:1006B000CA87639E770990080C085285970000004E
:1006C000E78060D711FD81479800B306F7009008D6
:1006D00018103E973E96034707000346060085071D
:1006E000318F2380E600E39177FF3546E2851305DD
:1006F00011012308B10197E00000E78040CA139779
:1007000004014183939784002183D98F10180C082A
:100710005285231FF10097000000E780C0D1E3114C
:1007200005EC814710183387F9003E960347070010
:1007300003460600B306FB008507318F2380E600E1
:10074000E3E227FFC109410BC1BB814785B794088C
:10075000BE9683C6060018083E972300D70085077B
:1007600089BF638006321723FFFFE70203915971A7
:100770002A84BE89B28B85473546130511022E8B1C
:10078000468C4289BA8A368A2300F10297E000003B
:10079000E780E0C010180C10228523170102970093
:1007A0000000E78040C963180512A147631FFC06DB
:1007B0009307900563930900E5473546DA851305ED
:1007C000110293140A012300F102C18097E0000096
:1007D000E780E0BC93178A0013D78400D98F900874
:1007E0000C1022852317F10297000000E780A0C4B7
:1007F0007DE1639209049307FA00BD88918391E03B
:10080000C144C207C183DE8C814A3EC6414DB24716
:1008100063E2FA0E6286B3854B01881097E0000010
:10082000E78080B54DC93D557DA093079004E396C0
:1008300009F8A54759B7834701050947C14C23006B
:10084000F10283471105B3C7F900A300F1029387B2
:100850002900814963E1FC04814618103306D70062
:100860008C083387D900B69556970347070083C590
:10087000050085062D8F2300E600E390D7FE414753
:100880006390E70690080C10228597000000E7802F
:1008900080BA35D189A0B3863A01BA871010B30562
:1008A000F60090083E9603C506000346060085073D
:1008B0008506298E2380C500E39297FF3387EC409D
:1008C00090080C102285BA9997000000E780A0B626
:1008D0008947014741D165611713FFFF6700A37D79
:1008E00090083E96034606001410BE962380C6006C
:1008F000850779B7B247850A93990A01939D8A00C3
:1009000093D909016391570F85473546DA85130559
:1009100011022300F10293D9890097E00000E780DB
:1009200000A8B3ED3D0190000C1022852317B10300
:1009300097000000E78020B059FD8147A68963EA4F
:10094000970626860C084A8597E00000E78020A5D8
:1009500081471810B306F700100898083E973E9696
:1009600003470700034606008507318F2380E60012
:10097000E3E197FE639FA90590080C10228597007C
:100980000000E78040AB21F981479810B306F700DB
:10099000900818183E973E96034707000346060046
:1009A0008507318F2380E600E391A7FF4109C10C41
:1009B000B9BD18089000B306F7003E963387FC00D7
:1009C00003470700034606008507318F2380E600B2
:1009D000B5B798084E97034707001C10CE972380A1
:1009E000E700850941BF85473546DA8513051102C1
:1009F0002300F10293D9890097E00000E780209A54
:100A0000B3ED3D0190000C1022852317B103970030
:100A10000000E78040A2E31005EC81471808900031
:100A2000B306F7003E963387FC00034707000346F2
:100A300006008507318F2380E600E391A7FF41463A
:100A40000C084A8597E00000E78060958147181000
:100A5000B306F700100898083E973E960347070034
:100A6000034606008507318F2380E600E391A7FF48
:100A700090080C10228597000000E780C09B1DD5D0
:100A800099BD7D5582801713FFFFE70203620111B4
:100A90002A842E8593055100328902C002C202C405
:100AA00002C69304740097F0FFFFE780A03D1D4647
:100AB000A6851305910097E00000E780408E10089E
:100AC0008A854A8597000000E780E09619ED930734
:100AD0001400180883C607000346070085070507AA
:100AE000B18EA38FD7FEE397F4FE05611713FFFFC6
:100AF0006700E35D1713FFFFE70283592E848C41E3
:100B00004111AA89838715003289914463D3070074
:100B1000A1449757FF1F9387A75F9C43A1C7C1CAF2
:100B20008D472310F10083C725004A852301F1007A
:100B300083C73500A301F10083C745002302F100FC
:100B400083C75500A302F10083C765009305910098
:100B5000A30301002303F1002304010097F0FFFF2A
:100B6000E78040320C404A860A8597F0FFFFE78015
:100B700080330328040083564400A6881D0881475B
:100B80000147E51642868A854E8597000000E7807A
:100B9000408E2A8919E5A685228597B0FFFFE78058
:100BA000E0C14A8541011713FFFF6700A3514A8640
:100BB0000A8597F0FFFFE780002F6DB71713FFFF3F
:100BC000E702034D2E848C414111AA8983871500C9
:100BD0003289914463D30700A1449757FF1F93873D
:100BE00027539C43A1C7C1C68D472310F10083C77B
:100BF00025004A852301F10083C73500A301F100D8
:100C000083C745002302F10083C75500A302F1000A
:100C100083C7650093059100A30301002303F1003E
:100C20002304010097F0FFFFE780C0250C404A86AF
:100C30000A8597F0FFFFE7800027835644000328CA
:100C400004008A85858EC2061D08C1822312D40045
:100C5000A68881470147E51642864E859700000029
:100C6000E78060B041011713FFFF6700A3454A8684
:100C70000A8597F0FFFFE78000234DBF1713FFFFA2
:100C8000E702A342B335B000011185052A89131587
:100C9000F601336515012308B1009305110136846F
:100CA0003AC632C03EC442C297F0FFFFE780801DC3
:100CB000A2471248425593D68700230BF1009305B3
:100CC000910193578800A30AD100A30BF100230CD4
:100CD000010197F0FFFFE780E01A32470246032840
:100CE0000400B337E000835644009207914411C2D8
:100CF000A1444A85A68842860C0897F0FFFFE7804A
:100D000040772A8919E5A685228597B0FFFFE780FD
:100D1000E0AA4A8505611713FFFF6700433B1713DD
:100D2000FFFFE702E33601113EC68647B335B00048
:100D30008505AA891315F6015D8D2308B100930579
:100D4000110136843A89B28442C446C297F0FFFF4B
:100D5000E780401322489248164593578800A30A1B
:100D6000F1009305910193D78800230B0101A30B98
:100D7000F100230C110197F0FFFFE780A01032472C
:100D8000104083564400B337E0009207032809005F
:100D9000914891C0A1480C084E8597000000E7805B
:100DA000809CAA8401E9835544004A8597B0FFFFDF
:100DB000E780C0A0268505611713FFFF6700833019
:100DC000AA959307F00F171701001307A798631749
:100DD000B50013C5F7FF1375F50F8280050583462F
:100DE000F5FFB58FBA9783C70700D5B703574500FE
:100DF00014419307F00F171601001306A6953697B6
:100E000042074183139506014181631BE500AD8FC5
:100E1000B29703C50700130515F31335150082803B
:100E2000850603C5F6FFA98FB29783C70700D9BF10
:100E30001713FFFFE7026327B28736842E86BA8630
:100E4000AA853E85BA8497F0FFFFE7806052634F22
:100E50000500228597E00000E78060802A86A6864C
:100E6000A285268597F0FFFFE78080501713FFFFCC
:100E70006700E3251713FFFFE70283215D712A8BCB
:100E8000AE8A171501001305658A2C00B284368AD4
:100E9000BA893E8997F0FFFFE780C04F2A845DE161
:100EA00034104146DA85280097F0FFFFE780404C78
:100EB0002A8449E98547A303F100A6C2930771007C
:100EC0002408BEC4A68685470D462C18281002DCCF
:100ED00002DED6C0BEC697F0FFFFE78000442A843A
:100EE00035E183477102A6860D4693F7F707230085
:100EF000FA00C1473EDE2C188947281026DCA303E0
:100F0000F10097F0FFFFE78040412A8405ED41465C
:100F1000A6854E8597D00000E78060488D47A6865D
:100F20000D462C182810A303F10097F0FFFFE7806F
:100F3000C03E2A8401E94146A6854A8597D0000033
:100F4000E780E045228561611713FFFF6700831783
:100F50001713FFFFE702631597F70000938707EF6A
:100F6000984383C7470079712A89AE841705010029
:100F70001305457C0C083AC42306F10097F0FFFFE7
:100F8000E78040412A8405ED14104146CA850808CF
:100F900097F0FFFFE780C03D2A8415E1140815464D
:100FA0002C00081097F0FFFFE780803C2A8401E9BD
:100FB00021462C08268597D00000E780403E2285F8
:100FC00045611713FFFF670083101713FFFFE70248
:100FD000C30D97F70000938767E79C477971AA8450
:100FE0002E8417050100130565750C083EC697F0A1
:100FF000FFFFE780203A0DE914104146A685080856
:1010000097F0FFFFE780C03605E1140811466C0039
:10101000081097F0FFFFE780A03519E58347F1013D
:1010200093F7F7032300F40045611713FFFF6700F0
:10103000030A1713FFFFE70243073688A1488147D9
:101040000147E54697F0FFFFE780A0421713FFFF37
:101050006700E3071713FFFFE70223053688A1485F
:1010600081470147E54697F0FFFFE780C06F171300
:10107000FFFF6700C3051713FFFFE702030301111A
:101080002A842E850C0832C697F0FFFFE780803057
:1010900009ED3247970601009386C6681008C145DE
:1010A000228597000000E780E0D805611713FFFF55
:1010B0006700E3011713FFFFE70223FF4111C14758
:1010C0002EC032C48A8509463EC23EC697F0FFFF55
:1010D000E780A02441011713FFFF670043FF1713A8
:1010E000FFFFE70283FC4111AE8613061009AA85B3
:1010F0000A8502C002C202C402C697F0FFFFE78061
:10110000202741011713FFFF670063FC1713FFFF40
:10111000E702A3F93287970601009386A6622E861E
:101120009305000297000000E780C0D01713FFFF6F
:101130006700E3F91713FFFFE70223F77971C1474F
:101140002ACC2ED032D42C080D4628003ECE3ED2DA
:101150003ED602C402C602C802CA97F0FFFFE7806B
:10116000C01B45611713FFFF670063F61713FFFFEE
:10117000E702A3F30111AA842E84170501001305C9
:10118000E55C8A8597F0FFFFE780C02015E514082D
:101190004146A6850A8597F0FFFFE780601D09EDAF
:1011A0008347E1010347F101A207D98FCA07C98329
:1011B0006177D98F2310F40005611713FFFF6700D3
:1011C00003F115CD1713FFFFE70223EE9757FF1F1B
:1011D000938787A190439755FF1F938525A11755A6
:1011E000FF1F1305659C97D00000E78000C51755C9
:1011F000FF1F1305659B1713FFFF670043ED17558E
:10120000FF1F1305659A82808DCD1713FFFFE7023C
:10121000C3E99757FF1F9387279D944301112E849D
:101220000A869755FF1F9385659C97D00000E7803D
:1012300040C60A850294014505611713FFFF670048
:1012400003E97D5582801713FFFFE70203E697D07D
:101250000000E78080D19757FF1F23A7A79817F5B5
:10126000FFFF1305E5C997B00000E780C0741713AE
:10127000FFFF6700C3E51757FF1F13072799931751
:10128000150008433E95FD572310F5008280171383
:10129000FFFFE70283E12A84084009E51713FFFFF7
:1012A0006700E3E21C4158401CC06313E5005CC0CA
:1012B0008347550023200500F99BA302F50097A062
:1012C000FFFFE780207CC9BF1713FFFFE70243DC65
:1012D0009757FF1F9387879598432A8411CB83479D
:1012E000350093F7070289C7035505008945029722
:1012F0001305440197B00000E780403B835504008C
:101300000355E40097300000E780A00C485819C549
:1013100097A0FFFFE7800077232A040213058403C8
:1013200097000000E780E0F68144B1499790FFFF05
:10133000E780C06D63CBA4028347340023200404FC
:1013400093F727FCA301F40000489790FFFFE78084
:10135000E06C13161500814522859710FFFFE7808A
:10136000C0D71713FFFF6700E3D5B3873403032902
:10137000040385043E994A8597000000E78060F1E8
:101380002304090065B78347350093F7070299E303
:10139000014582808357E500E39CB7FEC167FD17D6
:1013A0006316F60005458280054599A81713FFFFCF
:1013B000E702A3CF93170601C187B2842A840149AB
:1013C0006359F002835705009DCB01456367F60022
:1013D000034584003E953325A6001375F50F0DA037
:1013E0001C4813171900BA9783D70700E38E97FAA2
:1013F00005099790FFFFE7806062E343A9FE01457E
:101400001713FFFF6700A3CC1713FFFFE70243C8C2
:10141000AE89AA849790FFFFE78000562A8497D070
:10142000FFFFE780A02EAA860147130684019705D7
:101430000000938585E41745FF1F1305657D979090
:10144000FFFFE780801C2A8925C98C441304C5004E
:1014500022859E0593F5050897A0FFFFE780403C95
:10146000CC4083877400E18163DD070493E50508C0
:10147000228597A0FFFFE780A03A0D4693854400A0
:10148000228597A0FFFFE780C03683D50400228520
:1014900097A0FFFFE780E03D83D52400228597A039
:1014A000FFFFE780003D03D6490083A509002285A0
:1014B00097A0FFFFE780E0334A851713FFFF67001F
:1014C00063C093F5F5076DB71713FFFFE702E3BDA0
:1014D00001112A84328532C697A0FFFFE780E027FA
:1014E0009780FFFFE7806034835704001757FF1F82
:1014F0001307478B3246231BF100930700F8A30D17
:10150000F1001C471843231AA1008983858BB30778
:10151000F740B28548083ECE231C0100230D010090
:1015200097000000E78080EE05611713FFFF67005A
:1015300003BA1713FFFFE702A3B5004101453DC4FD
:101540009304C40026853289AE8997A0FFFFE78007
:10155000C02495452A8A2685035B040197A0FFFFD6
:10156000E7802021268597A0FFFFE780603E8D451C
:10157000AA8A268597A0FFFFE780A01F268597A04F
:10158000FFFFE780E03C5C48420A135A0A01D29709
:101590005CC423186401814763983A0146054D8174
:1015A000330625419337160013F5F70F1713FFFF86
:1015B000670043B11713FFFFE702A3AC89692A8BC9
:1015C000AE8B328AB68A81440144314CFD19979022
:1015D000FFFFE780A04363CDA4009790FFFFE78063
:1015E000E045018D33B5AA001713FFFF6700E3AC98
:1015F0003389840383270B003E9963170A008347CE
:10160000890085043E94E1B703560A00DE854A85C9
:1016100033F6C90097000000E780E0F16DD1054581
:10162000E1B71713FFFFE70243A801112A847C00EA
:101630000355E5003ECAB70707003ECC7C003ECE0E
:1016400097200000E78020082A898545480897A050
:10165000FFFFE78020399945480897A0FFFFE78002
:10166000E015AA844A8597200000E780A00823801F
:10167000A4009747FF1F9387E7729C4341661306B8
:1016800006F09396870113D78701558F93D687006D
:10169000F18E558FA207B706FF00F58FD98F11463F
:1016A0002C00138514003EC497D00000E78020CFA3
:1016B0005008A38204008945228597000000E78036
:1016C000E0E019C9AA851305840397A0FFFFE7800E
:1016D000E0313C4085073CC005611713FFFF670000
:1016E000039F1713FFFFE702439C9790FFFFE780DC
:1016F000E0342A8405049790FFFFE7802033330508
:10170000A402F14791453305F50297200000E780D8
:1017100020BA11E565551713FFFF6700439B9747F4
:10172000FF1F23ADA74E9790FFFFE78020312A844B
:1017300005049790FFFFE780602F3305A4028945D9
:10174000060597200000E780A0B669D59747FF1FE0
:1017500023AEA74A9790FFFFE780402E2A84050416
:101760009790FFFFE780802C3304A4029747FF1F68
:101770002390874A9790FFFFE780402C2A84979018
:10178000FFFFE780A02A930714003385A70297473D
:10179000FF1F2390A748970701009387E7BE1747CD
:1017A000FF1F232BF7460145BDB71713FFFFE702C5
:1017B000238EAA842E8901449749FF1F9389895E4D
:1017C000130A80069790FFFFE78040266347A40036
:1017D00001451713FFFF6700E38E3305440383A71A
:1017E00009024A86A6853E9597000000E780E0B989
:1017F00019E10504C1BF0545E9BF1713FFFFE70263
:101800004388AA8A2E8BB28B368C3A8A8144014453
:101810008149974CFF1F938CEC58130D80069790CD
:10182000FFFFE780A02063C9A40011E085494E8531
:101830001713FFFF670063883389A40383A70C0293
:101840005E86D6853E994A8597000000E780E0B322
:101850001DC19790FFFFE780601E0544636D450141
:10186000D2866286DA851305090397000000E780B7
:10187000A0D411C1854985045DB71713FFFFE702A6
:101880002381C16441112A8901449749FF1F93892B
:101890006951130A8006FD1436C632C42EC29790D1
:1018A000FFFFE780A01892452246B2466348A40095
:1018B000014541011713FFFF6700C380330544034F
:1018C00083A709023E9509C683473500C18B9DC792
:1018D00091C68347350093F707028DC363069900CD
:1018E0008357E500639C27010357050001CB63E79D
:1018F000E50083478500BA97E3CDF5FA050469BF93
:101900001703FFFFE702C378C1642A89014497499E
:10191000FF1F93892949130A8006FD149790FFFF42
:10192000E780C0106346A4001703FFFF67008379B8
:101930003305440383A709023E958357E500638A74
:101940009700630499006396270197000000E780E1
:10195000E0970504E1B71703FFFFE7020372896907
:101960002A8AAE8A328BB68B8144174CFF1F130C28
:101970006C43930C8006314DFD199790FFFFE78073
:10198000E00A63C6A4001703FFFF6700C372338930
:10199000940383270C028355CA015A863E994A85CF
:1019A00097000000E780609E31C1814D15A033840F
:1019B000AD038327090303D60B00D68533F6C90090
:1019C0003E94228597000000E780E0B609E9850D86
:1019D0009790FFFFE7808003E3CBADFC01A8228551
:1019E00097000000E780E08A23040400850471B7B3
:1019F0001703FFFFE702E3684169AA8A014A174B10
:101A0000FF1F130B2B3A7D19C14B054C9790FFFF1D
:101A1000E780C0016346AA001703FFFF6700E36980
:101A200093098006B3073A0383290B02BE9983D733
:101A3000E900638E270163842A01639A570103A496
:101A4000890301E84E8597000000E780C0BD050AC4
:101A500075BF83570401639977099304C4002685F1
:101A600097A0FFFFE78060D385452A8D2685835C9C
:101A7000040197A0FFFFE780C0CF268597A0FFFF56
:101A8000E780A0E762056185635905048D452685D9
:101A900097A0FFFFE780E0CD8945268597A0FFFF4F
:101AA000E78020CD8945268597A0FFFFE78060CCA1
:101AB0008545268597A0FFFFE780E0CC834705009A
:101AC000094793F7F707639AE7009945268597A09A
:101AD000FFFFE78040CBA30285014848337D2D01FD
:101AE000231894016A9548C40040A1BF1703FFFF63
:101AF000E702A35B37E404008327041D829797471E
:101B0000FF1F83C727171725FF1F1305659EA30017
:101B1000F5008327441C82978327841C8146130683
:101B2000F00F8145014582971703FFFF6700235A95
:101B30001747FF1F1307070418439745FF1F83C567
:101B400065139747FF1F93876711834687030346F3
:101B500097036397D5009747FF1F238DC710828097
:101B600083C587010347A7036317B6009747FF1F85
:101B70002382E710828003C687016317C700974757
:101B8000FF1F2389D70E828083C687011307500267
:101B90006319D700930760021747FF1F230CF70C48
:101BA000828083C68701130660026315D6009307FF
:101BB0007002DDB783C7870155BF9747FF1F938723
:101BC000E709D44B0947638DE6081703FFFFE702D7
:101BD000C34D1749FF1F1309A9053E848347090018
:101BE000918B9DCFB7E4040083A7041D829783A740
:101BF000441C1745FF1F13052504829783A7841CE7
:101C000081461746FF1F03462605814501458297F9
:101C100021C583470900ED9B1747FF1F230AF700E3
:101C20008347040093F7F70F85CB91471747FF1FB2
:101C30002320F70497000000E78080EB9700000066
:101C4000E78040EFB7E70400BC4F41469145174598
:101C5000FF1F0345250182971703FFFF67002347F6
:101C600082801703FFFFE70243448D47411163065B
:101C7000F504C5476308F50285476310F5029747E9
:101C8000FF1F238BA7FEB7E70400BC4B9305001092
:101C90001745FF1F034505FD829741011703FFFF0D
:101CA0006700E34285471747FF1F2307F7FCB7E7A5
:101CB0000400BC4B93050020E1BF9747FF1F9387AB
:101CC000E7F9D44B1147638DE600B7E7040083A71B
:101CD000071D8297B7E70400BC4B930500044DBF76
:101CE00005491747FF1F232527F983C7070032C679
:101CF0002E8493F7F70FD5D3B7E4040083A7041D10
:101D00007D141374F40F8297E37689FCB2459947EA
:101D100003C61500E3F0C7FCFC4409061745FF1F86
:101D20001305C5F58297BC48930500081745FF1FAA
:101D3000034545F3829779BF1703FFFFE702E336B8
:101D40001747FF1F130787F14047184B1C40974662
:101D5000FF1F23ABF6F06316E4001747FF1F23278E
:101D6000F7F0130584FE9790FFFFE78000AA035564
:101D700064FF9780FFFFE780807297A0FFFFE780F6
:101D800060D01703FFFF670083341703FFFFE702EC
:101D9000C3319747FF1F938767ECD84BDC4789C750
:101DA00097000000E78080F985471747FF1F232130
:101DB000F7EC9747FF1F9387E7DB9C4393050002EF
:101DC0001745FF1F034505EA83C787031747FF1F12
:101DD0002302F7EAB7E70400BC4B82971703FFFF23
:101DE0006700E32E9747FF1F23ACA7E68280170307
:101DF000FFFFE702E32937E404007C4CA1451745C7
:101E0000FF1F034525E682977C48A1451745FF1F24
:101E1000034545E59744FF1F938444E48297DC44DF
:101E200089EB97000000E78080D91703FFFF670068
:101E3000632903D567FF9780FFFFE7804066AA8983
:101E40006DD1D84891476310F7027C4C91451745F6
:101E5000FF1F034525E182977C4891451745FF1FE9
:101E6000034545E0829703A9490103D40901894745
:101E7000B7E904001747FF1F232CF7DE83A7091DCE
:101E800021044204829783C784011715FF1F13059D
:101E9000256661191717FF1FA30CF76483A7491C58
:101EA000418082979747FF1F238807DC83A7C91CBF
:101EB000814609469375F40F4A85829711E9974741
:101EC000FF1F83C7A7EB89C79710FF1FE78020CFAD
:101ED000B7E70400BC4F2146A1451745FF1F034546
:101EE00065D8829799B71703FFFFE702031C93F7A2
:101EF000052001112E8481CF97000000E78020E9A2
:101F00001345042005611703FFFF6700431C93F787
:101F10000510A9CF9744FF1F938444D4DC48970051
:101F20000000E78020C11747FF1F1307A7C418430D
:101F300083C78401034787036318F700DC4489C71C
:101F400097000000E78080DF85471747FF1F2321A8
:101F5000F7D2B7E70400BC4B930500021745FF1FFB
:101F6000034545D082971345041069BF93F70508D0
:101F7000BDC79747FF1F83C777D0E9171946974515
:101F8000FF1F9385C5CF1305D10093F4F70F1749B1
:101F9000FF1F0349A9CE97C00000E78040409397F8
:101FA0000401C1831747FF1F1307C7CD231DF1008D
:101FB000231CF1009747FF1F938747CA3ACE3ACABE
:101FC000D8432306010009CBDC439315890154084B
:101FD0000D46E185680082971345040825B793F7FD
:101FE0002500A5C39747FF1F938747C7D84B89474D
:101FF0006306F7029747FF1F83C787C313F72700BE
:1020000011EF918B99CFB7E70400BC4F1306000A7C
:1020100089451745FF1F0345E5C4829713452400F2
:10202000D5B59747FF1F9387E7B49C4383C78703C2
:102030001747FF1F2300F7C497000000E78060DB0D
:10204000F1BF93F7050281CB97000000E78060DACB
:102050001345040245BD93F7850081CB970000002E
:10206000E780E0D21345840071BD93F7150081CB62
:1020700097000000E780A0B41345140061B593F702
:10208000450081CB97000000E78060B31345440012
:1020900095BD93F7050495C39747FF1F83C707BCFA
:1020A00091CB97000000E780A0A491471747FF1F3E
:1020B0002320F7BC13450404B1B593F7050101458E
:1020C000E38207E49747FF1F938747B9D84B9147AF
:1020D0006310F7049747FF1F938787B59C4313D777
:1020E00027008583D98F858B91E7B7E7040083A705
:1020F000071D8297B7E70400FC4F91451745FF1F66
:10210000034545B6829785471747FF1F2322F7B639
:1021100013450401C5BB9747FF1F2381A7C68280D3
:102120001703FFFFE70263F89747FF1F23AE07B2CD
:102130009747FF1F23AC07B285471744FF1F1304BF
:1021400064A31747FF1F2325F7B21C4083C78703EB
:102150001747FF1F2300F7B29790FFFFE7804093D8
:1021600029C59717FF1F23A9A7381C401705000092
:102170001305A5D783C787031747FF1F230CF7AEA7
:102180001717FF1FA306F7369747FF1FA38807AC53
:10219000B7E7040083A7070882979747FF1F2383A9
:1021A000A7AC1703FFFF670083F2B7C7898E938739
:1021B00067ED1717FF1F2321F73445BF1747FF1F90
:1021C0000347C7A9795555E79747FF1F938707A985
:1021D00003C7170005079746FF1FA381E6A803C79B
:1021E00017008D463377D7029746FF1FA388E6A6D0
:1021F00083C617001747FF1F1307C797184393F6A7
:10220000F60FA9EE834787031747FF1F2304F7A69E
:1022100085471747FF1F2303F7A49747FF1F93879F
:1022200027A19C430145998BA9E71703FFFFE7020C
:10223000C3E737E404007C48C1451745FF1F034549
:1022400065A282973C4885451745FF1F034585A138
:10225000829701451703FFFF670063E783C71700F5
:1022600085466395F6008347970379BF8347A703A5
:1022700061BF82809747FF1F83C7479EA1CF170387
:10228000FFFFE70283E237E404009747FF1F23873D
:10229000079C7C4885451745FF1F0345A59C8297F1
:1022A0007C4C91451745FF1F0345C59B82977C4891
:1022B00091451745FF1F0345E59A82973C48C14564
:1022C0001745FF1F0345059A829701451703FFFF36
:1022D0006700E3DF795582801703FFFFE702E3DC45
:1022E0002A84035565FF9780FFFFE780401B9747CF
:1022F000FF1F9387A796D847BE841DEF9790FFFFD7
:10230000E78080779C48232004009DEB9747FF1FC0
:1023100023AE87949747FF1F23A88794B7E704004D
:10232000BC4B89451745FF1F0345C593829701455F
:102330001703FFFF6700A3D9630A8700184375BF1F
:1023400080C39747FF1F23A38792C9BF7955CDB795
:102350001703FFFFE70263D59747FF1F938747A245
:1023600088432326050023240500510597A000007B
:10237000E780C0331703FFFF670063D51703FFFF34
:10238000E702A3D21744FF1F1304849F1C4041118E
:1023900099CF9C472302B5002AC61CC197000000B4
:1023A000E78040FB1C409C4B99C33245829741011A
:1023B0001703FFFF6700A3D11703FFFFE702E3CE78
:1023C0004111444D328532842EC69790FFFFE7803D
:1023D000C0522AC422859790FFFFE780205403A8AB
:1023E0004400630C0800B24583574400184022465D
:1023F00083D54500AA862685029841011703FFFF71
:102400006700E3CC1703FFFFE70223CA404D1DC856
:1024100008C097050000938565031305440197A044
:102420000000E78040169747FF1F938767959C43FE
:10243000014589E79747FF1F23A487941703FFFFF0
:102440006700E3C87D55DDBF1703FFFFE702E3C563
:10245000011168009305F00F02C602C802CA02CC3F
:1024600002CE97000000E780A0F105611703FFFF8F
:102470006700E3C59747FF1F938787909C43D84722
:10248000A1679D076319F7021703FFFFE702E3C186
:10249000011132859790FFFFE7802046230AA100B3
:1024A0008145680097000000E78080ED0561170313
:1024B000FFFF6700C3C182809747FF1F9387478C48
:1024C0009C43D847A167938777036319F7021703E3
:1024D000FFFFE70283BD011132859790FFFFE78080
:1024E000C041230AA1008145680097000000E780F1
:1024F00020E905611703FFFF670063BD82809747EE
:10250000FF1F9387E7879C43D84795476316F704D7
:102510001703FFFFE70263B90111328532849790F8
:10252000FFFFE780803D230AA10022859790FFFFEF
:10253000E780C03E83574400231BA10081453ECC69
:102540001C4068003ECE97000000E78060E3056114
:102550001703FFFF6700A3B78280930785FF8DC332
:102560008327C5FF91CFDC4B81CF1703FFFFE70225
:10257000C3B3032585FF82971703FFFF670023B5C9
:1025800082801703FFFFE70243B22A8432859790C7
:10259000FFFFE7808036BD4763EBA70018449377C1
:1025A000F5000345B70041995D8DA305A70017030A
:1025B000FFFF6700C3B11703FFFFE70203AF01117D
:1025C0007C003ECAB70707003ECC7C003ECE5C4D87
:1025D000A9C72A8413858700AE8497A00000E780EE
:1025E000E0FCA1652A899D0548089770FFFFE780F8
:1025F000603E9305803EB345B902480893F5F50F58
:102600009790FFFFE780C021014781465008A685CB
:1026100022859770FFFFE780406105611703FFFF88
:102620006700E3AA1703FFFFE70223A89700000053
:10263000E780A0F81703FFFF670063A91703FFFFF8
:10264000E702A3A601117C00AE843ECAA165B707CC
:1026500007002A843ECC48087C00938575033ECE53
:102660009770FFFFE78000371C44480883C5B70018
:10267000BD899790FFFFE780A01A50080147814667
:10268000A68522859770FFFFE780205A0561170312
:10269000FFFF6700C3A31703FFFFE70203A12A841C
:1026A000AE8497000000E78000EEA68522859700A3
:1026B0000000E780E0F81703FFFF670043A117035E
:1026C000FFFFE702839E97000000E78060F7170393
:1026D000FFFF6700C39F1703FFFFE702039D032966
:1026E000C5014111630809022A843285B28497909A
:1026F000FFFFE78080202AC626859790FFFFE780AE
:10270000E021832749002A8691C7DC4781C7B2456B
:102710002285829741011703FFFF6700439B170340
:10272000FFFFE7028398444D91CC2A84328597902D
:10273000FFFFE780A01EDC40AA8589C79C4799C39C
:10274000228582971703FFFF670063981703FFFF37
:10275000E7020394032AC5014111630D0A062E897D
:10276000AA849545328532849770FFFFE7808026E2
:10277000854522859790FFFFE7804004AA89CA8596
:1027800022859790FFFFE780A00B83274A008DCB1F
:10279000DC439DC722859790FFFFE780A000832739
:1027A0004A00104083564400DC437115A307A10082
:1027B000B2961307F1004E86CA852685829701C519
:1027C0002380090001A88345F10022859790FFFF2F
:1027D000E780C0FE41011703FFFF6700A38E1703C8
:1027E000FFFFE702838C65711C083EC2B7078001BA
:1027F0003EC41C0832893EC62A84AE84970000007D
:10280000E780A0ED4A859790FFFFE780201183576E
:10281000A1008DC3AA855000228597000000E780A3
:1028200020F3014781465000A68522859770FFFF5F
:10283000E780A03F59611703FFFF67004389170333
:10284000FFFFE702E38465711C088329C5013EC2CE
:10285000B70780013EC41C082A84AE8432893EC674
:1028600097000000E780E0EB638A09024A859790B1
:10287000FFFFE780A00A8357A100AA8585C3500007
:10288000228597000000E780A0EC014781465000B8
:10289000A68522859770FFFFE780203959611703CD
:1028A000FFFF670023821703FFFFE70203806571C4
:1028B0001C083EC2B70780013EC42A841C0832852A
:1028C0003EC6AE849790FFFFE78040058357A10086
:1028D0008DC3AA855000228597000000E78040E75D
:1028E000014781465000A68522859770FFFFE7804B
:1028F000C033596117F3FEFF6700637D17F3FEFFD6
:10290000E702A37A444D81EC8347450093B7170053
:10291000B307F0403E8517F3FEFF6700437B184581
:10292000FD576DDB97070000938747032A845CCB34
:10293000970500009385A5C21385840097A0000029
:10294000E78060C480C003474400814761F71737C0
:10295000FF1F232997427DBF17F3FEFFE702437352
:102960008329C50141110329850081476387090A2D
:102970000324090191452A8A22859770FFFFE78089
:102980006005854522859790FFFFE78020E3894514
:10299000AA8A22859790FFFFE78040E2AA84977079
:1029A000FFFFE780400A83A749002A8B8DCB9C4319
:1029B0009DC722859790FFFFE780C0DE83A749006F
:1029C000A306A1001040835644009C431307D10086
:1029D000B296D6851306E1005285829709CD8357BA
:1029E0000B002380F400A183A380F40023800A005D
:1029F000A306010039A88357E10022852380F40053
:102A00008345D100A183A380F4009790FFFFE78066
:102A1000E0DA8347D100B337F0000347B9009207EB
:102A200001453D9BD98FA305F900410117F3FEFF36
:102A30006700436917F3FEFFE702236741110DEDBD
:102A40009737FF1F93870734804315C80440130945
:102A500084009DC95C4099C79C4B89C726852EC6BA
:102A60008297B2459307803EB385F5024A8597A0C9
:102A70000000E78060C121A0404DAA8469F84101AF
:102A800017F3FEFF6700A3644A8597A00000E78064
:102A9000E0C15C40EDD7DC4BFDD326858297C5B7FE
:102AA00017F3FEFFE70263602A8432859790FFFFE9
:102AB000E780A0E4AA85228597000000E780C0F7A0
:102AC00017F3FEFF6700A36017F3FEFFE702E35D65
:102AD0002A84AE8497000000E780C0FCA68522858A
:102AE00097000000E78060AD17F3FEFF6700235EEC
:102AF00008413355B5000589828017F3FEFFE702D0
:102B0000C35A1734FF1F1304E4291C5C0111231757
:102B100001008D83858BA303F1008327040B231809
:102B200001002319010003D7C7013ECA3C0023144A
:102B3000E1007D572315E1000357C4023ECC02CECD
:102B40002316E1009770FFFFE78020CE8357E10155
:102B5000231EA10093F707E093E71710231FF1004E
:102B60009737FF1F83C7A72695C305470145638A8B
:102B7000E7008347840393E727001737FF1F230FDE
:102B8000F724056117F3FEFF67006354814717F7C9
:102B90000000130767DB854613067100854548086A
:102BA00097900000E780408F69FD83478403F59B81
:102BB0001737FF1F2304F72285471737FF1F230806
:102BC000F720C1B717F3FEFFE702234B973DFF1F26
:102BD000938D4D1D03A6CD0639712A898147814405
:102BE000930600023357F600058B01C7850493F462
:102BF000F40F8507E398D7FE83A70D0B2317010277
